:020000040800F2
:100000000080002045CB0008F9730008FD7300084C
:10001000017400080574000809740008000000005D
:100020000000000000000000000000000D74000847
:10003000117400080000000015740008197400080D
:1000400095CB000895CB000895CB000895CB000810
:1000500095CB000895CB000895CB000895CB000800
:1000600095CB000895CB000895CB00081D740008BF
:100070002974000895CB0008357400084174000805
:1000800095CB0008000000004D74000895CB0008D7
:1000900095CB000895CB000895CB000895CB0008C0
:1000A00095CB000895CB000895CB000895CB0008B0
:1000B00095CB000895CB000895CB000895CB0008A0
:1000C00095CB000895CB000895CB000895CB000890
:1000D00095CB00086974000895CB000895CB000803
:1000E00095CB000895CB000895CB000895CB000870
:1000F00095CB000895CB000895CB000800000000C8
:100100000000000095CB00080000000095CB00081F
:1001100095CB00080000000095CB0008757400081E
:1001200095CB000895CB000895CB000895CB00082F
:1001300095CB0008000000000000000095CB0008EF
:1001400095CB000895CB00080000000000000000DF
:10015000000000000000000000000000000000009F
:1001600000000000000000000000000095CB000827
:1001700095CB000800000000000000000000000017
:100180000000000095CB0008000000000000000007
:10019000000000000000000000000000000000005F
:1001A000000000000000000095CB000895CB00087F
:1001B00095CB000895CB000895CB00080000000007
:1001C0000000000095CB00080000000000000000C7
:0801D00095CB000895CB000857
:100200000348044B834202D0034B03B118477047A5
:100210007007002070070020000000000548064914
:100220000B1AD90F01EBA301491002D0034B03B104
:10023000184770477007002070070020000000007A
:1002400010B5064C237843B9FFF7DAFF044B13B11E
:100250000448AFF300800123237010BD7007002015
:100260000000000098CB000808B5044B1BB10449FE
:100270000448AFF30080BDE80840CFE7000000006D
:100280007407002098CB000870B50D4E0D4D761BFD
:10029000B61006D0002455F8043B01349847A64216
:1002A000F9D1094E094D761B0CF076FCB61006D03C
:1002B000002455F8043B01349847A642F9D170BD9B
:1002C00058CF000858CF00085CCF000858CF00086E
:1002D000024B0146186800F059B900BF0000002029
:1002E000024B0146186800F0EFB800BF0000002084
:1002F000844641EA000313F003036DD1403A41D331
:1003000051F8043B40F8043B51F8043B40F8043BEF
:1003100051F8043B40F8043B51F8043B40F8043BDF
:1003200051F8043B40F8043B51F8043B40F8043BCF
:1003300051F8043B40F8043B51F8043B40F8043BBF
:1003400051F8043B40F8043B51F8043B40F8043BAF
:1003500051F8043B40F8043B51F8043B40F8043B9F
:1003600051F8043B40F8043B51F8043B40F8043B8F
:1003700051F8043B40F8043B51F8043B40F8043B7F
:10038000403ABDD2303211D351F8043B40F8043B1F
:1003900051F8043B40F8043B51F8043B40F8043B5F
:1003A00051F8043B40F8043B103AEDD20C3205D32F
:1003B00051F8043B40F8043B043AF9D2043208D027
:1003C000D2071CBF11F8013B00F8013B01D30B8899
:1003D00003806046704700BF082A13D38B078DD077
:1003E00010F003038AD0C3F10403D21ADB071CBF49
:1003F00011F8013B00F8013B80D331F8023B20F8B3
:10040000023B7BE7043AD9D3013A11F8013B00F8EB
:10041000013BF9D20B7803704B7843708B78837073
:1004200060467047830730B548D0541E002A3FD03D
:10043000CAB2034601E0013C3AD303F8012B9D0701
:10044000F9D1032C2DD9CDB245EA05250F2C45EA6B
:10045000054536D9A4F1100222F00F0C03F1200E4D
:10046000E6444FEA121C03F1100242E9045542E946
:10047000025510327245F8D10CF1010214F00C0F44
:1004800003EB021204F00F0C13D0ACF1040323F0C1
:1004900003030433134442F8045B9342FBD10CF092
:1004A00003042CB1CAB21C4403F8012B9C42FBD1BB
:1004B00030BD64461346002CF4D1F9E703461446D8
:1004C000BFE71A46A446E0E7002958D030B551F8F6
:1004D000043C83B0002BA1F10404B8BFE4180190E0
:1004E00000F07CF9284A0198136833B1A3420DD972
:1004F000216804EB010C63452FD06360146003B0E6
:10050000BDE8304000F06CB9A34210D81A465B68D1
:10051000002BF9D1116802EB010C644519D02FD3DF
:100520006360546003B0BDE8304000F059B9116811
:1005300002EB010CA44516D022D8216804EB010C73
:100540006345EDD11D685B682944C4E9001354601C
:10055000D5E7236819441160D1E71D685B68294419
:10056000C4E90013CAE7246821445418A342116067
:10057000C5D1D3E900432144C2E90013BFE7704766
:100580000C230360BBE700BF8C070020F8B5CD1C2F
:1005900025F0030508350C2D38BF0C25002D064627
:1005A00023DBA94221D8254F00F018F93A6822B37D
:1005B000144603E063682246FBB11C4623685B1BBC
:1005C000F8D40B2B15D8636894420CBF3B60536082
:1005D000304600F005F904F10B00231D20F0070060
:1005E000C21A01D01B1AA350F8BD0C23336000209F
:1005F000F8BD23601C442560EAE77968C9B1294643
:10060000304600F01DF8431C0CD0C41C24F0030439
:10061000A04205D0211A304600F012F8013001D076
:100620002560D5E70C233046336000F0D9F8002070
:10063000F8BD304600F004F87860E0E78C07002051
:1006400038B5074D0022044608462A6002F0D2FF62
:10065000431C00D038BD2B68002BFBD0236038BD75
:10066000940700200CB410B59CB01EAB6FF0004492
:10067000CDE906140291084953F8042B059102A90B
:100680000193049400F08CF9029B00221A701CB0B4
:10069000BDE8104002B070470802FFFF0EB410B56D
:1006A0009DB06FF000411FABCDE9060104910949EF
:1006B00053F8042B0290084C0868019302A9059492
:1006C00000F06EF9029B00221A701DB0BDE81040C8
:1006D00003B07047000000200802FFFF0000000088
:1006E000000000000000000000000000000000000A
:1006F00000000000000000000000000000000000FA
:1007000090F800F06DE9024520F007016FF0000C51
:1007100010F0070491F820F040F049804FF00004F9
:100720006FF00700D1E9002391F840F000F10800D4
:1007300082FA4CF2A4FA8CF283FA4CF3A2FA8CF30C
:100740004BBBD1E9022382FA4CF200F10800A4FA73
:100750008CF283FA4CF3A2FA8CF3E3B9D1E90423C7
:1007600082FA4CF200F10800A4FA8CF283FA4CF3FE
:10077000A2FA8CF37BB9D1E9062301F1200182FAB8
:100780004CF200F10800A4FA8CF283FA4CF3A2FABE
:100790008CF3002BC6D0002A04BF04301A4612BACC
:1007A000B2FA82F2FDE8024500EBD2007047D1E9CF
:1007B000002304F00305C4F100004FEAC50514F05E
:1007C000040F91F840F00CFA05F562EA05021CBF2F
:1007D00063EA050362464FF00004A9E7704700BFD3
:1007E000704700BF2DE9F0478F689F420C461D46B9
:1007F000164638D88246888910F4906F0ED1086862
:100800003D462A46314600F023FCA2682368D21BED
:100810002B44A26023600020BDE8F0874B69096982
:1008200003EB4308236808EBD878A3EB01096B1CA2
:100830004FEA68084B444345424684BF98464246C7
:10084000430513D511465046FFF7A0FE074608B3EF
:1008500021694A46FFF74CFDA38923F4906343F0D6
:100860008003A38107E008681F46CAE7504600F0EE
:100870006BFC074650B107EB0900A8EB09032761A1
:10088000C4F81480A36020602F46BAE7216950465F
:10089000FFF71AFE0C23CAF80030A38943F0400387
:1008A0004FF0FF30A381B7E72DE9F04F936883B095
:1008B0009146002B6ED017688D6880460C460868FC
:1008C000083744E0A38913F4906F2ED0D4E90415BF
:1008D000A0EB010A05EB450505EBD5750AEB060013
:1008E0006D100130A8422A4684BF05462A465B05A2
:1008F00037D511464046FFF749FE00283BD0524607
:1009000021690190FFF7F4FCA289019B22F4906217
:1009100042F08002A281A5EB0A0203EB0A006561A6
:10092000A260236120603546B2465946524600F027
:100930008FFBA068D9F808102368451B8E1B03EBBA
:100940000A00A5602060C9F808601EB3083757E99F
:1009500002B6002EFAD0B542AA46B3D93546B24601
:10096000E3E7404600F0F0FB03460028D3D12169BD
:100970004046FFF7A9FD0C23C8F80030A3890022E8
:1009800043F040034FF0FF30A381C9E9012203B0D7
:10099000BDE8F08F0020C9F8040003B0BDE8F08F77
:1009A0002DE9F04F92468A8915069DB0884681460A
:1009B0001C4603D50A69002A00F0EF800022099244
:1009C0009AF800307E4D039420228DF829203022A1
:1009D0008DF82A200126002B72D0544603E014F82B
:1009E000013F002B76D0252BF9D1B4EB0A0B74D143
:1009F0002278002A64D000234FF0FF32CDE905238E
:100A0000049307938DF853301A93013404E0049A49
:100A100006FA03F313430493A246052214F8011BBC
:100A2000284600F0C5FA431B0028F0D1049BD806E5
:100A300044BF20228DF8532019079AF8001044BFB4
:100A40002B228DF853202A2954D1039A116804329D
:100A5000002903927CDB07919AF801100AF1010A40
:100A60002E2959D0574C0322204600F0A1FA40B15C
:100A7000049B001B402404FA00F0034304930AF192
:100A8000010A1AF8011B50488DF82810062200F0C0
:100A90008FFA002862D04D4B002B52D003AA00924F
:100AA0004B4B424604A94846AFF3008007467A1CE8
:100AB00006D0099B3B4409939AF80030002B8CD157
:100AC000B8F80C305B0654BF09984FF0FF301DB0EA
:100AD000BDE8F08FB4EB0A0BF2D05B4652464146BC
:100AE0004846FFF77FFE0130EAD0099B22785B443D
:100AF00009937EE7A1F13002092AB1D8079B1AF8C1
:100B0000011F03EB830302EB4303A1F13002092A27
:100B1000F5D92E290793A5D19AF801102A2927D1B2
:100B2000039B9AF802101A6805920433002A0AF10E
:100B300002000393B8BF4FF0FF338246B8BF05935E
:100B400090E7039B073323F0070308330393B0E7D1
:100B5000494243F00203079104937DE703AA009200
:100B60001B4B424604A9484600F0CAF807469EE7D8
:100B7000A1F130020023092A05930AF1010A3FF688
:100B800071AF1AF8011F03EB830302EB4303A1F1DA
:100B90003002092AF5D9059364E74021FFF7F6FCF6
:100BA000C8F80000C8F8100018B14022C8F8142096
:100BB00004E70C23C9F800304FF0FF3087E700BF8F
:100BC00014CF00081CCF000820CF00080000000050
:100BD000E50700082DE9F84F92461F460A698B6821
:100BE000DDF828909A42B8BF1A46CAF8002091F85A
:100BF00043300C46064613B10132CAF80020226881
:100C000091065DD5DAF800300233CAF80030226868
:100C100012F0060F11461ED1E168CB1A002BD8BF87
:100C2000114618DD04F1190B4FF0000805E0E568E6
:100C3000DAF80030ED1A45450CDD01235A463946F5
:100C40003046C847013008F10108F0D14FF0FF30BD
:100C5000BDE8F88F216894F84330003B18BF0123AA
:100C60008A060AD5E1185A1C302081F84300224434
:100C700094F8451082F84310023304F143023946D8
:100C80003046C8470130E1D0236803F00603042B47
:100C90001DD0A3682269934225DD4FF000089B1AFE
:100CA00098441A34002501E045451CDA0123224608
:100CB00039463046C847013005F10105F4D1C5E792
:100CC00012F0060F12D0003B18BF0123D5E7DAF867
:100CD0000030E1682269C91AA368934221EAE178E9
:100CE000DDDC0029DDDC0020BDE8F88FE168DAF802
:100CF0000030CB1A002BD8BF114693DCABE700BF06
:100D00002DE9F0470C4684B09046227E0C990746A8
:100D1000994604F14300002A33D0A2F15803DDB212
:100D2000202D67D8202B65D8DFE813F0DE006400A3
:100D30006400640064006400640064006400640093
:100D40006400A3006E0064006400640064006E0030
:100D5000640064006400640021007F00C00064003F
:100D60006400AE0064007F0064006400E500236856
:100D70001A0640F104810B6862691D1D0D601B6835
:100D80001A60002382462361CDF80090434603AAEF
:100D900021463846FFF71EFF013020D02369524616
:100DA00041463846C847013019D02368E068039EA1
:100DB0009B0719D5831B002B16DD04F1190A0025AA
:100DC00004E0E068039E831BAB420DDD0123524625
:100DD00041463846C847013005F10105F1D14FF0D1
:100DE000FF3004B0BDE8F087B042B8BF304604B071
:100DF000BDE8F087012384F84220236104F1420A10
:100E0000002384F84330BFE723681A0602D45E0645
:100E100000F1C1800D682A6804350D601546002A6E
:100E20006BDBDFF884C10A2610E023681D0640F161
:100E30009C800B681D1D0D601D68DFF86CC16F2A5A
:100E40000CBF08260A26002384F843306268A2609B
:100E5000002A7FDB236823F004032360002D5BD18D
:100E6000002A79D18246082E65D0A0EB0A002061C5
:100E70008AE70B680122186804330B6004F1420A08
:100E800084F842002261BBE70B686268181D0860A5
:100E9000D3F800A00021504600F08AF8002800F0A6
:100EA0008180A0EB0A0060602061A9E7236843F01D
:100EB000200323607822DFF8F4C084F845200A6814
:100EC000151D0D601D0643D4590641D51588DE0752
:100ED00044BF43F020032360002D44D1236823F056
:100EE000200323601026AEE7582384F84530DFF84E
:100EF000B8C02368E3E72368DCE76268A2602D21BD
:100F0000002AC5F1000584F8431002DB23F0040336
:100F10002360DFF894C00A268246B5FBF6F306FB91
:100F200013512A461CF801100AF8011DB2421D4651
:100F3000F3D2082E99D12368D90796D56268236920
:100F40009A4292DC30230AF8013C0AF1FF3A8CE71E
:100F50001568BCE7002DDFD19CF8003084F84230E2
:100F600004F1420A7FE710266DE713F0400F0B688B
:100F700003F104050D600CBF1D681D885DE713F0CB
:100F8000400F0B68626903F104050D601B6814BF14
:100F90001A801A60F5E60A68B2F9005004320A6055
:100FA0002A463CE760687FE728CF00083CCF00086E
:100FB00001F0FF01102A2BDB10F0070F08D010F80A
:100FC000013B013A8B422DD010F0070F42B3F6D10E
:100FD000F0B441EA012141EA014122F007047FF027
:100FE00000070023F0E80256083C85EA010586EA7E
:100FF000010685FA47F5A3FA87F586FA47F6A5FABA
:1010000087F68EB9EED1F0BC01F0FF0102F00702C5
:1010100032B110F8013B013A83EA010313B1F8D170
:101020000020704701387047002D06BF3546033851
:10103000073815F0010F07D1013015F4807F02BF8A
:10104000013015F4C03F0130F0BC0138704700BFDB
:1010500088420DD98B1883420AD900EB020CBAB131
:10106000624613F801CD02F801CD9942F9D17047DB
:101070000F2A0ED8034602F1FF3C4AB10CF1010CD5
:10108000013B8C4411F8012B03F8012F6145F9D184
:10109000704740EA01039B0750D1A2F1100370B5DD
:1010A00001F1200C23F00F0501F1100E00F11004E6
:1010B000AC441B095EF8105C44F8105C5EF80C5CF4
:1010C00044F80C5C5EF8085C44F8085C5EF8045C6C
:1010D00044F8045C0EF1100EE64504F11004E9D169
:1010E000013312F00C0F01EB031102F00F0400EBBF
:1010F000031327D0043C24F003064FEA940C1E444B
:101100001C1F8E465EF8045B44F8045FB442F9D1BC
:101110000CF1010402F0030203EB840301EB8401F0
:1011200002F1FF3C4AB10CF1010C013B8C4411F877
:10113000012B03F8012F6145F9D170BD02F1FF3C8D
:1011400003469BE72246EBE7F8B51446F9B1CAB16E
:1011500006460D4600F020F8A04202D32F4638463E
:10116000F8BD21463046FFF711FA07460028F6D0B1
:1011700022462946FFF7BCF830462946FFF7A4F976
:101180003846F8BD2746FFF79FF93846F8BDBDE859
:10119000F8401146FFF7FAB951F8040C0028A0F105
:1011A0000400BCBF0B58C018704700BF000000000F
:1011B00051EC100B204A21F00043934220DD00B592
:1011C0001E4A934285B009DD10EE102A0B4602F04C
:1011D00023FA41EC100B05B05DF804FB684600F003
:1011E0001FFF00F0030001289DED021B9DED000B89
:1011F0000AD0022816D090B1012001F06DFFEAE775
:101200009FED0B1B01F000BA01F066FF53EC102BB1
:1012100003F1004300EE903A05B05DF804FB01F0E5
:10122000F3F9D8E701F0F0F9F0E700BFAFF3008081
:101230000000000000000000FB21E93FFFFFEF7FFE
:1012400051EC100B204A21F00043934227DD00B5FA
:101250001E4A934285B009DD10EE102A0B4602F0BB
:10126000DBF941EC100B05B05DF804FB684600F0BB
:10127000D7FE00F0030001289DED021B9DED000B41
:1012800012D0022817D090B101F0BEF953EC102B08
:1012900003F1004300EE903A05B05DF804FB9FEDCA
:1012A000081B002001F018BF01F0AEF9DBE70120B8
:1012B00001F012FFD7E7012001F00EFFE6E700BFC3
:1012C0000000000000000000FB21E93FFFFFEF7F6E
:1012D000F8B52DED028B57EC106B55EC114B00F06F
:1012E00003F9634BB0EE408AF0EE608A93F9003068
:1012F00001332AD022462B462046294602F0DEFD45
:1013000018BB32463B463046394602F0D7FD00282E
:1013100044D1002200233046394602F09DFDD8B169
:10132000002200232046294602F096FD00283DD1E8
:1013300045EC104B01F098FF38B1204629460022B9
:10134000002302F093FD00285CD1B0EE480AF0EED5
:10135000680ABDEC028BF8BDB0EE480AF0EE680AF0
:1013600001F082FF58B351EC180B0022002302F069
:1013700073FD0028E9D047EC106B01F075FF0028E1
:10138000E3D045EC104B01F06FFF0028DDD002F0F8
:10139000C5FF22239FED2E8B0360D6E7204629460A
:1013A0000022002302F058FD0028CED09FED2A8BAA
:1013B000B0EE480AF0EE680ABDEC028BF8BD47ECCF
:1013C000106B01F051FF0028CDD045EC104B01F01F
:1013D0004BFF0028C7D053EC182B18EE100A194603
:1013E00002F06CFD20BB02F099FF034622221A6036
:1013F000304639460022002302F038FD48B99FEDFF
:10140000188BA2E702F08AFF21239FED178B036060
:101410009BE745EC104B01F0BFFF224651EC100B4F
:101420002B4602F019FD0028E9D19FED0F8B8CE7C8
:1014300002F074FF002200232121016010461946AA
:1014400002F0CCFB41EC180B7FE700BFAFF300804C
:101450000000000000000000000000000000F03F5D
:10146000000000000000F07F000000000000F0FF1E
:101470006400002038B52DED028B55EC104B00F0C8
:10148000F5FF184BB0EE408AF0EE608A93F9003019
:1014900001330DD022462B462046294602F00EFD90
:1014A00030B9002200232046294602F0DFFC30B983
:1014B000B0EE480AF0EE680ABDEC028B38BD02F0CF
:1014C0002DFF00220023212101601046194602F061
:1014D00085FB41EC180BB0EE480AF0EE680ABDEC53
:1014E000028B38BD640000202DE9F04F57EC116BE2
:1014F0002DED0C8B27F0004A5AEA060287B03DD04A
:1015000055EC104B724925F00048884510EE102A22
:10151000A9462CDC11EE103ABB4636D08A4526DCB3
:101520006B498A4521D0B9F1000F39DB00210091C8
:10153000002B51D1664B9A4500F0A280654B9A452D
:1015400000F0B080BBF1804F00F0C084624B9B453F
:1015500042D1B9F1000F3FDB45EC104B07B0BDECB9
:101560000C8BBDE8F04F00F081BF002BDBD008F101
:10157000404808F5801858EA020309D19FED500B46
:1015800007B0BDEC0C8BBDE8F08F0CB9C245C7DDD0
:10159000524807B0BDEC0C8BBDE8F04F01F0F4BE33
:1015A0004F498A4500F38580A1F154718A450FDDCA
:1015B0004FEA2A51A1F2FF31142940F39B84C1F173
:1015C000340123FA01F000FA01F1994200F0ED84B0
:1015D00000210091002BB1D045EC104B029201F09C
:1015E00039FE029A5ABBB8F1000F04D0394B29F0EA
:1015F00040429A4223D1BBF1000F07DA53EC102B83
:101600003449002002F0EAFA41EC100BB9F1000F66
:10161000B6DA009B08F1404808F5801858EA030341
:1016200040F08D8453EC102B1046194601F0F4FF66
:1016300002460B4602F0D2FA41EC100BA0E7009AEA
:101640004FEAD973013B0493134335D0254B9A4598
:101650004CDD03F104739A45234B40F3DB8398453B
:1016600040F36083BBF1000F40F3608316A3D3E91E
:1016700000231046194602F087F941EC100B7FE772
:1016800008F1404303F5801313433FF477AF164B43
:10169000984540F37A83BBF1000FC0F2478347ECD3
:1016A000106B6DE7BBF1000FC0F21A8445EC104BD4
:1016B00066E7022100913BE722462B46B4E700BFD4
:1016C000000000000000F03F9C7500883CE4377E7D
:1016D0000000F07F0000F03F0000E03F38CF00083E
:1016E000FFFF3F430000E041FFFFEF3FE44B09EA0B
:1016F0000303002253B951EC100BE24B02F044F902
:1017000041EC100B10EE908A6FF034024FEA285330
:10171000A3F2FF339A18DC4B0592C8F3130848F084
:101720007F54984544F4401407DDD84B984540F366
:10173000148401320592A4F580149FEDB96B9FEDDE
:10174000BA7B53EC162BB0EE47CAF0EE67CA002501
:10175000B0EE47DAF0EE67DA5BEC10ABA34650462A
:10176000594643EC1A2B01F057FF53EC1A2B8046D5
:1017700089465046594601F051FF02460B4600206B
:10178000C34902F02BFA41EC1B0B404653EC1B2BD8
:10179000494602F0F9F841EC180B0A460146CDE93A
:1017A00002120021029164104BEC19AB44F000547A
:1017B000DDE902AB04F500230020591904460D466B
:1017C00002460B465046594602F0DEF802460B46EA
:1017D0004046494601F020FF53EC1A2B80468946CB
:1017E0002046294601F018FF02460B4651EC190B22
:1017F00001F012FF52465B4602F0C6F802460B4665
:101800004046494601F008FF53EC1B2B02F0BCF8A0
:1018100053EC182B41EC190B51EC180B02F0B4F8F7
:1018200083A3D3E9002304460D4602F0ADF882A35A
:10183000D3E9002301F0F2FE22462B4602F0A4F881
:101840007FA3D3E9002301F0E9FE22462B4602F0F4
:101850009BF87DA3D3E9002301F0E0FE22462B464E
:1018600002F092F87AA3D3E9002301F0D7FE2246D2
:101870002B4602F089F878A3D3E9002301F0CEFECD
:101880002246804689462B462046294602F07CF8AF
:1018900002460B464046494602F076F85246044658
:1018A0000D465B4651EC180B01F0B8FE53EC192BBA
:1018B00002F06AF822462B4601F0B0FE52468046FE
:1018C00089465B465046594602F05EF802460B4692
:1018D00043EC1A2B6F4B002201F0A0FE42464B4610
:1018E00001F09CFE00240D4622462B4650465946E8
:1018F00002F04AF8674B82468B4600222046294672
:1019000001F08AFE53EC1A2B01F086FE02460B46CC
:101910004046494601F080FE53EC182B02F034F8A3
:1019200022462B4604460D4651EC190B02F02CF8CA
:1019300002460B462046294601F070FE8046894645
:1019400042464B465046594601F068FE44A3D3E94F
:101950000023002004460D4602F016F8524641ECE2
:10196000190B5B462046294601F056FE02460B46FF
:101970004046494601F050FE3BA3D3E9002302F064
:1019800003F802460B462046294614461D4638A356
:10199000D3E9002301F0F8FF02460B462046294612
:1019A00001F03CFE53EC1D2B01F038FE80460598FB
:1019B000894601F07FFF424682468B464B4651ECFA
:1019C000190B01F02BFE53EC1C2B01F027FE5246A5
:1019D0005B4601F023FE52465B46002004460D465E
:1019E00001F01AFE53EC1C2B01F016FE53EC192BE0
:1019F00001F012FE02460B464046494601F00CFE3D
:101A0000009B049A013B134382468B4640F0B6810B
:101A10009FED197BB0EE478AF0EE678A3CE000BF8D
:101A2000000000000000F03F000000000000000087
:101A3000EF4E454A287ECA3F65DBC9934A86CD3FB3
:101A400001411DA96074D13F4D268F515555D53F99
:101A5000FFAB6FDBB66DDB3F033333333333E33F31
:101A6000000000E009C7EE3FFD033ADC09C7EE3F86
:101A7000F5015B14E02F3EBE000000000000F0BF47
:101A80000000F07F000040438E98030079B60B0001
:101A90000000F03F000008400023CDE900670093FC
:101AA000DDE90089304642464B46394601F0B4FD37
:101AB00022462B4601F068FF32463B4606460F465B
:101AC0005046594601F060FF02460B463046394603
:101AD00001F0A4FD42464B4606460F4620462946E5
:101AE00001F052FF04460D462B4630463946224649
:101AF00001F094FDC24B9942804689468A4640F3E4
:101B0000188101F13F4303F5E003034340F00782EE
:101B1000A3A3D3E900233046394601F07FFD0246F6
:101B20000B46404649469046994622462B4601F0D0
:101B300073FD02460B464046494602F0B5F90028BF
:101B400040F0ED81CAF30A534FF48012A3F2FE3342
:101B500042FA03F35344AB49C3F30A52A2F2FF32F1
:101B600041FA02FCC3F3130141F48011C2F11402E3
:101B700041FA02F2002023EA0C01BAF1000F0092B0
:101B80000B46024602DA0099494200912046294656
:101B900001F042FD009B1B05029302460B460446E2
:101BA0000D463046394601F039FD89464FF00008B0
:101BB0007DA3D3E900234046494601F0E5FE2246D5
:101BC0002B4682468B464046494601F025FD02469B
:101BD0000B463046394601F01FFD75A3D3E90023BB
:101BE00001F0D2FE74A3D3E9002304460D4640461B
:101BF000494601F0C9FE02460B462046294601F03F
:101C00000DFD06460F4632463B465046594601F00A
:101C100005FD52465B4604460D4601F0FDFC0246BA
:101C20000B463046394601F0F7FC2246804689468D
:101C30002B462046294601F0A7FE61A3D3E90023E5
:101C400006460F4601F0A0FE5FA3D3E9002301F092
:101C5000E3FC32463B4601F097FE5DA3D3E9002347
:101C600001F0DCFC32463B4601F08EFE5AA3D3E97C
:101C7000002301F0D1FC32463B4601F085FE58A31B
:101C8000D3E9002301F0CAFC32463B4601F07CFE5A
:101C900002460B462046294601F0BEFC06460F468A
:101CA00032463B462046294601F06EFE02460B4670
:101CB0003046394616461F4600224FF0804301F059
:101CC000ABFC02460B463046394601F087FF4246E0
:101CD00006460F464B462046294601F055FE424631
:101CE0004B4601F09BFC02460B463046394601F05C
:101CF00093FC22462B4601F08FFC02460B46002047
:101D0000414901F089FC029A0B461344B3F5801F48
:101D1000C0F24381194653EC182B01F035FE41EC1B
:101D2000100B2DE4BBF1000FFFF6A0AC9FED2E0BC6
:101D300026E4DFF8DCC021F00043634540F3E78090
:101D4000324B0B4403430AD122462B4601F064FC7C
:101D500032463B4602F09EF800283FF4F3AE24A33F
:101D6000D3E9002351EC180B01F00EFE20A3D3E9B8
:101D7000002301F009FE41EC100B01E49FED1E7BF6
:101D8000B0EE478AF0EE678A86E6BBF1000FCDDA47
:101D900007F1004300EE106A00EE903AFFF7F0BB47
:101DA000FE822B654715973C00000000432EE63F5E
:101DB000EF39FAFE422EE63F396CA80C615C20BE7A
:101DC000D0A4BE726937663EF16BD2C541BDBB3E41
:101DD0002CDE25AF6A56113F93BDBE166CC1663F1F
:101DE0003E5555555555C53F000000000000000008
:101DF00059F3F8C21F6EA501000000000000F03F7B
:101E0000FFFF8F40FFFF0F000000F03F00346F3FE7
:101E1000FFCB9040984585DB7D4B98453FF722AC42
:101E200051EC100B7A4B002201F0F6FB68A3D3E9CA
:101E3000002304460D4601F0A7FD67A3D3E9002364
:101E400082468B462046294601F09EFD714B41ECAF
:101E5000180B00222046294601F096FD02460B464B
:101E60005FA1D1E9000101F0D7FB22462B4601F02A
:101E70008BFD02460B460020674901F0CDFB224650
:101E8000804689462B462046294601F07DFD0246C4
:101E90000B464046494601F077FD53A3D3E90023A2
:101EA00001F072FD02460B4651EC180B01F0B4FB39
:101EB0008046894642464B465046594601F0AEFBA5
:101EC000002052465B4604460D4691E522462B46CD
:101ED0002046294601F058FD41EC100BFFF750BB9E
:101EE0004B49002022462B4601F078FE41EC100BB6
:101EF000FFF746BB002B44D1C1F114014AFA01F0AF
:101F000000FA01F151455AD00093FFF717BB424A3E
:101F100093425BDCDDE900120291009146E634A3B6
:101F2000D3E9002351EC180B01F02EFD30A3D3E9C7
:101F3000002301F029FD41EC100BFFF721BB009BB2
:101F4000012B7FF41DAB10EE901A10EE102A01F158
:101F5000004343EC102BFFF713BB9FED277BB0EE44
:101F600047CAF0EE67CA9FED267BB0EE47DAF0EE87
:101F700067DA9FED257B4FF4802553EC172BFFF795
:101F8000EBBB45EC104B009201F064F9009A002A7B
:101F90007FF492AB0092FFF726BB41EC100B009848
:101FA00001F096FA51EC100BB5E600F00100C0F11B
:101FB00002010091002B3FF4C1AAFFF70DBB00F016
:101FC0000100C0F102030093FFF7B8BA1B15BBE58F
:101FD000000000604715F73F44DF5DF80BAE543E4C
:101FE000555555555555D53FFE822B654715F73F3D
:101FF0009C7500883CE4377E0000004003B8E23F57
:1020000006D0CF43EBFD4C3E000000000000F83F3F
:102010000000F03F0000D03F0000E03F0000000063
:102020002DE9F04F53EC102B2DED048B904923F04C
:1020300000458D428BB0044640F38C808D498D4223
:102040001F462BDC002F194610EE100A7EA3D3E9A1
:10205000002340F3B68101F0DFFA874B9D428046B2
:10206000894600F08F807AA3D3E9002301F0D4FAE7
:1020700002460B46C4E900234046494601F0CCFA2B
:1020800073A3D3E9002301F0C7FAC4E902010126D2
:1020900030460BB0BDEC048BBDE8F08F77498D4224
:1020A00040F3928076498D4261DC2E15A6F21646E9
:1020B00010EE100AA5EB06519046894601F014FF78
:1020C00001F0F8FB02460B4640464946CDE90423A1
:1020D00001F0A2FA6B4B002201F056FC89468046C3
:1020E00001F002FF054601F0E5FB02460B464046C3
:1020F0004946CDE9062301F08FFA624B002201F038
:1021000043FC02460B46CDE908230022002301F0E0
:10211000A3FE002800F05381002D0CBF01230223F1
:10212000594A0192022200922146324604A800F048
:10213000ABFB002F0646ABDA6168226801F1004371
:10214000E168C4E90023A26801F10043C4E9022365
:1021500046429DE7002000210026C4E902013046E6
:1021600084ED000B0BB0BDEC048BBDE8F08F10EEDE
:10217000100A194601F050FA0026C4E90201C4E928
:10218000000185E734A3D3E9002301F045FA34A325
:10219000D3E900238046894601F03EFA02460B4609
:1021A000C4E900234046494601F036FA2CA3D3E99E
:1021B000002301F031FA0126C4E9020130460BB0D8
:1021C000BDEC048BBDE8F08F01F044F859EC108BA6
:1021D00010EE100A24A3D3E90023494601F0D4FBF2
:1021E0002A4B002201F01AFA01F07EFE064601F0A9
:1021F00061FB02460B4643EC182B13A3D3E90023E3
:10220000B0EE489AF0EE689A01F0BEFB02460B462B
:102210004046494601F000FA0DA3D3E90023824667
:102220008B4651EC180B01F0AFFB1F2E41EC180B45
:1022300030DC174B721E53F82230AB422AD00246D4
:102240000B469BE0AFF3008000004054FB21F93FB8
:102250003163621A61B4D03D0000601A61B4D03DB0
:102260007370032E8A19A33B83C8C96D305FE43FA6
:10227000FB21E93F7BD90240FB21F93FFB2139419A
:10228000FFFFEF7F0000704130CC00080000E03F0E
:10229000B0CB00082B150393504653EC182B59462E
:1022A00001F0BAF9C1F30A53C3EB1555102D80465E
:1022B000894669DD64A3D3E9002351EC190B01F0D1
:1022C00063FB8046894642464B465046594601F0DC
:1022D000A3F902460B465046594692469B4601F0EA
:1022E0009BF942464B4601F097F959A3D3E90023E5
:1022F0008046894651EC190B01F046FB42464B469D
:1023000001F08AF902460B465046594643EC182B19
:1023100001F082F9039AC1F30A53D31A312B804694
:10232000894631DD4DA3D3E9002351EC190B01F0AF
:102330002BFB8046894642464B465046594601F0A3
:102340006BF902460B465046594692469B4601F0B1
:1023500063F942464B4601F05FF942A3D3E90023FB
:102360008046894651EC190B01F00EFB42464B4664
:1023700001F052F902460B4643EC182B50465946E1
:1023800001F04AF98046894642464B46C4E9008935
:102390005046594601F040F953EC182B01F03CF936
:1023A000002FC4E90201BFF673AE09F10043C4E98E
:1023B000008301F10043C4E90203764268E6032387
:1023C000AEE601F02BF9244B9D428046894616D09B
:1023D0001BA3D3E9002301F021F902460B46C4E90F
:1023E00000234046494601F017F915A3D3E900231D
:1023F00001F014F94FF0FF36C4E9020148E612A3D8
:10240000D3E9002301F00AF911A3D3E900238046A0
:10241000894601F003F902460B46C4E90023404611
:10242000494601F0F9F80AA3D3E9002301F0F6F8D0
:102430004FF0FF36C4E902012AE600BFAFF3008087
:102440003163621A61B4D03D0000601A61B4D03DBE
:102450007370032E8A19A33BFB21F93F0000002E65
:102460008A19A33BC14920259A837B392DE9F04184
:10247000634A55EC104BAA4300F09F80002D10EEEC
:1024800010CA2B4654DD291563D0C3F31303A1F200
:10249000FF37C90743F4801304D45B0003EBDC73FC
:1024A0004FEA4C0C4FEADC72002602EB43037F102C
:1024B0004FEA4C0C4FF0160E34464FF40012A118A0
:1024C000994202DC5B1A8C1816445B00BEF1010EC7
:1024D00003EBDC734FEA52024FEA4C0CEFD1754626
:1024E00020204FF000420AE044D04FEADC7101386E
:1024F00001EB43034FEA4C0C4FEA520243D0A34294
:1025000002EB0E01F0DD002901EB020E0ADBA04612
:102510001B1B614588BF03F1FF33ACEB010C154475
:102520004446E2E7BEF1000FF1DB04F10108EFE7FA
:1025300025F00042224338D0002D4ED129464FEAE3
:10254000DC22153913464FEA4C5C002AF7D0D6023C
:1025500050D400205B00DD02044600F10100F9D5F3
:102560001A4663460CFA00FCC0F12000C340091B68
:1025700013438AE76145B8D8002901EB020ED1DB8D
:1025800098460023C9E753EA0C0310D1680871107C
:10259000F30701F17F5101F5001148BF40F0004001
:1025A00001EB0753024643EC102BBDE8F0816A1C97
:1025B00016BF681C01364008E9E710EE102A10EE3D
:1025C000100A2B46294601F0DFF922462B4601F07E
:1025D00025F841EC100BBDE8F08110EE102A2046E2
:1025E000294601F019F802460B4601F0F7FA41ECD2
:1025F000100BDAE7634620204FF0FF34B6E700BF48
:102600000000F07F000000002DE9F84F57EC106B40
:1026100027F00049B9F1795F2DED048B5BEC11AB2C
:1026200071DA10EE100A394601F05EFC002800F065
:10263000F68032463B463046394601F0A5F97CA388
:10264000D3E9002304460D4601F09EF97AA3D3E9AD
:10265000002300F0E3FF22462B4601F095F978A312
:10266000D3E9002300F0D8FF22462B4601F08CF975
:1026700075A3D3E9002300F0D1FF22462B4601F0D9
:1026800083F973A3D3E9002300F0C6FF22462B464B
:1026900001F07AF970A3D3E9002300F0BFFF2246CE
:1026A0002B4601F071F941EC180B714B00222046CA
:1026B000294601F069F953EC182B804689462046DB
:1026C000294601F061F952465B4604460D46304604
:1026D000394601F059F902460B462046294600F0DA
:1026E0009BFF02460B464046494600F095FF0246D6
:1026F0000B4600205F4900F08FFFBDEC048B41ECDE
:10270000100BBDE8F88F10EE102A10EE100A3B46B1
:10271000394601F039F946A3D3E9002304460D46B2
:1027200001F032F944A3D3E9002300F077FF2246F9
:102730002B4601F029F942A3D3E9002300F06CFFF6
:1027400022462B4601F020F93FA3D3E9002300F0F5
:1027500065FF22462B4601F017F93DA3D3E900237C
:1027600000F05AFF22462B4601F00EF93AA3D3E9B6
:10277000002300F053FF2B46224601F005F93E4BA3
:10278000994541EC180B90DD3C4B99453CDC00220F
:10279000A9F50013374900209046994600F03CFF08
:1027A00041EC190B324B00222046294601F0ECF88F
:1027B00042464B4600F030FF53EC182B80468946CA
:1027C0002046294601F0E0F852465B4604460D4695
:1027D0003046394601F0D8F802460B4620462946D5
:1027E00000F01AFF02460B464046494600F014FF2F
:1027F00002460B4651EC190B00F00EFFBDEC048BAA
:1028000041EC100BBDE8F88F9FED157BDFF8709061
:10281000B0EE479AF0EE679A4FF00008C2E7BDECC1
:10282000048B9FED110BBDE8F88F00BFAFF3008064
:10283000D43888BEE9FAA8BDC4B1B4BD9EEE213E2D
:10284000AD529C804F7E923E9015CB19A001FA3E6E
:102850007751C1166CC1563F4C5555555555A53F3E
:10286000000000000000E73F000000000000F03F13
:102870000000E03F0000F03F3233D33F0000E93F6B
:102880000000D23F000000002DE9F04FADF5197DAA
:102890001C4608930B91BA4BA299049053F821104F
:1028A0000591631E12F1140F0393C0F24B83B549D7
:1028B000D31E81FB0301DB17C3EBA1030793013395
:1028C000A3EB8303DB00D3180693079A039BD41A68
:1028D000059AD6181AD40136A39F264420AD4FF08E
:1028E00000084FF0000908E057F8240000F0E2FF6C
:1028F0000134B442E5E8020108D0002CF4DA0134D6
:1029000040464946B442E5E80201F6D1059B002B5A
:10291000C0F2C683089BDDF80C9020AA02EBC30A24
:10292000DA000292059A1A440192049A0DF5E07BAE
:1029300002EBC308039B002BC0F2A781049E5746FD
:102940000024002577E90223F6E8020101F01CF8D3
:1029500002460B462046294600F060FE46450446E6
:102960000D46EFD1019B09F101099945EBE80245BC
:102970000AF1080ADED1049A029B1344059A0192D7
:102980009B460BAB03EB82030A930CAB03EB820376
:10299000083B0993019A98AB03EBC203002A53E961
:1029A000284529DD0DF5E07A0AEBC2080DF1300962
:1029B000754B00222046294600F0E6FF01F094FA0C
:1029C00000F078FF714B002206460F4600F0DCFF56
:1029D00002460B462046294600F01EFE01F084FA0E
:1029E00078E9022349F8040B3946304600F016FE18
:1029F000D04504460D46DBD1DDF8189045EC104B70
:102A0000484600F065FD55EC104B00224FF07F5317
:102A100010EE100A294600F0B7FF41EC100B00F051
:102A20002FFC5B4B51EC100B002200F0ADFF024677
:102A30000B462046294600F0EFFD0D46044601F006
:102A400053FA804600F036FF0B46024629462046E0
:102A500000F0E2FD4B46002B06460F4640F39A80FD
:102A6000019A511E0CAAC9F1180352F8212042FA0A
:102A700003F000FA03F3D31AC9F117050CAA43FABD
:102A800005F5002D42F82130804400F38D800022AE
:102A900000233046394601F0DFF9002800F0598262
:102AA000019B059A03F1FF3A524510DC03F1804384
:102AB0000CAA013B0A9802EB8303002253F8041985
:102AC000834242EA0102F9D1002A40F0E180059BED
:102AD0000CAA013B52F82330002B40F0D180099A18
:102AE000012352F8041901330029FAD0019AD318AE
:102AF0000293531C9946019A08990A449046079AF2
:102B000002EB030A0AF1804AA39A0AF1FF3A02EBA8
:102B10008A0A20AA02EBC80870AA02EBC303019339
:102B20005AF8040F00F0C6FE0B460399024600292E
:102B3000C8E90023474608F108081EDB049E00246C
:102B4000002501E077E90223F6E8020100F01CFF0E
:102B500002460B462046294600F060FD5E450446CD
:102B60000D46EFD1019BE3E802450193029B09F179
:102B700001099945D4DD01930CE700240025F1E714
:102B800038CD0008ABAAAA2A0000703E00007041B0
:102B9000000020406BD1019B0CAA013B52F823504E
:102BA000ED15002D7FF773AF019B002B08F1010895
:102BB00040F3CD810C9C002C51D1019B012B20D0E6
:102BC0000CAB012253F8044F002C4BD0531C0CA922
:102BD000C4F1807441F822400199994210DD0CAA99
:102BE0000CA852F8232000EB830300EB81006FF068
:102BF0007F4100E01A688A1A43F8042B8342F9D116
:102C00000124069B002B0EDD012B00F06C81022BB2
:102C100009D1019B5A1E0CAB0CA953F82230C3F307
:102C2000150341F82230022D7FF431AF32463B4686
:102C3000B749002000F0F0FC06460F46002C3FF498
:102C400026AF06989FEDAE0B00F042FC30463946A9
:102C500053EC102B00F0E0FC06460F4617E701236B
:102C60000022B4E7019901328A42ABD1C9E7A94BEE
:102C7000002201F00FF9002840F05281054606E7D6
:102C8000019B01339946029335E70024002569E64C
:102C9000069B0395A3F118020CABCDF81C8053F8EA
:102CA0002A30069273B9019B03F18043023B0CA9C1
:102CB00001EB830353F804190AF1FF3A183A00298B
:102CC000F8D006929FED8E0B069800F001FCBAF149
:102CD000000F55EC104BC0F2D98170AB03EBCA0B5F
:102CE0000CAA0AF10103069302EB8306DFF828928F
:102CF0004FEACA0304930BF108074FF0000856F897
:102D0000040D00F0D7FD22462B4600F03DFE4B4659
:102D100067E9020142462046294600F035FE0CAB29
:102D20009E4204460D46EAD148ABCDE9013ADDF8B2
:102D300014A0BAF1000F4FF000092CDB72A3D3E905
:102D40000023DFF8D8815F4600260024002503E039
:102D5000B14510DBF8E80223F7E8020100F014FEA9
:102D600002460B462046294600F058FC0136B24583
:102D700004460D46ECDA019B029A03EBC9034A456F
:102D8000C3E90045ABF1080B09F1010306D0BAF124
:102D9000000F9946D2DA00240025ECE7A29BDDF86B
:102DA00008A0022B1EDC002B00F3098113D1049C28
:102DB000019D08342C440020002174E9022300F016
:102DC0002DFCA542F9D1039B13B101F10043194633
:102DD0000B9BC3E90001079B03F007000DF5197D6C
:102DE000BDE8F08FA29B032BF5D1BAF1000F00F0E4
:102DF0006981019A049BD318D3E9004502EBCA0B01
:102E00007BE902672046294632463B4600F006FC35
:102E1000A046A94604460D4622462B463046394672
:102E200000F0FAFB4B46424600F0F8FB019B5B4585
:102E3000CBE90201CBE90045E2D1BAF1010F40F341
:102E40004181019A049B0AF1005A0AF1FF3A1344A6
:102E50004FEACA01D3E9004501F1080A0291924400
:102E60000DF5947B7AE902672046294632463B46B7
:102E700000F0D4FBA046A94604460D4622462B4648
:102E80003046394600F0C8FB42464B4600F0C6FBD0
:102E9000D345CAE90201CAE90045E3D1029C019B7E
:102EA00010341C4403F110050020002174E90223B2
:102EB00000F0B4FBA542F9D1039B002B40F0BD808C
:102EC0000B9CC4E904010198D0E90023C4E9002364
:102ED000D0E90223C4E90223079B03F007000DF5A4
:102EE000197DBDE8F08F019B5A1E0CAB0CA953F85D
:102EF0002230C3F3160341F8223094E6AFF300808A
:102F0000000000000000F03F00000040FB21F93FFE
:102F10000000F03F0000E03F0000703E50CD000890
:102F2000019B002B08F10108C8BF02253FF742AE04
:102F300032463B466549002000F06EFB02250646FE
:102F40000F46A4E500216FF017030791BBE40024AE
:102F500057E647EC106B069E03957042CDF81C8037
:102F600000F0B6FA55EC104B594B10EE100A002247
:102F7000294600F08FFF002855D0564B019F0022B4
:102F8000183620462946069600F0FEFC00F0ACFFFD
:102F9000064600F08FFC4E4B002200F0F5FC0B467D
:102FA00002462946204600F037FB00F09DFF07F15E
:102FB000010A0CAB43F8270043F82A6082E6019D22
:102FC000069B002005EBC304002174E9022300F0F6
:102FD00025FBA542F9D1039B002B47D10B9BC3E9ED
:102FE00000010B4601990246D1E9000100F014FBF3
:102FF000BAF1000F0DDD4AAD0124F5E802230134DA
:1030000000F00CFBA245F8DA039B13B101F1004379
:1030100019460B9BC3E90201079B03F007000DF55E
:10302000197DBDE8F08F2046294600F05DFF019B29
:103030000CAA9A4642F8230044E6019E01F100439F
:1030400074680B993268F568C1E9040304F1004320
:10305000C1E90023B26805F10043C1E90223079BDF
:1030600003F007000DF5197DBDE8F08F0B9A01F113
:10307000004353600B46019910600246D1E90001FC
:1030800000F0CAFABAF1000FB5DCBFE7A29B022B31
:103090000ADC002B11DC7FF49EAE0020002192E6BA
:1030A000089BDB00029366E4A29B032B7FF493AEA4
:1030B00048AB002000210193FEE648AB0020002130
:1030C000019388E700200021F6E600BF0000F03FF2
:1030D000000070410000703E2DE9F04F55EC104BA0
:1030E00085B025F00043B3F1795F8DED001B0390AF
:1030F00007DA10EE100A294600F0F6FE002800F06C
:10310000898022462B462046294600F03DFC064693
:103110000F4632463B462046294600F035FC43A385
:10312000D3E9002382468B463046394600F02CFC1A
:1031300040A3D3E9002300F06FFA32463B4600F08B
:1031400023FC3EA3D3E9002300F068FA32463B4655
:1031500000F01AFC3BA3D3E9002300F05DFA3246ED
:103160003B4600F011FC39A3D3E9002300F056FAE6
:10317000039B80468946ABB3DDE900012A4B002260
:1031800000F002FC42464B4680468946504659466E
:1031900000F0FAFB02460B464046494600F03CFA76
:1031A00032463B4600F0F0FBDDE9002300F034FA44
:1031B0001BA3D3E9002306460F465046594600F0AC
:1031C000E3FB02460B463046394600F027FA02463A
:1031D0000B462046294600F01FFA41EC100B05B0C3
:1031E000BDE8F08F02460B463046394600F0CCFB76
:1031F0000BA3D3E9002300F00FFA52465B4600F020
:10320000C3FB22462B4600F009FA41EC100B05B037
:10321000BDE8F08F45EC104B05B0BDE8F08F00BF66
:10322000495555555555C53F0000E03F7CD5CF5A0F
:103230003AD9E53DEB9C2B8AE6E55A3E7DFEB15737
:10324000E31DC73ED561C119A0012A3FA6F81011A0
:103250001111813F51EC100B10EE102A21F00043A8
:1032600043EC102B704700BF82B08DED000B01982E
:1032700040F0004000F58010C00F02B0704700BF62
:1032800051EC100BF8B5C1F30A53A3F2FF35132D1F
:1032900010EE106A0C4630DC002D1EDB384F2F413B
:1032A00001EA070303432DD033A3D3E9002300F041
:1032B000B5F90022002300F0F7FD48B1002C04DA34
:1032C0004FF4801343FA05F52C4424EA0704002642
:1032D0002346324643EC102BF8BD27A3D3E9002345
:1032E00000F09CF90022002300F0DEFD0028EFD062
:1032F000002C29DB00263446EAE7332D05DDB5F541
:10330000806F19D041EC100BF8BDA3F213434FF0BE
:10331000FF37DF400742F5D017A3D3E9002300F0C1
:103320007DF90022002300F0BFFD0028D0D0002C42
:1033300013DB26EA0706CBE710EE102A0B4600F057
:103340006DF941EC100BF8BD24F000430D4A1E430B
:10335000002E18BF14460026BAE7142D08D001230A
:10336000C5F1340503FA05F5AE1928BFE418E0E706
:103370000134DEE7AFF300809C7500883CE4377EC3
:10338000FFFF0F000000F0BF9FED010B704700BF73
:10339000000000000000F87FF0B553EC102BC3F3E1
:1033A0000A5CACF2FF31132910EE100A83B01C4600
:1033B0004FEAD37E3ADC002930DB424D45FA01FC6E
:1033C00003EA0C0515432DD003EA5C0318434FEACA
:1033D0005C0C0CD024EA0C0C4FF48024132944FA22
:1033E00001F10CBF4FF0004000204CEA01043649C7
:1033F00001EBCE0E2346DEE9004502462946204673
:1034000000F00CF9CDE90001DDE9000122462B4670
:1034100000F002F941EC100B03B0F0BD23F00041C5
:10342000114324D143EC102B03B0F0BD332908DD48
:10343000B1F5806FF6D1194600F0F0F841EC100BB1
:10344000F2E7ACF2134C4FF0FF3121FA0CF10A42D3
:10345000E8D010EA51024FEA5103C8D020EA030332
:103460004FF0804040FA0CFC43EA0C00BFE7C3F386
:1034700013031843144A4342034302EBCE0E1B0BC3
:10348000620C03F40023520443EA02073B46DEE9E0
:10349000006710EE102A3046394600F0BFF8CDE93B
:1034A000000132463B46DDE9000100F0B5F804F0CA
:1034B000004421F00041024641EA040343EC102B92
:1034C00003B0F0BDFFFF0F0088CD00080000000032
:1034D00038B553EC102BC3F30A5104469C4689BB04
:1034E00010EE101A23F0004C5CEA010129D01946B5
:1034F00000223D4B3D4D10EE100A00F045FAAC4263
:1035000002460B4616DB8C46C1F30A51363921447C
:1035100040F2FE70814221DC002947DC11F1350FB9
:1035200034DA4CF250318C4218DC002B26A1D1E960
:10353000000144DB24A3D3E9002300F025FA41EC89
:10354000100B38BD40F2FF708142E0D110EE100A3E
:10355000194600F063F841EC100B38BD002B1CA19C
:10356000D1E9000107DB1AA3D3E9002300F00CFA2C
:1035700041EC100B38BD18A1D1E9000114A3D3E927
:10358000002300F001FA41EC100BF3E72CF0FF4CA4
:103590002CF4E00C36314CEA015310461946002257
:1035A000134B00F0F1F941EC100B38BD2CF0FF4C3F
:1035B0002CF4E00C4CEA015343EC102B38BD08A16D
:1035C000D1E90001B6E700BF59F3F8C21F6EA501AB
:1035D0009C7500883CE4377E9C7500883CE437FE8F
:1035E00059F3F8C21F6EA58100005043B03CFFFFA5
:1035F0000000903C044A05491368002B08BF0B46A5
:103600001844106018467047980700205053002057
:1036100081F0004102E000BF83F0004330B54FEA83
:1036200041044FEA430594EA050F08BF90EA020FF0
:103630001FBF54EA000C55EA020C7FEA645C7FEA83
:10364000655C00F0E2804FEA5454D4EB5555B8BFA6
:103650006D420CDD2C4480EA020281EA030382EA17
:10366000000083EA010180EA020281EA0303362DA9
:1036700088BF30BD11F0004F4FEA01314FF4801C7C
:103680004CEA113102D0404261EB410113F0004F8E
:103690004FEA03334CEA133302D0524263EB430345
:1036A00094EA050F00F0A780A4F10104D5F1200EE3
:1036B0000DDB02FA0EFC22FA05F2801841F100013E
:1036C00003FA0EF2801843FA05F359410EE0A5F112
:1036D00020050EF1200E012A03FA0EFC28BF4CF043
:1036E000020C43FA05F3C01851EBE37101F00045F9
:1036F00007D54FF0000EDCF1000C7EEB00006EEB06
:103700000101B1F5801F1BD3B1F5001F0CD349088F
:103710005FEA30004FEA3C0C04F101044FEA4452E6
:1037200012F5800F80F09A80BCF1004F08BF5FEA6D
:10373000500C50F1000041EB045141EA050130BD4D
:103740005FEA4C0C404141EB0101013C28BFB1F55F
:10375000801FE9D291F0000F04BF01460020B1FAAA
:1037600081F308BF2033A3F10B03B3F120020CDA7D
:103770000C3208DD02F1140CC2F10C0201FA0CF05B
:1037800021FA02F10CE002F11402D8BFC2F1200CC0
:1037900001FA02F120FA0CFCDCBF41EA0C01904076
:1037A000E41AA2BF01EB0451294330BD6FEA0404BF
:1037B0001F3C1CDA0C340EDC04F11404C4F12002AA
:1037C00020FA04F001FA02F340EA030021FA04F3BC
:1037D00045EA030130BDC4F10C04C4F1200220FA13
:1037E00002F001FA04F340EA0300294630BD21FA51
:1037F00004F0294630BD94F0000F83F4801306BF17
:1038000081F480110134013D4EE77FEA645C18BF0A
:103810007FEA655C29D094EA050F08BF90EA020FA1
:1038200005D054EA000C04BF1946104630BD91EA99
:10383000030F1EBF0021002030BD5FEA545C05D19C
:103840004000494128BF41F0004130BD14F58004DB
:103850003CBF01F5801130BD01F0004545F0FE414F
:1038600041F470014FF0000030BD7FEA645C1ABF84
:10387000194610467FEA655C1CBF0B46024650EABB
:10388000013406BF52EA033591EA030F41F40021E7
:1038900030BD00BF90F0000F04BF0021704730B56D
:1038A0004FF4806404F132044FF000054FF0000142
:1038B00050E700BF90F0000F04BF0021704730B503
:1038C0004FF4806404F1320410F0004548BF4042D8
:1038D0004FF000013EE700BF42004FEAE2014FEA2D
:1038E00031014FEA02701FBF12F07F4393F07F4F08
:1038F00081F06051704732F07F4208BF704793F00B
:103900007F4F04BF41F40021704730B54FF460741D
:1039100001F0004521F000411CE700BF50EA010220
:1039200008BF704730B54FF000050AE050EA0102C9
:1039300008BF704730B511F0004502D5404261EB39
:1039400041014FF4806404F132045FEA915C3FF47A
:10395000D8AE4FF003025FEADC0C18BF03325FEA17
:10396000DC0C18BF033202EBDC02C2F1200300FAC8
:1039700003FC20FA02F001FA03FE40EA0E0021FAED
:1039800002F11444BDE600BF70B54FF0FF0C4CF4DB
:10399000E06C1CEA11541DBF1CEA135594EA0C0F8D
:1039A00095EA0C0F00F0DEF82C4481EA030621EAC8
:1039B0004C5123EA4C5350EA013518BF52EA033503
:1039C00041F4801143F4801338D0A0FB02CE4FF0B5
:1039D0000005E1FB02E506F00042E0FB03E54FF0E5
:1039E0000006E1FB03569CF0000F18BF4EF0010EDD
:1039F000A4F1FF04B6F5007F64F5407404D25FEAD9
:103A00004E0E6D4146EB060642EAC62141EA55518B
:103A10004FEAC52040EA5E504FEACE2EB4F1FD0CCD
:103A200088BFBCF5E06F1ED8BEF1004F08BF5FEA4B
:103A3000500E50F1000041EB045170BD06F00046FD
:103A400046EA010140EA020081EA0301B4EB5C04AA
:103A5000C2BFD4EB0C0541EA045170BD41F48011A2
:103A60004FF0000E013C00F3AB8014F1360FDEBFC7
:103A7000002001F0004170BDC4F10004203C35DAA3
:103A80000C341BDC04F11404C4F1200500FA05F326
:103A900020FA04F001FA05F240EA020001F00042C7
:103AA00021F0004110EBD37021FA04F642EB06013D
:103AB0005EEA430E08BF20EAD37070BDC4F10C0467
:103AC000C4F1200500FA04F320FA05F001FA04F22B
:103AD00040EA020001F0004110EBD37041F1000117
:103AE0005EEA430E08BF20EAD37070BDC4F1200522
:103AF00000FA05F24EEA020E20FA04F301FA05F28A
:103B000043EA020321FA04F001F0004121FA04F231
:103B100020EA020000EBD3705EEA430E08BF20EA01
:103B2000D37070BD94F0000F0FD101F0004640003B
:103B300041EB010111F4801F08BF013CF7D041EABD
:103B4000060195F0000F18BF704703F000465200C1
:103B500043EB030313F4801F08BF013DF7D043EA92
:103B60000603704794EA0C0F0CEA135518BF95EA48
:103B70000C0F0CD050EA410618BF52EA4306D1D1CF
:103B800081EA030101F000414FF0000070BD50EAEE
:103B9000410606BF1046194652EA430619D094EA78
:103BA0000C0F02D150EA013613D195EA0C0F05D162
:103BB00052EA03361CBF104619460AD181EA0301B6
:103BC00001F0004141F0FE4141F470014FF000006E
:103BD00070BD41F0FE4141F4780170BD70B54FF009
:103BE000FF0C4CF4E06C1CEA11541DBF1CEA135589
:103BF00094EA0C0F95EA0C0F00F0A7F8A4EB05046B
:103C000081EA030E52EA03354FEA013100F0888061
:103C10004FEA03334FF0805545EA131343EA12632A
:103C20004FEA022245EA111545EA10654FEA0026DF
:103C30000EF000419D4208BF964244F1FD0404F598
:103C4000407402D25B084FEA3202B61A65EB0305F4
:103C50005B084FEA32024FF480104FF4002CB6EBB1
:103C6000020E75EB030E22BFB61A754640EA0C0031
:103C70005B084FEA3202B6EB020E75EB030E22BF71
:103C8000B61A754640EA5C005B084FEA3202B6EBB2
:103C9000020E75EB030E22BFB61A754640EA9C0071
:103CA0005B084FEA3202B6EB020E75EB030E22BF41
:103CB000B61A754640EADC0055EA060E18D04FEAFF
:103CC000051545EA16754FEA06164FEAC30343EA9F
:103CD00052734FEAC2025FEA1C1CC0D111F4801F6C
:103CE0000BD141EA00014FF000004FF0004CB6E765
:103CF00011F4801F04BF01430020B4F1FD0C88BF04
:103D0000BCF5E06F3FF6AFAEB5EB030C04BFB6EB0E
:103D1000020C5FEA500C50F1000041EB045170BD01
:103D20000EF0004E4EEA113114EB5C04C2BFD4EB2E
:103D30000C0541EA045170BD41F480114FF0000EB2
:103D4000013C90E645EA060E8DE60CEA135594EA2E
:103D50000C0F08BF95EA0C0F3FF43BAF94EA0C0F31
:103D60000AD150EA01347FF434AF95EA0C0F7FF4A6
:103D700025AF104619462CE795EA0C0F06D152EAFA
:103D800003353FF4FDAE1046194622E750EA4106DE
:103D900018BF52EA43067FF4C5AE50EA41047FF4EF
:103DA0000DAF52EA43057FF4EBAE12E74FF0FF3C54
:103DB00006E000BF4FF0010C02E000BF4FF0010C25
:103DC0004DF804CD4FEA410C7FEA6C5C4FEA430C9E
:103DD00018BF7FEA6C5C1BD001B050EA410C0CBFED
:103DE00052EA430C91EA030F02BF90EA020F00204F
:103DF000704710F1000F91EA030F58BF994208BFB6
:103E000090422CBFD8176FEAE37040F00100704772
:103E10004FEA410C7FEA6C5C02D150EA013C07D1C9
:103E20004FEA430C7FEA6C5CD6D152EA033CD3D014
:103E30005DF8040B704700BF8446104662468C460E
:103E40001946634600E000BF01B5FFF7B7FF002841
:103E500048BF10F1000F01BD4DF808EDFFF7F4FF6A
:103E60000CBF012000205DF808FB00BF4DF808EDF5
:103E7000FFF7EAFF34BF012000205DF808FB00BF18
:103E80004DF808EDFFF7E0FF94BF012000205DF83A
:103E900008FB00BF4DF808EDFFF7CEFF94BF0120EF
:103EA00000205DF808FB00BF4DF808EDFFF7C4FFE8
:103EB00034BF012000205DF808FB00BF4FEA410C31
:103EC0007FEA6C5C02D150EA013C0AD14FEA430C14
:103ED0007FEA6C5C02D152EA033C02D14FF0000051
:103EE00070474FF0010070474FEA410212F500128F
:103EF00015D211D56FF47873B3EB625212D94FEA31
:103F0000C12343F0004343EA505311F0004F23FA1A
:103F100002F018BF404270474FF00000704750EA6F
:103F2000013005D111F0004008BF6FF0004070472C
:103F30004FF00000704700BF4A0011D212F5001286
:103F400011D20DD56FF47873B3EB62520ED44FEAF1
:103F5000C12343F0004343EA505323FA02F0704771
:103F60004FF00000704750EA013002D14FF0FF30AF
:103F700070474FF0000070477BB972B90029BEBF8F
:103F800000204FF0004106E008BF00281CBF6FF082
:103F900000414FF0FF3000F0BFB9ADF1080C6DE902
:103FA00004CE002909DB002B1ADB00F04DF8DDF808
:103FB00004E0DDE9022304B07047404261EB4101B7
:103FC000002B1BDB00F040F8DDF804E0DDE9022304
:103FD00004B0404261EB4101524263EB430370473E
:103FE000524263EB430300F02FF8DDF804E0DDE913
:103FF000022304B0404261EB41017047524263EB3F
:10400000430300F021F8DDF804E0DDE9022304B009
:10401000524263EB4303704753B94AB9002908BFC2
:1040200000281CBF4FF0FF314FF0FF3000F074B993
:10403000ADF1080C6DE904CE00F006F8DDF804E0FF
:10404000DDE9022304B070472DE9F047089D0446DE
:104050008E46002B4DD18A42944669D9B2FA82F23B
:1040600052B101FA02F3C2F1200120FA01F10CFA77
:1040700002FC41EA030E94404FEA1C48210CBEFBAF
:10408000F8F61FFA8CF708FB16E341EA034306FB38
:1040900007F199420AD91CEB030306F1FF3080F0C7
:1040A0001F81994240F21C81023E63445B1AA4B214
:1040B000B3FBF8F008FB103344EA034400FB07F7B6
:1040C000A7420AD91CEB040400F1FF3380F00A81F7
:1040D000A74240F207816444023840EA0640E41BEC
:1040E00000261DB1D4400023C5E900433146BDE898
:1040F000F0878B4209D9002D00F0EF800026C5E93A
:10410000000130463146BDE8F087B3FA83F6002E51
:104110004AD18B4202D3824200F2F980841A61EBC9
:10412000030301209E46002DE0D0C5E9004EDDE7E7
:1041300002B9FFDEB2FA82F2002A40F09280A1EBCF
:104140000C014FEA1C471FFA8CFE0126200CB1FB24
:10415000F7F307FB131140EA01410EFB03F088421D
:1041600008D91CEB010103F1FF3802D2884200F2AA
:10417000CB804346091AA4B2B1FBF7F007FB10113C
:1041800044EA01440EFB00FEA64508D91CEB0404DA
:1041900000F1FF3102D2A64500F2BB800846A4EB35
:1041A0000E0440EA03409CE7C6F12007B34022FA20
:1041B00007FC4CEA030C20FA07F401FA06F31C434F
:1041C000F9404FEA1C4900FA06F3B1FBF9F8200C5C
:1041D0001FFA8CFE09FB181140EA014108FB0EF0A2
:1041E000884202FA06F20BD91CEB010108F1FF3AF2
:1041F00080F08880884240F28580A8F102086144FE
:10420000091AA4B2B1FBF9F009FB101144EA01410B
:1042100000FB0EFE8E4508D91CEB010100F1FF34B6
:104220006CD28E456AD90238614440EA0840A0FB4E
:104230000294A1EB0E01A142C846A64656D353D024
:104240005DB1B3EB080261EB0E0101FA07F722FA48
:1042500006F3F1401F43C5E9007100263146BDE871
:10426000F087C2F12003D8400CFA02FC21FA03F3D4
:10427000914001434FEA1C471FFA8CFEB3FBF7F055
:1042800007FB10360B0C43EA064300FB0EF69E427A
:1042900004FA02F408D91CEB030300F1FF382FD213
:1042A0009E422DD9023863449B1B89B2B3FBF7F6BB
:1042B00007FB163341EA034106FB0EF38B4208D994
:1042C0001CEB010106F1FF3816D28B4214D9023ED5
:1042D0006144C91A46EA004638E72E46284605E7F3
:1042E0000646E3E61846F8E64B45A9D2B9EB0208C4
:1042F00064EB0C0E0138A3E74646EAE7204694E754
:104300004046D1E7D0467BE7023B614432E7304686
:1043100009E76444023842E7704700BF014B186860
:10432000704700BF000000200368B3F1A04F00D029
:104330007047024B01221A70704700BF780F0020AF
:104340000368B3F1A04F00D07047024B01221A60FE
:10435000704700BF981B00200349044B0020012236
:1043600008701A70704700BF8C1B00207408002072
:104370000249034A01230B70137070478C1B002005
:10438000740800200349044B0020012208701A70B1
:10439000704700BF053F0020F83E00200249034A55
:1043A00001230B7013707047053F0020F83E00207A
:1043B000044B02689A4200D07047034B01221A70E6
:1043C000704700BF00140040790F002038B5084B3B
:1043D000984200D038BD074D0446287800F084FD8F
:1043E000294620460122BDE8384007F0B9B800BF91
:1043F000E80E0020E43C002000B50F4B012283B002
:104400001A7002F0D7FA0D4B1B68033B012B02D93F
:1044100003B05DF804FB0A4806F0F2FD00210948EC
:1044200005F008FD0021084A00918023054805F0A9
:1044300049FD03B05DF804FBE31C0020941B002041
:10444000040E0020A00800208C1900200C4B10B591
:1044500000241C7002F090FA0A4B1B68033B012BEE
:1044600000D910BD084806F0FFFD2146074805F0B9
:1044700017FD21460548BDE8104005F0A9BD00BF65
:10448000E31C0020941B0020040E0020A008002044
:1044900010B50E4B0E490F4C0F4882B04FF0010C77
:1044A0004FF4806283F800C004F0BEF90B4806F0B8
:1044B000A7FD0021204605F0BDFC0021084A00911F
:1044C0008023204605F0FEFC02B010BDA01C002099
:1044D0007C0F0020A00800209C070020040E002074
:1044E0008C19002038B50A4B0A4D0B4800241C706B
:1044F00004F050FA094806F0B7FD2146284605F0B9
:10450000CFFC21462846BDE8384005F061BD00BF1C
:10451000A01C0020A00800209C070020040E002002
:1045200008B5184806F0C8FC174B1B68023B042B63
:1045300024D8DFE803F00F14191E0300114B4FF4C9
:10454000A0329A620F4806F017FCBDE808400D48FB
:1045500006F09ABC0B4B4FF480429A62F2E7094B8B
:104560004FF400429A62EDE7064B4FF440429A62E4
:10457000E8E7044B4FF480329A62E3E7014B0022F4
:104580009A62DFE7940A0020CC1C002000000000A3
:1045900000B595B03822002106A8FBF743FF0020A4
:1045A000CDE90000CDE90200049005F0EFFA9FED9F
:1045B0001A7B022301210322CDE90C130E921C2148
:1045C000062206A88DED067BCDE90F31CDE911322B
:1045D000139304F0F1FA08B172B6FEE79FED107B79
:1045E0008DED007B9FED107B0346042168468DED29
:1045F000027B049304F08EFD08B172B6FEE702461A
:104600004FF080614FF4807004F022FD15B05DF82A
:1046100004FB00BFAFF30080210000000000010098
:104620000F00000003000000000000000000000078
:104630002DE98048BA4CBB4EBB4F9FB0002525806A
:1046400004F086FAFFF7A4FFCDE91255CDE9145521
:104650001695F36C43F02003F364F36C03F020032E
:104660000493049BF36C43F00103F364F36C03F0D5
:1046700001030593059BF36C43F00203F364F36CB1
:1046800003F0020306932A464FF400414FF0904096
:10469000069B05F0BFF8A5482A46382105F0BAF870
:1046A0004FF002080522002312A94FF09040CDE9F7
:1046B0001223CDF8508004F0B5FF4FF4807202232E
:1046C000CDE9122312A9002200234FF09040CDE93A
:1046D00014234FF0020A4FF0000B169504F0A2FFCE
:1046E0004FF40042012312A94FF09040CDE912236C
:1046F000CDE914AB04F096FF382201238B4812A9B0
:10470000CDE91223CDE914AB04F08CFF4022002345
:104710008648CDF8508012A9CDE9122304F082FF1B
:10472000B36C43F00403B364B36C03F0040302936B
:10473000029BB36C43F00103B364B36C03F0010359
:104740002A46294603930B20039B05F0B7FA0B205A
:1047500005F0F2FA2A4629460C2005F0AFFA0C20A3
:1047600005F0EAFA2A4629460E2005F0A7FA0E209F
:1047700005F0E2FA2A4629460F2005F09FFA0F209D
:1047800005F0DAFA2946302212A8FBF74BFE684BF7
:104790003B60384605F038FB08B172B6FEE71E23D1
:1047A000CDE91600CDF848801490199002464FF4D8
:1047B00080784FF0010912A938461593ADF84C8066
:1047C000CDF8609005F050FC034608B172B6FEE7E4
:1047D0003846102212A98DF84D30159305F044FC8F
:1047E000054608B172B6FEE7524E0790CDE90800C3
:1047F000CDE90B00CDE90D00CDE90F000A9001468F
:10480000202212A8FBF70EFE4FF0A0474FF44033D2
:10481000C6E90073A6F81C8004233046C6E9025599
:10482000C6E90455C6E90B55C6E91155C6F82090EE
:1048300086F8245086F83890F56386F84090F56441
:10484000C6F85090B36103F0C7F808B172B6FEE73E
:10485000079007A9304604F0EFF808B172B6FEE7FA
:10486000354B0C9340F6FA720523CDE90E234FF435
:104870008053324A8DF8340010930AA94FF4400354
:104880003046CDE90A2303F08BFD08B172B6FEE78E
:1048900021A3D3E90023CDE9122304227F23CDE90C
:1048A000142330460422002312A9CDE9162303F075
:1048B0000BFB08B172B6FEE7214D224E149040F278
:1048C0008F63CDE91200C5E90063A86040F2E733C9
:1048D000A8612846EB6006F00BFB034608B172B6F0
:1048E000FEE7284612A91293149306F0E1FD08B1E1
:1048F00072B6FEE7144B154A1490CDE91200C3E9D5
:10490000010098611A60184641F6FF52DA6006F01D
:10491000EFFAE8B172B6FEE7002090B6060000009C
:10492000D21C002000100240A00800200004004813
:10493000000800509C070020002090B60000C07DB9
:10494000500E002000140040040E00200010004013
:10495000202312939D48002312A9149306F0A8FD6A
:1049600008B172B6FEE79A4D9A4B2B60CDE9130061
:10497000CDE916004FF4001301274FF040082846F8
:104980001297CDF86080159305F0FEF9064608B140
:1049900072B6FEE712A92846DFF874A28E4D05F024
:1049A0000DFA4FF4E133C5E900A328460C23C5E90D
:1049B0000266C5E90666C5E908662E61AE626B61EE
:1049C00007F0B8FD014608B172B6FEE7284607F0C9
:1049D00041FE014608B172B6FEE7284607F07CFEAC
:1049E00008B172B6FEE7284607F016FE08B172B6A7
:1049F000FEE77A4D7A4B0C90CDE91200CDE9140018
:104A0000CDE90A00C5E90100C5E90400A8612B60F1
:104A10002846EF23EB6006F06BFA08B172B6FEE7AA
:104A20004FF4805312A92846129306F06BFB08B18D
:104A300072B6FEE720220C9000230AA92846CDE991
:104A40000A2306F035FD024608B172B6FEE7654856
:104A5000DFF8C0E102614FF4003141624FF4A03150
:104A6000C0E90A1282618022C0E900E2C0F8088031
:104A7000077506F081F908B172B6FEE75A4D5B4A38
:104A80002A6002F1015202F58012002302F68C32F4
:104A900001272846C5E90237C5E90433C5E90633CD
:104AA0006A602B6205F096FD014608B172B6FEE71A
:104AB000284606F00BF9014608B172B6FEE7284613
:104AC00006F02EF9064608B172B6FEE7014620222E
:104AD00012A8FBF7A7FC464DDFF83CC1AE834FF4AC
:104AE0004033C5E900C328460423C5E90266C5E989
:104AF0000466C5E90B662F6285F8246085F8386086
:104B0000EE6385F84060AB6102F066FF08B172B6F3
:104B1000FEE7384A0623CDE9122300227F23CDE9A0
:104B2000142312A9042200232846CDE9162303F0FA
:104B3000CBF9014608B172B6FEE72F4D302212A81C
:104B4000FBF770FC2D4B2B60284605F05DF9024603
:104B500008B172B6FEE7284612A90225CDE9142253
:104B6000CDE91755ADF84C2016921992129505F023
:104B70007BFA08B172B6FEE7214B224A58601861F1
:104B80009861D8621A60184660221F759A6006F014
:104B9000F3F808B172B6FEE71B4B1C4918624FF0E0
:104BA00002084FF00009C3E904894FF000084FF0F4
:104BB00000090822C3E906891846C3E900129D606E
:104BC00007F020FF50B372B6FEE700BF040E0020CE
:104BD00078080020000C0240E80E00209C0E002007
:104BE00000340140940A0020480A0020005400408C
:104BF00008080020000029C3B4080020001000505D
:104C0000D00A002004030140100B0020005C00408B
:104C10000038014000030140000100500A2003F069
:104C2000B9FF01F069FA00F001FA01F089F801F02A
:104C3000A5F800F0A1FD00F0E7FD8248DFF87C82D6
:104C4000DFF87C92DFF87CB2DFF87CA27E4E7F4DED
:104C500006F01AF9FFF764FC7D4806F019FA3A46A7
:104C60007C497D487D4F06F07BFC01F08FFCFFF70F
:104C70000FFC7B4B1B78002B2ED07A4B1B7863B13B
:104C8000794B7A4A1B68009379487A4B4FF48061DC
:104C900000F050FB734A0023137098F80030DBB12A
:104CA000D9F80030002B6FD05A1E032A63D9052B88
:104CB00005D170496D482B46402200F0D1FC6E4B67
:104CC0006E481A786E4B294603EB0222402307F008
:104CD0002FFE002388F800306A4B1B78002B37D05A
:104CE000694B1B7883B1694B604A1878684B03EBBA
:104CF0000030684B1B6800934FF480615D4B00F0FF
:104D0000FBF9614A00231370634B1B786BB1D9F830
:104D1000003053B35A1E012A3CD9052B05D1554901
:104D200052482B46402200F04FFA98F800307BB1F1
:104D3000D9F80030033B012B0AD84F4B1878504B61
:104D4000402103EB002000F097FA002388F80030A0
:104D5000524B1B78002B8CD0514B1A78514B1B783F
:104D60009A4220D000F0D0F8F6E740482A46402189
:104D700000F010FAD9E74C4B00933E493B482B46D4
:104D8000402200F089FC9AE738482A46402100F08A
:104D9000D9FC94E7444B0093364934482B464022D3
:104DA00000F0CCF9C1E723880BB101F011F83F4BBB
:104DB0001A8832B13E49284806F0A6FC3B4A002337
:104DC0001380BBF8003001339BB2ABF800305B07B7
:104DD0002AD1234B1B78D3B1DAF8003043B33B68B8
:104DE0000BB901F07BFA0023CAF8003031233B6095
:104DF0001E48402100F05CF92E4A8000C3B21370B7
:104E000032789A4203D00720337000F0EFF81D4B40
:104E10001B784BB1327828494E239A420B7003D04D
:104E20000720337000F0E2F81C4A0023137020E7DB
:104E30003B68002BDCD0013B3B60002BD8D101F05C
:104E40004DFAD5E7940A0020D01C0020A01B0020BA
:104E5000500E0020E43C0020E80E00209C1B0020A7
:104E6000A01C0020780F0020244700208C17002071
:104E70007C0F00208C1800208C1B00200C47002089
:104E80008C190020E31C0020F83E0020053F002084
:104E9000E41C0020083F0020043F0020790F002080
:104EA000C81C0020C91C002047E17A14E83E0020FD
:104EB000E83C0020284700200C3F00207408002018
:104EC000941B00207A0F0020981B002072B6FEE78A
:104ED00003780133194001700846704780FB0110C8
:104EE00000F31E004000704710B4054A054C1178CD
:104EF0004B1C03F01F03137060545DF8044B7047A4
:104F0000C81C0020A81C002010B5064C064A2378B7
:104F1000D05C01F05FF82378013303F01F032370A6
:104F200010BD00BFC91C0020A81C002038B5114BC3
:104F30001149124A1B680C681168022B214408D0E1
:104F4000042B06D023F00203012B08BFA1F21E712F
:104F500001E001F21E710023094A0A4D0020FFF70B
:104F60000BF803462B6020460021BDE8384001F0D5
:104F7000A1BC00BF941B002088170020A41C0020A7
:104F8000305705002447002038B500F0F5FB114BE1
:104F90001149124A1B680C681168022B214408D081
:104FA000042B06D023F00203012B08BFA1F21E71CF
:104FB00001E001F21E710023094A0A4D0020FEF7AC
:104FC000DBFF03462B6020460021BDE8384001F09E
:104FD00071BC00BF941B002088170020A41C002077
:104FE0003057050024470020704700BF034A0123C3
:104FF000118803FA00F0084310807047D21C00208B
:10500000044901220B8802FA00F023EA00030B8016
:10501000704700BFD21C0020034B1B8843FA00F0EE
:1050200000F00100704700BFD21C002038B5144BBF
:10503000144A154C042500211D60144B11604FF4D7
:10504000FA30134A20601A6001F034FC114802243F
:1050500004601148082404601048114C4FF4FA62AF
:10506000026010481023036040F2E2410E482160C4
:1050700000F0DEFB0D4B4FF6FF721A8038BD00BF0B
:10508000941B0020A41C0020881700202447002027
:10509000F59CF45ECC1C0020EC3E00208017002024
:1050A000841700207C17002010420020D21C002012
:1050B00071B101398BB20021021F8C4600EB8300D5
:1050C00052F8043F002B0DDD904201EBA311F7D104
:1050D0001F2301E0013B0CD041FA03F2D207D8B202
:1050E000F8D5704783FAACF3904201EBA311E7D1F6
:1050F000EEE71846704700BF70B50E4D0E4C2B689A
:10510000049A636091B14FEAA20E4E0073440022EC
:10511000A1686360091502F1010C20F812101FFA52
:105120008CF2B24219467344F2DB2960024B9B6851
:1051300070BD00BF003F0020000C02402DE9F84385
:10514000124E134D3168089F6960D2B102F1FF38E9
:105150001FFA88F803EB88081C1F00E03168D5F8B7
:10516000089039443160696054F8041F0FFA89F0DF
:10517000FFF7B4FE21684FEA2940FFF7AFFEA045D4
:10518000ECD1034B9B68BDE8F88300BFFC3E0020D8
:10519000000C024010B40B4C011F043A00F1FC0C4F
:1051A00051F8043F206800FB03F3002BB8BF03F65F
:1051B000FF7304321B138C451360F1D15DF8044B6F
:1051C000704700BF901B0020002A4ED030B51C1D38
:1051D000A04218BFA14214BF01240024551E00F1B3
:1051E000040CADB261450CBF002404F001040A2D8B
:1051F00094BF002404F0010444B340EA01041C43BA
:10520000640723D19FED1A6B5508A3F1080401EB45
:10521000C505A0F1080E8C4694ED027B8EED027B55
:10522000ACEC026BAC4504F108040EF1080EF3D1AE
:1052300022F00104A2421FFA84FC06D053F82C206D
:1052400040F82C20002341F82C3030BD1A1F0438C0
:1052500003EB85030439002552F8044F40F8044F4E
:105260009A4241F8045FF7D130BD7047AFF3008038
:10527000000000000000000000294AD02DE9F84F8E
:105280002B4B0139D3E900450FF28C09D9E900898C
:105290000FF28C0BDBE900AB89B2071D064607EB6A
:1052A000810742464B4620462946FEF7B7F952464B
:1052B0005B4604460D46FEF7EDFD45EC104BC8B9C4
:1052C000FBF7BEFF53EC102B10EE100A1946FEF749
:1052D000A5F915A3D3E90023FEF7A0F9FEF72CFEEC
:1052E00080B246F8040BBE42DBD1114BC3E9004546
:1052F000BDE8F88F40F2FF7346F8043BBE424FF022
:1053000000044FF00005CCD1094BC3E90045BDE8CE
:10531000F88F7047AFF30080333333333333C33FF9
:105320001F85EB51B81E19400000000000FC9F4093
:10533000F03E00202DE9F04F2DED028B08EE903A63
:10534000BC4B08EE102AADF6340D1A68BA4B5A6001
:105350000491002900F06881831E01930CAB0024A6
:105360000B930DF58663DFF8F0A2069403940A937D
:105370000094114601E0AF4B1968DDF86038019CDC
:10538000AD48AC4AAD4E19448368116034F8022F21
:1053900001944160AA49A2F580520D7819B21B14FC
:1053A00002FB03F346F82530009B02FB01F1DA070C
:1053B0004AF8251040F11481A24A05F03F01146813
:1053C00056F821805AF821E00294A5F10E03A81E98
:1053D00034469C4903F03F0300F03F00D1F80890A9
:1053E0005AF823205AF8201054F82000029C56F84E
:1053F000233084FB022CCEFB042CA5F10C0707F014
:105400003F07C1FB092C84FB0331C8FB0431C0FBFF
:1054100009318A4C5AF82700C9FB002C54F82700A0
:105420002E1F06F03F06C0FB09318648D0F81080D9
:105430005AF82600A5F10A0E0EF03F0EC0FB082C0C
:1054400054F82600C0FB08315AF82E00C8FB002C87
:1054500054F82E00AF1F07F03F07C0FB0831794812
:10546000D0F818B05AF82700A5F1080606F03F0654
:10547000C0FB0B2C54F82700C0FB0B315AF8260058
:10548000CBFB002C54F82600073D05F03F05C0FB80
:105490000B316C48C6695AF825000596C0FB062CEE
:1054A00054F82500C0FB0631DB0F43EA410366498F
:1054B000664E0978D20F46F82130039B42EA4C022F
:1054C000DFF898C1DB074CF8212040F181808D1E68
:1054D00001F01F0005F01F05A1F10E0303F01F03EB
:1054E00056F825405CF8207056F820005CF8232020
:1054F00008900994081F029C56F8233000F01F0002
:1055000007905CF8250084FB0225C4FB0725C9FB36
:105510000025A1F10C0EA1F10A00089F0EF01F0E4C
:1055200000F01F00029084FB0330C4FB07305CF8DE
:105530002E70099CC9FB0725C9FB043056F82E7054
:10554000079CC9FB07305CF82470C8FB072556F898
:105550002470029CC8FB07305CF82470A1F1060E91
:105560000EF01F0EC8FB072556F824700B9CC8FBD5
:1055700007305CF82E70A1F1080909F01F09CBFB78
:10558000072556F82E70CBFB07305CF829700739D9
:1055900001F01F01CBFB072556F82970CBFB073024
:1055A0005CF8217056F82110059EC6FB0725C6FB46
:1055B0000130D20F069942EA450244F82120DB0F60
:1055C0000A9A43EA400342F821304B1C9BB20693EF
:1055D0001D481F21FFF77CFC039B01339BB2039303
:1055E00017483F21FFF774FC009C049B0134A2B2D2
:1055F000934200927FF4BFAE18EE102A0B99144824
:105600004FF4807307F0D2F812480A9918EE902AE6
:105610004FF4807307F0CAF8074B9B680DF6340D02
:10562000BDEC028BBDE8F08F0CAB0B930DF58663E0
:105630000A93E1E720470020000C024010410020BF
:1056400019470020680000201847002090400020E3
:10565000284D002030530020903F0020103F0020B4
:10566000CAB1013A92B210B5A0F1040C0C1FA3F11B
:10567000040E00EB820054F8043F5CF8042F83FB17
:1056800003135B1082FB022103EB610360454EF8BC
:10569000043FF0D110BD70472DE9F04FDFF898A01E
:1056A000DFF89080DAF80040C8F8044083B0002AA0
:1056B0003AD002F1FF391FFA89F91E4600EB89033F
:1056C000DFF878B0DFF8789001930F1F051F01E035
:1056D000DAF800400C9B1919D8F80840CAF80010F5
:1056E000C8F80410D9F8001020B201FB00F0400106
:1056F00055F8041FFFF7F2FB8446D9F8000057F86D
:10570000041F241404FB00F040016446FFF7E6FB8D
:10571000DBF80010019B02290CBF0019201A9D42E2
:10572000306006F10406D3D1024B9B6803B0BDE89C
:10573000F08F00BF000C02401C470020941B00208B
:10574000EC3E002010B40B4C011F043A00F1FC0C9D
:1057500051F8043F206800FB03F3002BB8BF03F6A9
:10576000FF7304321B138C451360F1D15DF8044BB9
:10577000704700BFEC3E00201C4B10B51B685A1E42
:10578000032A82B01BD923B1053B012B01D902B0FA
:1057900010BD1748174B4FF48074CDE90004042264
:1057A0008021154806F0E8FF144A124B1448CDE951
:1057B00000248021042206F0DFFF02B010BD0C4A55
:1057C000104B0D484FF48074CDE900248021042251
:1057D00006F0D2FF094A0B4B0948CDE9002480218D
:1057E000042206F0C9FF02B010BD00BF941B0020C8
:1057F0002C470020A4020020284D0020344D00201A
:1058000030530020A400002000B583B04021009157
:10581000044B054A0548802107F07AF803B05DF88B
:1058200004FB00BF10440020104200200C47002061
:105830002DE9F0412DED028B0546ADF5816D50004F
:105840001E460F46FEF726F81FA3D3E90023FEF7F6
:10585000C5F941EC180B7800FEF71CF81AA3D3E940
:105860000023FEF7BBF9B0EE481AF0EE681A41ECDF
:10587000100B02228021684601F0BAF8B008FEF74A
:1058800019F8022241EC100B6846802101F078FBE8
:105890000FA7D7E90067043D6C460DF58068F4E872
:1058A000020132463B46FEF76FF8FEF71DFB44450A
:1058B00045F8040FF3D10DF5816DBDEC028BBDE809
:1058C000F08100BFAFF3008000000000C05CD54055
:1058D0000000C0FFFFFFDF41044B054A05491B786C
:1058E000126809680448FFF7A3BF00BF7C170020B7
:1058F000801700208417002010420020094A10B5AC
:10590000C0EBC000084C02EBC0022188D36A0748F4
:105910001B68127C08440649FAF7C0FE2388184425
:10592000208010BDA4040020E83E0020E83C0020B8
:1059300098CD000810B5094A094C0A492388C0EBE4
:10594000C00002EBC00208481844D36A127CFAF780
:10595000A5FE23881844208010BD00BFA4040020A9
:10596000E83E0020A0CD0008E83C00200B4AC0EB38
:10597000C00002EBC00238B5D36A094C1968208810
:10598000084B094D127C03EB810328440749FAF7C1
:1059900085FE23881844208038BD00BFA404002061
:1059A000E83E002048070020E83C0020A0CD000889
:1059B00098B51D4BC0EBC00003EBC00000AF027CEC
:1059C000C16AD31D03F4FC73ADEB030D0B7869467C
:1059D000F2B168460DEB020C20244FF0850E0EE06C
:1059E00080F800E09A1FD2B29A4200F101004FF015
:1059F000FF3388BF0023844503EA020308D0052B48
:105A0000EED8A3F180020BB10270EBE70470E9E776
:105A1000064C074823881844FAF740FE23881844A8
:105A20002080BD4698BD00BFA4040020E83E0020B1
:105A3000E83C00202DE9F043304B3149C0EBC00079
:105A400003EBC00089B0C36A68461A68FAF726FEFD
:105A50009DF80090B9F1000F4DD00025294F2C463C
:105A60002E464FF02E086846FAF74AFE001B07FB49
:105A700000F0B0F1553F16D806F120030DEB0306F8
:105A80008CB116F8213C05F12002202B6A4404BF9A
:105A900005F120026A4405F101050CBF02F8103C33
:105AA00002F8108CEDB20134E4B205F120026B1C57
:105AB0000DEB020504F120026A4405F8109C12F86F
:105AC000209CDDB22646B9F1000FCCD10E4C0F4818
:105AD00023880F49184405F120030DEB030500232B
:105AE00005F8103C04AAFAF7D9FD23881844208051
:105AF00009B0BDE8F0834D46E8E700BFA4040020EC
:105B0000A4CD0008ABAAAAAAE83E0020E83C0020E9
:105B1000ACCD00082DE9F041154D164C2878C0EBAE
:105B2000C00204EBC202C300D17B31B1181A04EBEE
:105B3000C000BDE8F041036B1847D66A5769316869
:105B4000394431609769B94207D3D269914204D888
:105B5000FFF74CFA2878C300E8E71B1A04EBC303ED
:105B600093F820200AB13760F2E7DB693360EFE792
:105B70003C530020A40400202DE9F041154D164CA3
:105B80002878C0EBC00204EBC202C300D17B31B164
:105B9000181A04EBC000BDE8F041036B1847D66A41
:105BA00057693168C91B31609769B94207D3D26917
:105BB000914204D8FFF71AFA2878C300E8E71B1AC5
:105BC00004EBC30393F8202012B1DB693360F1E7E3
:105BD0003760EFE73C530020A4040020F8B5234DC4
:105BE000234C2878FFF702FA2978224B224A93F8AF
:105BF00000E017780131C9B2297000220846164624
:105C000004E05FFA8CF086451646F7D9C0EBC00376
:105C100004EBC30200F1010CD17B04294FF0010217
:105C20004FF00001EDD014F83330BB42E9D106B19A
:105C30002870124E124FFFF7D9F93088114900230E
:105C40001A463844FAF72AFD33882A780E49063373
:105C50009BB2F8183380382303FB02430133FAF771
:105C60001DFD338818443080F8BD00BF3C53002030
:105C7000A40400204407002042530020E83E0020F6
:105C8000E83C0020B0CD0008BCCD0008F8B5244D9C
:105C90002878FFF7ABF92878224B01381F78C0B27B
:105CA000B842287002D3781EC0B228701E4B1F4C19
:105CB00093F800E007F1FF3C00265FFA8CFC05E05A
:105CC000C8B287424FF0010698BF6046C0EBC003E0
:105CD00004EBC302411ED27B042AF1D014F8333006
:105CE0007345EDD106B12870114E124FFFF77EF9C2
:105CF0003088114900231A463844FAF7CFFC33881C
:105D00002A780E4906339BB2F8183380382303FBF8
:105D100002430133FAF7C2FC338818443080F8BDDF
:105D20003C5300204407002042530020A4040020DC
:105D3000E83E0020E83C0020B0CD0008BCCD0008C3
:105D4000094B07CB30B4094C1B88A381084B616019
:105D5000A2604FF48061074A074D19800023137039
:105D600020602B7030BC7047C8CD0008D41C0020C8
:105D700040530020425300203C53002038B50E4CC5
:105D80000E4D20880E4900231A462844FAF786FC57
:105D900021880C4B06311A780B4B89B26818218088
:105DA000382101FB023301330849FAF777FC2388D5
:105DB0001844208038BD00BFE83E0020E83C0020A9
:105DC000B0CD00083C530020A4040020BCCD000846
:105DD0002DE9F04FDFF8009199F8003083B0002BE7
:105DE0006BD00025364FDFF8F4802C460AE0FF2BFD
:105DF00017D02046FFF704F999F800300135ECB2CE
:105E0000A3425AD92046FFF707F90028F4D02D4ABB
:105E1000C4EBC403127817F833309A424FEAC40631
:105E2000E5D1311B07EBC10ACB0001939AF80F3083
:105E3000052BDED0B8F80000DFF8A4B09AF81220E5
:105E40009AF8113020495844FAF728FCB8F8003085
:105E50001844019B80B203F12101A8F800003944E5
:105E60005844FAF71BFCB8F800209AF80F30104499
:105E700080B2042BA8F800000BD0144B1B78A3426F
:105E80000CBF134B134B1B882BF800300130A8F8C4
:105E90000000361B07EBC6062046736B9847019936
:105EA000B8F80000253139445844FAF7F7FBB8F840
:105EB00000301844A8F800009BE703B0BDE8F08F5D
:105EC000A404002042530020B0CD00083C53002021
:105ED000D8CD000818CF000844070020E83E002075
:105EE000E83C002070B5032812D8DFE800F0541E0B
:105EF0001202FFF741FE2B492B4B0A882B4D02F172
:105F00000800088003CB54191B785051616023723C
:105F100070BD244C25482388254918443222FAF7BD
:105F2000BDFB23880533238070BD2249224D0B78A9
:105F3000224A2878D0540133DBB2012B88BF0023DA
:105F4000184CD25C0B702A7023881D491D4A174ECD
:105F500012889A534FF6FF700880581C80B20023B5
:105F600020801A4618493044FAF798FB23882A788B
:105F7000164906339BB2F0182380382303FB021323
:105F800001331349FAF78AFB238818442080BDE8BF
:105F90007040FFF71DBFFEF7A5FABDE87040FEF7A1
:105FA0002BBA00BFE83E0020E8CD0008E83C002006
:105FB000E0CD0008425300203C5300204053002015
:105FC000D21C0020DCCD0008B0CD0008A4040020C5
:105FD000BCCD00082B3838B538282DD8DFE800F0C4
:105FE000392C3C2C2C2C2C2C2C2C2C2C2C2C2C2CD4
:105FF0002C2C2C2C2C2C3F44494E1F5365751D2CEA
:106000002C2C2C2C2C2C2C2C2C2C2C2C2C2C2C2CD0
:106010002C2C2C2C2C2C782C2D00FFF7DFFD2F495D
:106020002F4B0A882F4D02F10800088003CB54192A
:106030001B7850516160237238BD284C2948238851
:10604000294918440022FAF729FB238804332380C6
:1060500038BDFFF75FFDE2E7FFF78EFDDFE7BDE844
:1060600038400020FFF73EBFBDE838400120FFF771
:1060700039BFBDE838400220FFF734BFBDE83840E3
:106080000320FFF72FBF194B194A1B78C3EBC3033B
:1060900002EBC3025369D16903EB8303B1EB430FF6
:1060A0004FEA4300BBD95061B9E7104B104A1B7847
:1060B000C3EBC30302EBC3035A69092AAFD90D49E5
:1060C000A1FB0212D2085A61A9E7FFF7DFFDA6E79C
:1060D000FEF7BCF9BDE83840FEF7DAB9E83E00202B
:1060E000E8CD0008E83C0020E0CD00083C5300204B
:1060F000A4040020CDCCCCCC2DE9F04F6B4E6C4CE1
:1061000033886C48DFF8CC91DFF8CCC16A4E8BB095
:106110001919069314339FB207F116031FFA83FE71
:106120000EF118030EEB040BCDF804E01FFA83FE0A
:1061300073461A330EEB0408CDF808E01FFA83FE0D
:106140000EF11C030EEB040A3A19CDF80CE01FFA0D
:1061500083FE0992724602F11E039BB20546079127
:10616000049205930FCD0895069D00972851079836
:10617000009DC360089B41600146826018681B79DE
:1061800008610B75B9E80F0028510998019D8260DC
:106190000246C360B9F8043041609382D9F8000028
:1061A00099F8063010619375BCE80F002851CBF8C0
:1061B0000410BCE80300414FCBF80C309CF80030D1
:1061C000CBF80820CBF81000CBF814108BF818305F
:1061D0000FCF029D2851C8F80410C8F8082003CF3B
:1061E000C8F80C303B88A8F81830BB78C8F8100005
:1061F000C8F8141088F81A300FCE039D059F285157
:10620000CAF80410CAF8082007CE2D4DCAF80C3081
:106210003378CAF81000CAF81410CAF818208AF89F
:106220001C300FCD214EA64437800095049D285187
:10623000CEF80C30009BCEF80410CEF8082007CB27
:10624000CEF818201A461B88AEF81C309378CEF88A
:106250001000CEF814108EF81E30E01919491A4DAE
:1062600047F23052FAF71AFA338803CD08339BB25B
:106270001F19324603F10A061851B6B22B88168050
:10628000A0193B81094EAB787960BB720F4900229F
:10629000FAF704FA33880E4A043311889BB25A1C69
:1062A000195332800BB0BDE8F08F00BFE83E0020EC
:1062B000E83C0020F4CD00085CCE000840CE000889
:1062C0007CCE00089CCE0008A4CE0008E0CD0008DB
:1062D000DCCD00080CCE000824CE000809490A4B8A
:1062E0000A8802F1080010B4084C088003CB02EBC6
:1062F000040C1B781051CCF804108CF808305DF8B1
:10630000044B7047E83E0020E8CD0008E83C002040
:106310002DE9F84F984B984205460C4666D94FF048
:1063200000088000C2464FF00C09FDF7B3FA8CA3B9
:10633000D3E90023FDF752FC0F460646FDF7D4FDD6
:106340000546FDF7B7FA02460B4630463946FDF7DB
:1063500063F985A3D3E9002306460F46FDF714FB36
:10636000FDF7EAFD8346E0B3FDF794FA32463B467B
:10637000FDF734FC814B0022FDF750F9FDF7DCFD01
:106380007F4A904228BF1046010B01F0F001C0F394
:106390000722C3B2ED01A5F500754FEACB1B2270B1
:1063A000BBFBF0F21544637000FB12B3C5F301426E
:1063B00041EA1341A2702A0AE270180A00226171B0
:1063C000012184F80A9084F80BA084F80C80A07155
:1063D0002571E371227261726273A273E273BDE888
:1063E000F88FFF236648F0211A46D3E7654B9842A1
:1063F00052D8B3EB400F4FEA4007C0F09D80B3EB9B
:10640000800F4FEA8007C0F09B80B3EBC00F4FEACC
:10641000C007C0F09980B3EB001F4FEA0017C0F02F
:106420008780B3EB401F4FEA4017C0F09180B3EB79
:10643000801F4FEA8017C0F08F80C7014FF0070917
:1064400080263846FDF726FA0B46024648A1D1E9D8
:106450000001FDF7C3FBFDF76FFD10F0010F824651
:10646000494B18BF00F1010A07FB0AF098424FEAB6
:10647000091906FB05F04AD90AFB00F00AF1007A77
:10648000AAF1040A4FEACA18CAF341235FFA88F84E
:106490009944CAF3470A48E7FDF7FCF902460B4660
:1064A00033A1D1E90001FDF799FBFDF745FD052872
:1064B000824616D910F0010F01D000F1010A324BCB
:1064C00005FB0AF0984213D90AF1007AAAF1040AEE
:1064D0004FEACA18CAF341295FFA88F8CAF3470A93
:1064E00023E7294B4FF0060A05FB0AF09842EBD848
:1064F0000AF1007AAAF1020A4FEACA18CAF341293E
:1065000000EB4500CAF3470A5FFA88F80DE70AF185
:106510000073023B0AF1020A4FEAC318C3F3412297
:1065200000FB0AF05FFA88F89144C3F3470AFCE6DF
:106530004FF00409102684E74FF00109022680E796
:106540004FF0020904267CE74FF00309082678E79C
:106550004FF00509202674E74FF00609402670E742
:106560000000000060E3764100000000FEFF2F41C4
:1065700000000000A3E1C14180D1F0080000E03F2D
:10658000FFFF0F0068780400FF45C323F0B5C84C37
:1065900087B0002705AD6426059764230322C02138
:1065A000204604F0CDFA0028F7D10123CDE90136C9
:1065B00002460095C021204604F090F90306EBD472
:1065C000FF23BB4E8DF8143064230322C0213046D4
:1065D00004F0B6FA04460028F6D101236422CDE97E
:1065E0000132B34800950322C021B14E04F046F8B1
:1065F0008DF8144064230322C021304604F0A0FA31
:1066000004460028F6D101236422CDE90132A848CE
:1066100000950F22C021A64E04F030F88DF81440EA
:1066200064230322C021304604F08AFA044600287D
:10663000F6D101236422CDE901329D48009518224C
:10664000C0219B4E04F01AF88DF8144064230322F5
:10665000C021304604F074FA0028F7D101246423E5
:10666000CDE901439248009523462A22C021904E4D
:1066700004F004F88DF8144064230322C02130464E
:1066800004F05EFA04460028F6D101236422CDE925
:106690000132874800952B22C021854E03F0EEFF82
:1066A0008DF8144064230322C021304604F048FAD8
:1066B00004460028F6D101236422CDE901327C484A
:1066C00000952F22C0217A4E03F0D8FF8DF8144098
:1066D00064230322C021304604F032FA0446002825
:1066E000F6D101236422CDE90132714800953022B0
:1066F000C0216F4E03F0C2FF8DF8144064230322C3
:10670000C021304604F01CFA04460028F6D10123CB
:106710006422CDE90132664800953122C021644EE1
:1067200003F0ACFF8DF8144064230322C0213046EF
:1067300004F006FA0028F7D101246423CDE90143CF
:106740005B48009523463222C021594E03F096FF44
:106750008DF8144064230322C021304604F0F0F980
:1067600004460028F6D101236422CDE901325048C5
:1067700000953322C0214E4E03F080FF8DF8144067
:1067800064230322C021304604F0DAF904460028CD
:10679000F6D101236422CDE9013245480095372224
:1067A000C021434E03F06AFF8DF814406423032296
:1067B000C021304604F0C4F904460028F6D1012374
:1067C0006422CDE901323A4800953822C021384E82
:1067D00003F054FF8DF8144064230322C021304697
:1067E00004F0AEF90028F7D101236422CDE901328B
:1067F0002F4800953922C02103F040FF2C4C4F2335
:106800008DF8143064230322C021204604F098F947
:106810000028F7D101236422CDE9013224480095F4
:106820001022C02103F02AFF214C5F238DF8143081
:1068300064230322C021204604F082F90028F7D106
:1068400001236422CDE90132194800951122C021AB
:1068500003F014FF164C80238DF8143064230322B8
:10686000C021204604F06CF90028F7D101236422EE
:10687000CDE901320E4800951222C02103F0FEFE40
:106880000B4C12238DF8143064230322C0212046C0
:1068900004F056F90028F7D101236422CDE9013232
:1068A0000095B722C021024803F0E8FE07B0F0BD12
:1068B000480A00202DE9F0438BB006A9FFF728FD18
:1068C00006AD2C4C0DF12009C5F119080DF1170684
:1068D000642715F8013B8DF8173064230322C0218B
:1068E000204604F02DF90028F7D1012308EB05021A
:1068F000CDE90137009692B2C021204603F0BEFEDA
:106900004D45E6D11B4C0DF1220734254FF06408AC
:1069100017F8013B8DF8173064230322C02120466D
:1069200004F00EF90028F7D101232A460135CDE9FC
:1069300001380096C0212046ADB203F09FFE372DEE
:10694000E6D120230B4C8DF8173064230322C0219D
:10695000204604F0F5F80028F7D101236422CDE9A0
:1069600001320096B122C021024803F087FE0BB02D
:10697000BDE8F083480A002010B586B0FF230C4C18
:106980008DF8173064230322C021204604F0D8F884
:106990000028F7D101230DF117026421CDE901315F
:1069A0000092C0210322024803F068FE06B010BD29
:1069B000480A002010B586B0FC230C4C8DF8173027
:1069C00064230322C021204604F0BAF80028F7D13E
:1069D00001230DF117026421CDE901310092C0219C
:1069E0000322024803F04AFE06B010BD480A002008
:1069F0002DE9F04F2DED088B85B0044600915BEC3E
:106A000010AB51EC110B042A1BD8DFE812F01F0069
:106A1000DC00660043010500009B002B04DDDA006A
:106A200000212046F9F7FEFC009B03F1FF3B0BEB36
:106A3000DB7BB74B4FEA6B0B002204EBCB04C4E9C2
:106A4000002305B0BDEC088BBDE8F08F009B002B48
:106A5000F7DD581EFCF72EFFAE4B0022FCF794FF2B
:106A600000258046894613E047EC106BFAF7E8FBF7
:106A700032463B4651EC100BFDF7B0F852465B46F0
:106A8000FCF782FF009B0135AB42E4E80201D8D05D
:106A90002846FCF70FFF42464B46FCF7BDFD524629
:106AA0005B46FCF771FF92A3D3E90023FCF76CFF70
:106AB00091A3D3E9002306460F46FDF7F5F9002818
:106AC000D2D08FA3D3E9002330463946FDF7CEF963
:106AD0000028C9D050465946D4E78E4B0022FCF717
:106AE00053FF06460F4632463B4650465946FCF792
:106AF00093FD5B4680468946524630463946FCF750
:106B00008DFD009B002B49EC198B41EC1A0B98DD95
:106B1000581EFCF7CFFE7F4B0022FCF735FF002507
:106B200023469FED798B2C460FF2C41BDBE900ABAB
:106B3000804689461D4608E085ED008B009B0134A8
:106B4000A34205F108053FF47CAF2046FCF7B2FEF6
:106B500042464B46FCF760FD0022002306460F46E6
:106B6000FDF77AF90028E7D132463B4651EC190B84
:106B7000FCF70AFF52465B46FCF706FF41EC100BA0
:106B8000FAF716FB32463B4651EC1A0B8DED020B21
:106B9000FCF7FAFE52465B46FCF7F6FE41EC100BA2
:106BA000FAF706FBDDE9020153EC102BFCF734FD8C
:106BB00052465B46FDF712F832463B46FDF70EF8AB
:106BC000C5E90001BAE7009A002A02F00103B8BF44
:106BD0005B42012B00F04281002A7FF732AF501E4A
:106BE0001746FCF767FE4B4B0022FCF7CDFE002555
:106BF0004BEC1AAB9FED448B0FF2F409D9E90089F5
:106C000041EC190B2646AB4608E086ED008B0BF1F4
:106C1000010B5F4506F108063FF413AF5846FCF739
:106C200049FE53EC192BFCF7F7FC00220023044625
:106C30000D46FDF711F90028E7D122462B4651EC0D
:106C40001A0BFCF7A1FE42464B46FCF79DFE41ECB9
:106C5000100BFAF7ADFA42464B46204629468DED19
:106C6000000BFCF791FE41EC100BFAF7A1FADDE9FD
:106C7000000142464B468DED000BFCF7AFFF22466C
:106C80002B46FCF7ABFFDDE90023FCF7C7FCC6E9A8
:106C90000001BCE71F4B0022FCF776FE06460F46BC
:106CA00032463B4650465946FCF7B6FC5B468046AA
:106CB0008946524630463946FCF7B0FC009B002B13
:106CC00049EC188B41EC190B7FF7BBAE581EFCF753
:106CD000F1FD104B0022FCF757FE0FF21C09D9E919
:106CE000008941EC1B0B4FF0000AA34688E000BF6F
:106CF000182D4454FB210940F168E388B5F8E4BE3F
:106D0000F168E388B5F8E43E0000000000000000F0
:106D10000000F03F0000E03F45EC104BFAF790FA1E
:106D2000224651EC100B2B46FCF758FF41EC1A0B96
:106D300032463B4651EC190BFCF726FE88A3D3E9FB
:106D40000023FCF721FE42464B4604460D46FDF764
:106D5000ABF840B186A3D3E9002320462946FDF7CE
:106D600085F8002874D145EC104BFAF769FA2246F1
:106D700051EC100B2B46FCF731FF53EC192BFCF7B1
:106D800003FE02460B4651EC1A0BFCF745FC32465B
:106D90003B4606460F4651EC180BFCF7F5FD70A379
:106DA000D3E90023FCF7F0FD42464B4604460D466E
:106DB000FDF77AF840B16EA3D3E9002320462946B7
:106DC000FDF754F8002846D145EC104BFAF738FA95
:106DD000224651EC100B2B46FCF700FF53EC182B0E
:106DE000FCF7D2FD02460B4630463946FCF714FC50
:106DF000009B0AF1010A5345EBE802013FF421AE82
:106E00005046FCF757FD53EC1B2BFCF705FC54A335
:106E1000D3E9002306460F46FCF7B6FD42464B4633
:106E200004460D46FDF740F800283FF475AF50A327
:106E3000D3E9002320462946FDF718F800283FF43F
:106E40006BAF9FED457BB0EE47AAF0EE67AA6FE708
:106E500053EC192B97E753EC182BC5E7002A7FF763
:106E6000F0AD501EFCF726FD434B0022FCF78CFDD5
:106E7000274641EC190B002642E045EC104BFAF78F
:106E8000DFF9224651EC100B2B46FCF7A7FE80469B
:106E9000894653EC182B50465946FCF775FD30A334
:106EA000D3E90023FCF770FD2FA3D3E900230446A8
:106EB0000D46FCF7F9FF40B12DA3D3E9002320468E
:106EC0002946FCF7D3FF002841D145EC104BFAF7D7
:106ED000B7F9224651EC100B2B46FCF77FFE5246C9
:106EE0005B46FCF751FD02460B4640464946FCF71F
:106EF00093FB009B0136B342E7E802013FF4A1ADEA
:106F00003046FCF7D7FC53EC192BFCF785FB024607
:106F10000B4643EC182B12A3D3E90023FCF734FDF6
:106F200011A3D3E9002304460D46FCF7BDFF00285A
:106F3000A3D00FA3D3E9002320462946FCF796FFF0
:106F400000289AD0DFF834904FF00008A1E75246AD
:106F50005B46CAE7AFF30080000000000000F03F8E
:106F6000182D4454FB210940F168E388B5F8E4BECC
:106F7000F168E388B5F8E43E0000E03F0000F03F30
:106F80002DE9F04F2DED088B89B0012A0790039170
:106F900000F0BA81B0EE409AF0EE609A56EC105BC9
:106FA000144610EE100A002200233146FCF75EFF63
:106FB00000287FD1C64B002228463146FCF774FFDB
:106FC00028B19FEDBD7BB0EE479AF0EE679A039D26
:106FD000AB1CDB0018460693F9F77AF902900028FB
:106FE00000F09281681CFCF765FC022C41EC1B0B45
:106FF00067D0032C00F08D810E2C53D1039B03EB43
:10700000D374012B4FEA640438DDDDF80890ACA797
:10701000D7E90067C846002582468B4601352846D9
:10702000FCF748FC32463B46FCF7AEFC52465B465A
:10703000FCF7D4FD41EC100BFAF702F9A542A9ECDC
:10704000020BEBDB57EC196B002598ED000B47ECBE
:10705000116BFAF73DF90135A542A8EC020BF4DB00
:10706000069B103B05930599029A00231144F2E810
:10707000026701339C4261E90267F8DC039B002B45
:1070800010DD069B103B05931E46079C029D26447F
:10709000D4E90001F5E80223FCF776FCE4E80201FC
:1070A000A642F5D1029809B0BDEC088BBDE8F04FBF
:1070B000F9F716B99FED847BB0EE479AF0EE679A28
:1070C00085E7039B002BEDDD069B029ADFF80CB2EF
:1070D0000192103B0593D318A146049355EC1B4B2A
:1070E0004846FCF7E7FB2B461BEE102AFCF794FA08
:1070F0002B461BEE102AFCF771FD02460B46FCF7EF
:1071000043FC02460B4600207249FCF785FA41EC2D
:10711000100BFAF7AFF953EC192B51EC100BFCF7ED
:1071200033FC6D4B0022FCF72FFC4FF0010841ECC3
:10713000180B0024002535E0B8F1020F42D0B8F159
:10714000030F00F0B580B8F1040F00F0CB80B8F168
:10715000050F00F0C980B8F1060F00F0CC80B8F13F
:10716000070F00F0CE8049F68050B8F1090F08BF34
:107170005846FCF79FFB02460B4630463946FCF763
:107180002DFD02460B46FCF7FFFB02460B46204650
:107190002946FCF743FA08F10108B8F10A0F044642
:1071A0000D4611D04046FCF785FBB0EE480AF0EEE4
:1071B000680A41EC110BFAF78BF8B8F1010F57ECA4
:1071C000106BB9D14046D4E7424B0022FCF726FAB7
:1071D000414B41EC1A0B002251EC190BFCF7D4FB8C
:1071E0004FF0010A41EC180B0024002530E0BAF101
:1071F000020F3DD0BAF1030F5CD0BAF1040F6FD08B
:10720000BAF1050F72D0BAF1060F71D0BAF1070FBB
:1072100074D049F68050BAF1090F08BF5846FCF700
:1072200049FB02460B4630463946FCF7D7FC02467E
:107230000B46FCF7A9FB02460B4620462946FCF705
:10724000EDF90AF1010ABAF10A0F04460D4611D010
:107250005046FCF72FFBB0EE480AF0EE680A41EC0E
:10726000110BFAF735F8BAF1010F57EC106BBED1DC
:107270005046D4E7174B0022FCF7D0F902460B46E4
:1072800051EC1A0BFCF7AAFC019B049AE3E80201FB
:107290009A4209F1020901937FF420AF039B03EBAB
:1072A000D374012B4FEA64043FF7DDAE059EECE694
:1072B00006205EE70620B2E7000000000000244040
:1072C000182D4454FB21094000000000000000007C
:1072D000000024400000F03F0000E03F80890500EE
:1072E00018209CE7182044E7782042E7782096E7AA
:1072F0004FF4347093E74FF434703AE741F2B03012
:107300008DE741F2B03034E709B0BDEC088BBDE841
:10731000F08F039B002B7FF7C5AE069A029F049760
:10732000103A07EB0209C3F10108CDF804900FF2FF
:10733000B00BDBE900ABC1469FED278BB846059249
:1073400006460F4610E045EC104BF9F779FF224650
:1073500051EC100B2B46FCF741FCE8E80201019BC5
:10736000434509F102091FD04846FCF7A3FA32460B
:107370003B46FCF733FC52465B46FCF705FB1AA381
:10738000D3E9002304460D46FCF78EFD0028DAD031
:1073900017A3D3E9002320462946FCF767FD002800
:1073A000D1D051EC180BD8E7049E55EC194B9946F7
:1073B00096ED000B45EC114BF9F78AFFA6EC020B9A
:1073C000B145F5D1039B03EBD374012B4FEA640461
:1073D0003FF749AE6AE700BF000000000000F03F41
:1073E000182D4454FB210940F168E388B5F8E4BE48
:1073F000F168E388B5F8E43EFEE700BFFEE700BFB2
:10740000FEE700BFFEE700BFFEE700BF704700BF1A
:10741000704700BF704700BF01F0AABB014802F0EF
:1074200067BB00BFC8080020014802F061BB00BF75
:1074300028090020014802F05BBB00BF880900203A
:10744000014802F055BB00BFE809002008B5044818
:1074500000F0D0FBBDE80840024800F0CBBB00BF05
:107460009C07002008080020014804F049BA00BF2A
:10747000E80E0020014803F021BF00BF500E00209D
:107480000B4B1A6E42F001021A661A6E82B002F0BD
:1074900001020092009A9A6D42F080529A659B6DAB
:1074A00003F080530193019B02B002F0EDBB00BFDB
:1074B0000010024030B5044695B04422002103A8D4
:1074C000F8F7B0FF2368B3F1A04F04D0384A9342D5
:1074D00040D015B030BD4FF400424FF0005303A828
:1074E0000392129301F052FF002857D1314A1368DA
:1074F0000133012B136009D12F4BDA6C42F4005297
:10750000DA64DB6C03F400530193019B2B4D2C498F
:107510000522C5E9001280214FF48072C5E90412EA
:1075200000234FF4806120222846C5E90233C5E9D3
:1075300006122B6202F074F9002832D100221146A3
:1075400065651220AC6202F0B9FB122002F0F4FB78
:1075500015B030BD4FF400424FF0005303A8039222
:10756000129301F013FFF8B9124A13680133012B8B
:10757000136009D1104BDA6C42F40052DA64DB6C10
:1075800003F400530293029B00221146122002F0E2
:1075900095FB122002F0D0FB15B030BDFDF796FC34
:1075A000A4E7FDF793FCC9E7FDF790FCDCE700BF1B
:1075B000000100504453002000100240C808002081
:1075C000080002400A4B02689A4200D07047D3F884
:1075D000482442F00802C3F8482403F5806382B0CF
:1075E0009B6C03F008030193019B02B0704700BF3E
:1075F000000C024070B50368394A8AB000249342F7
:10760000CDE90444CDE90644089410D0354A9342AC
:1076100001D00AB070BD344BDA6C42F48022DA64D7
:10762000DB6C03F480230393039B0AB070BD2E4BE5
:107630002E4EDA6C42F48032DA64DA6C02F4803274
:107640000192019ADA6C42F00102DA64DB6C03F019
:107650000103029330220323054604A94FF0904012
:10766000CDE90423029B01F0DDFF214A0623C6E990
:10767000002310228023C6E9022433614FF40072F4
:107680004FF40063C6E9052330462023C6E90734DA
:1076900002F0C6F8E8B9174C1749AE600722C4E9F2
:1076A0000012002310218022C4E9021322614FF44A
:1076B00000714FF40062C4E9051220462022C4E99B
:1076C0000723B56202F0ACF830B9EC60A5620AB0ED
:1076D00070BDFDF7FBFBDEE7FDF7F8FBF5E700BF4C
:1076E000000800500010005000100240280900203F
:1076F0001C000240880900204400024010B50446E6
:1077000098B00021442207A8CDE90211CDE9041167
:107710000691F8F787FE194B22689A4201D018B0FB
:1077200010BD402307A8079301F030FE18BB144C8E
:107730001448E36C43F00203E364E36C03F00203D8
:1077400000934FF4C0721223CDE9022300220023DC
:10775000CDE9042302A904230693009A01F062FFF5
:10776000A36D43F40013A365A36D03F40013019309
:10777000019B18B010BDFDF7A9FBD8E700540040ED
:10778000001002400004004800B50268244989B096
:1077900000238A42CDE90233CDE90433069305D0B4
:1077A000204B9A421BD009B05DF804FB03F18043E3
:1077B00003F504339FED167BDA6C42F00102DA64C4
:1077C000DB6C03F00103009302A94FF090408DEDB4
:1077D000027B009B01F026FF09B05DF804FB03F576
:1077E0008633FC33DA6C42F00102DA64DB6C9FED25
:1077F0000A7B03F00103019302A94FF090408DED45
:10780000027B019B01F00EFF09B05DF804FB00BF95
:107810000A000000030000008000000003000000D8
:10782000000301400403014000B51E4A036893426F
:1078300085B008D01C4A93421FD01C4A93420FD0F7
:1078400005B05DF804FB1A4B9A6D42F010029A6580
:107850009B6D03F010030193019B05B05DF804FBE1
:10786000134B1A6E42F400521A661B6E03F4005357
:107870000393039B05B05DF804FB0D4B996D41F03C
:10788000200199659B6D002203F0200302933720AD
:107890001146029B02F012FA372005B05DF804EBA6
:1078A00002F04ABA001000400014004000340140C9
:1078B0000010024030B5044699B00021442207A8C8
:1078C000CDE90211CDE904110691F8F7ABFD2A4B81
:1078D00022689A4201D019B030BD012307A807934E
:1078E00001F054FD002841D1244B254D1A6E42F47D
:1078F00080421A661A6E02F480420092009ADA6C94
:1079000042F00102DA64DB6C03F0010301934FF4EF
:10791000C0620223CDE902230022019B0023CDE9AE
:10792000042302A907234FF09040069301F07AFE4A
:10793000144919220023C5E900122846102180228B
:10794000C5E90213C5E90533C5E907332A6101F02A
:1079500067FF70B9002211462520A567AC6202F0CE
:10796000ADF9252002F0E8F919B030BDFDF7AEFA07
:10797000BAE7FDF7ABFAEDE700380140001002402E
:10798000E80900205800024010B5044692B0442295
:10799000002101A8F8F746FD0D4B22689A4201D05C
:1079A00012B010BD4FF4005301A8019301F0EEFC9A
:1079B00058B9084B9A6D42F400029A659B6D03F426
:1079C00000030093009B12B010BDFDF77FFAF0E7B3
:1079D000005C00400010024030B583B000230193EA
:1079E000002800F0C980C56D0446002D00F092808B
:1079F000226893689B0005D5936823F0204323F009
:107A00003F0393609368DD0019D4704B70481B6886
:107A100091689B09A0FB030321F010419B0921F011
:107A20003F0101335B0041F0805191600193019B64
:107A30002BB1019B013B0193019B002BF9D1936872
:107A4000D80059D4E36D43F01003E365236E0120A1
:107A500003432366936813F0040FE36D53D1D906F3
:107A600051D4E36D23F4817343F00203E36593681B
:107A7000DB070ED4574B4FF0A04189689B680B433E
:107A8000DD0706D4544965688B6823F47C132B43C7
:107A90008B60E568E36B94F824102B43A5682B43B7
:107AA000657F012943EA453343EA01435FD0E16A38
:107AB00021B1256B01F4787129430B43D5684749FF
:107AC00029400B43D3601369616B23F040630B4380
:107AD00013619368590723D593686369012B4ED0CE
:107AE000136B23F00F031363E36D23F0030343F0E1
:107AF0000103E36503B030BD936813F0040F4FF04A
:107B00000000E36DABD0E36D012043F01003E365AB
:107B100003B030BDFFF7CEFC256684F8585067E708
:107B200093681B07D9D4D16894F83830257F21F4A5
:107B300080415B0021F0020143EA85330B43216958
:107B4000D360136919BB23F480331361D2F8C030BA
:107B500023F47F5323F03F03C2F8C03094F8403041
:107B6000012B21D0136923F001031361B5E7A16A4A
:107B7000013943EA41439AE7012003B030BD116B5C
:107B8000236A21F00F01013B0B431363ACE743F47D
:107B900080331361D2F8C03023F47F5323F03F03C6
:107BA0000B43C2F8C030D9E71169636CA56C21F4AE
:107BB000FF6121F004012B430B43E16C0B43216D6A
:107BC0000B4343F00103136187E700BF6C070020FC
:107BD000632D3E0500010050000300500740F0FFF8
:107BE000704700BF08B5806AFFF7FAFF08BD00BF05
:107BF000704700BFF8B503688F4A1D685E689768D4
:107C0000A907044607F01F0702D5B20700F19F80BD
:107C1000690779D5720777D5E26DD20603D4E26D94
:107C200042F40072E265DA6812F4406F1CD1834AB4
:107C3000934200F0DE80DA68900415D41A681107C8
:107C400012D59A68520700F1E5805A6822F00C02BA
:107C50005A60E36D23F48073E365E36DDB0403D4C2
:107C6000E36D43F00103E3652046FCF75DFB236809
:107C70000C221A60A8064DD5B1064BD5E26DD1068F
:107C800003D4E26D42F40052E2656C49DA6CD868C4
:107C90008B4202F4C07268D0D968D2B98A0100F16F
:107CA000A0801A68500614D5890212D49A68120767
:107CB00000F1B9805A6822F060025A60E36D23F443
:107CC0008053E365E36DD80503D4E36D43F001030E
:107CD000E365204600F0A6FE236860221A602906AC
:107CE00001D5320656D4E80501D5F1055DD4AA05C3
:107CF00001D5B00542D4E90601D5F2060FD46805D6
:107D000001D571055DD4F8BD2807B3D5310783D4FB
:107D1000A806B1D46A06E2D57006E0D5AEE7E26BFC
:107D200032B1002F6BD0444A926812F4604F0BD0EE
:107D3000E36D43F48063E365236E43F0020323663F
:107D40002046FFF755FF236810221A60D7E7C36D5E
:107D5000D80603D4E36D43F40063E365204600F0E6
:107D600069FE236802221A6052E7002F94D0B91FDF
:107D7000012991D94FF0A041C9688EE7E36D43F422
:107D80008023E365204600F053FE23684FF4007221
:107D90001A60B0E7E36D43F48033E3652046FCF7F7
:107DA000CFFA236880221A609DE7E36D43F4003325
:107DB000E365204600F03AFE23684FF480721A60B3
:107DC00095E7E26D42F48042E265226E4FF48061F5
:107DD00042F00802226620461960BDE8F84000F033
:107DE00023BE00F4406001F4005202437FF471AFFF
:107DF00057E7092F07D94FF0A042D2681CE7DA688D
:107E0000D707A1D594E740F22122FA40D2073FF5E7
:107E100012AFF0E7E36D43F01003E365236E43F028
:107E20000103236620E7E36D43F01003E365236E4F
:107E300043F0010323664CE70003005000010050AB
:107E4000836ADA6D12F0500F10B5DA6D1DD1196822
:107E500042F40072DA650A6812F0080FCA681BD093
:107E600012F4406F0DD1CA6894040AD4DA6D22F47A
:107E70008072DA65DA6DD10403D4DA6D42F0010262
:107E8000DA651846FCF750FA10BDD2060AD45B6DCD
:107E9000BDE810405B6B18479007E7D51846FCF724
:107EA00043FAF1E71846FFF7A3FE10BD806A08B554
:107EB000C36D43F04003C365036E43F004030366E0
:107EC000FFF796FE08BD00BFF0B590F8582083B0CC
:107ED0000346012A4FF00000019000F045811C6824
:107EE000012083F85800A26855074CD448680A68F6
:107EF0004FEA901E0EF00C0E04F1300C00F01F0043
:107F00005EF80C50C2F384621F26824006FA00F02D
:107F100025EA000002434EF80C20A268500743D522
:107F2000A2680868A26812F0010F02460CD1C24D87
:107F3000CE68AE4200F0C180D4F8B010C0F3120099
:107F400021EA0001C4F8B010BC490A422AD0BC4959
:107F5000BC4D8868AA4200F0E0761DD0BA4DAA4216
:107F60001AD0BA4DAA4240F0318110F0807019D178
:107F7000B74A944216D08A6822F0E072164346F05F
:107F800080768E6003E0DA6D42F02002DA6500222E
:107F900083F8582003B0F0BD020203D4B4F1A04F1F
:107FA00000F0F5800020F2E7A26812F0080240F02D
:107FB000828088680E68B0F1004F00F01B814FEAA4
:107FC000D65C04F114070CF0040CC6F304565CF8FC
:107FD00007504FF0070EB0400EFA06F625EA0605E8
:107FE00028434CF80700606920F0004060610F6989
:107FF000E568042F2FD004F16000C5F3C10550F8E7
:1080000027E0DFF85CC26E000D680EEA0C0C05F08C
:10801000F84545EA0C0C4D69B54045EA0C0545F0BC
:10802000004540F827500F698E6950F8275025F019
:108030008075354340F827500D7F0E69012D50F8AB
:10804000265008BF4FF0007225F000752A4340F813
:108050002620086866E70868226E226EC0F31205C3
:10806000C2F38462002D40F0FD80C0F38465AA4213
:1080700000F07181626E666E04F16002C6F3846680
:1080800004F16407AE4200F054819668966802F1EC
:108090000807C6F38466AE4200F03981D668D66818
:1080A00002F10C07C6F3846295427FF43BAF3A6855
:1080B00022F000423A60086834E7D4F8B020C0F3F8
:1080C00012052A43C4F8B020002D50D090FAA0F237
:1080D000002A00F0F880B2FA82F2013202F01F02A8
:1080E000092A40F2F08090FAA0F2002A00F04F81B5
:1080F000B2FA82F20132920602F0F84290FAA0F54A
:10810000002D00F04981B5FA85F5013505F01F0510
:10811000012606FA05F5154390FAA0F0002800F0B4
:108120003981B0FA80F0421C02F01F006FF01D068A
:10813000032212FB0062120542F000722A43D60DA0
:10814000886806F0040604F11405C2F3045200FA2C
:1081500002F74FF0070C70590CFA02F220EA020203
:108160003A4372510A68EFE6022003B0F0BD800E78
:10817000013000F01F06092E50D885060122B240BA
:1081800005F0F845154306EB46021205D6E72C49E3
:1081900030488A6822F0E072164346F400068E608A
:1081A00002682D499209A1FB02129209013202EBE9
:1081B000420292000192019A002A3FF4F3AE019A22
:1081C000013A0192019A002AF9D1EBE6234DAA4225
:1081D0007FF4E8AE10F480007FF4E4AE1C4A9442D1
:1081E0003FF4E0AE8A6822F0E072324342F480024B
:1081F0008A60CCE6F50D04F1140005F00405C6F321
:1082000004562F584FF0070C0CFA06F627EA06061C
:108210002E50606940F000406061E8E606EB4602DF
:1082200085061E3A012005F0F845120500FA06F60B
:1082300042F00072354381E700007F400000088073
:1082400000030050000021C31000C090000052C77E
:10825000000100506C070020632D3E05000084CB18
:1082600000F0FF0390FAA0F51DB1B5FA85F5AA421A
:1082700071D0626E666E04F16002C6F3846604F12A
:10828000640790FAA0F51DB1B5FA85F5AE4250D05D
:108290009568966802F10807C6F3846690FAA0F51F
:1082A0001DB1B5FA85F5AE4231D0D568D56802F179
:1082B0000C07C5F3846290FAA0F5002D3FF432AEAE
:1082C000B5FA85F5F0E690FAA0F2002A59D0B2FA94
:1082D00082F20132920602F0F84290FAA0F5002DE7
:1082E0004DD0B5FA85F5013505F01F05012606FAD2
:1082F00005F5154390FAA0F0002845D0B0FA80F0BB
:10830000013000F01F0000EB4000020516E738685E
:1083100020F000403860D068086802F10C07D2688D
:10832000C0F31205C2F38462002DC4D1C0F384658A
:10833000BAE6386820F000403860906808689668AF
:10834000C0F3120502F10807C6F38466002DA5D11B
:10835000C0F384659FE6206E224620F0004042F87C
:10836000600F606E0868666EC0F3120504F1640762
:10837000C6F38466002D84D1C0F3846582E60225AD
:10838000B7E74FF08062A8E74FF44012D6E64FF00F
:108390008062B3E6014AD1E60225BCE6000050FE49
:1083A00090F858204B68012A00F0FF8030B5012278
:1083B000046880F85820A2685207844635D5A3681F
:1083C0000A68B74B9A4276D0E36803F01803182B7B
:1083D00000F0CF80E3680869C3F3C103C3F102036F
:1083E0005B0003F01E03D840E36803F01803182B6A
:1083F0004B6900F0BC80E168C1F3C101C1F1020129
:10840000490001F01E01CB40920C02F00C02203416
:1084100043EA0043115901F0F0214FF0000E0B43E5
:1084200013518CF858E0704630BDA26812F0080F66
:108430000A68C6D19A4882424DD0B3F1A07F00F0BD
:10844000A28000F29980B3F5400F00F09C80B3F158
:10845000807F00F0DC80B3F5000F00F0D88002F0E0
:108460000100C2F3015300EBC00003EB800304F1F1
:108470000C0522F0024255F8230022F4601220EA93
:10848000020245F82320874B0A689A4200F0AC802C
:10849000DCF85C3023F48023CCF85C304FF40073BC
:1084A00023600B7B012B63680CBF43F4007323F440
:1084B0000073636085E7E068E368C3F3C1034FEAD4
:1084C000430EC0F3C1000B69400003FA00F04B6992
:1084D00003FA0EF398E7B3F1A07F00F0C78027D826
:1084E000B3F5400F00F0B580B3F1807F33D1E3687E
:1084F00023F0FB4323F4800343F08073E360236A9B
:108500008A6923F4E04313432362DCF85C30802261
:1085100023F48033CCF85C3022600B7B0A68012B9B
:1085200063680CBF43F0800323F08003636048E777
:10853000B3F1C07F3BD0B3F1E07F41D1E2688B68FB
:1085400022F0FB4203F0F84322F48002134343F08D
:10855000E073E360D3E7B3F5000F31D1E36823F0B4
:10856000FB4323F4800343F40003E360C7E79B006D
:108570004AE70B69980037E7B3F1C07F47D0B3F102
:10858000E07F7FF46CAF474B9A428B681FD0C3F3F8
:108590001200002855D1C3F3846301209840D4F819
:1085A000A4300343C4F8A43072E702207047E368A4
:1085B00023F0FB4323F4800343F0C073E3609EE7A2
:1085C000E36823F0FB4323F48003E36097E7C3F3FE
:1085D0001202002A57D1C3F3846301229A40D4F8CF
:1085E000A0301343C4F8A030DCF85C304FF4807244
:1085F00023F40033CCF85C3022600B7B012B6368E2
:108600000CBF134323F48073264A6360DCE602F058
:108610000103C2F3015E03EBC3030EEB830E04F10F
:108620000C0022F0024550F82E3025F4601522F09F
:108630007E4222F4F00223EA05031A4340F82E207A
:1086400021E793FAA3F333B3B3FA83F301209840FD
:10865000A5E7E2688B6822F0FB4203F0F84322F4BE
:108660008002134343F44003E36048E7E2688B6809
:1086700022F0FB4203F0F84322F48002134343F05C
:10868000A073E3603BE793FAA3F333B1B3FA83F348
:1086900001229A40A3E7012081E701229FE700BF62
:1086A0000000C07DFFFF170003689A68520770B58D
:1086B000044636D59A68DA68960104D5A08B40F254
:1086C0000112904232D002299A680ED0520702D588
:1086D0009A68960756D501293AD09A68100739D476
:1086E000032914BF04250C2502E010073ED40825F9
:1086F00000F04AFA236806469B681D4214D000F039
:1087000043FA831B052B2368F6D99A682A42F3D0D3
:10871000E36D43F01003E365236E012003432366FA
:1087200070BD9A681607C6D4002070BD1A68550639
:1087300006D41E4A01E0013AEAD019684806FAD583
:1087400040221A609A68510702D59A68920722D58A
:108750000425CDE79A689207C2D49A6822F00042B5
:1087600022F03F0242F020029A60B9E79A6891072E
:10877000BDD49A6822F0004222F03F0242F020026B
:108780009A60B4E79A6822F0004222F03F0242F079
:1087900010029A609FE79A6822F0004222F03F029E
:1087A00042F0100204259A60A2E700BF000040A337
:1087B00003689A68D20701D5002070479968184A63
:1087C000114270B5064608D0F36D43F01003F3650F
:1087D000336E01200343336670BD9A68114D2A4001
:1087E00042F001029A6000F0CFF9336804461A683B
:1087F000D00713D49A68D10704D49A682A4042F06B
:1088000001029A6000F0C0F9031B022B3368EED915
:108810001A68D207D8D51A68D007EBD5002070BDEA
:108820003F000080C0FFFF7F2DE9F041374B056816
:108830009B68AD686C0714D4164690F85820012A3E
:1088400004460ED003F01F08B8F1090F4FF00103E2
:1088500080F8583008D9002384F858300120BDE84A
:10886000F0810220BDE8F08140F2212323FA08F3D1
:10887000DB4313F00105EED10F46FFF799FF002807
:108880003BD1E36D216823F4706323F0010343F4CB
:108890008073E3651E4B994233D0E36D23F480135C
:1088A000E365E36D606D1B4D13F480531CBF236EB5
:1088B00023F006032366C562174D0563174D456314
:1088C0001C250D60002584F858504D6845F01005B2
:1088D0004D60CD6845F0010533463A46CD604031E4
:1088E00001F034F82268936823F0004323F03F033B
:1088F00043F004039360BDE8F08184F85850BDE86C
:10890000F081B8F1000FC8D0CBE700BF00030050E2
:1089100000010050417E0008E57B0008AD7E0008A4
:1089200038B503689A68950702D59B68002038BD62
:108930009A68D4072BD59A6802F00D02012A0446E2
:1089400008D0E36D43F01003E365236E0120034379
:10895000236638BD9A6822F0004222F03F020321CC
:1089600042F002029A60196000F00EF923689B68D9
:10897000D90705460BD500F007F9401B02282368EC
:1089800002D99A68D207DCD49B68DB07F3D40020B5
:1089900038BD00BF38B590F85830012B28D00123DE
:1089A00080F8583003210446FFF77EFE0546D0B913
:1089B0002368606DDA6822F00102DA6090F8252001
:1089C000022A18D05A6822F010025A602046FFF797
:1089D000A7FF054638B9E36D23F4885323F001035C
:1089E00043F00103E365002384F85830284638BD7E
:1089F0000225284638BD01F003F8054660B1E36D55
:108A0000226843F04003E365536823F010032046D7
:108A10005360FFF785FFE6E72268536823F01003F1
:108A20005360D3E7704700BF704700BF704700BF77
:108A3000704700BF704700BFF0B490F858200D6831
:108A4000012A9CB04FD00468034600220120B4F1F3
:108A5000A04F189283F85800199208D0D96D83F866
:108A6000582041F02001D9651CB0F0BC7047234A62
:108A7000906840070BD5A268DA6D42F02002012011
:108A8000DA65002283F858201CB0F0BC7047A0685B
:108A90004607F1D4D5B11A4E4F68B06893F838C084
:108AA00020F46040384340EA4C30B060A4689068DD
:108AB000204310F0010014D18A681543B26822F4F3
:108AC000716222F00F021543B560DAE70C4DA96818
:108AD00021F46041A960A1689068084310F001008A
:108AE00005D00020CDE702201CB0F0BC7047AA687A
:108AF00022F4716222F00F02AA60C2E70001005066
:108B00000003005038B50F4B1B680BB9012038BD6E
:108B10000D494FF47A720546B2FBF3F30868B0FBD7
:108B2000F3F001F017F904460028EFD10F2DEDD82E
:108B3000024629464FF0FF3001F0C0F8034B2046B3
:108B40001D6038BD640700206C0700206807002006
:108B500010B5032001F0A0F80020FFF7D3FF10B1FB
:108B60000124204610BD0446FEF78AFC204610BDB5
:108B7000034A0449136809680B441360704700BF37
:108B80004853002064070020014B1868704700BF5D
:108B90004853002038B50446FFF7F6FF631C05462E
:108BA00002D0044B1B681C44FFF7EEFF431BA3429B
:108BB000FAD338BD64070020002800F0C3812DE9F6
:108BC000F0410368D90782B004462DD5A6498A68CA
:108BD000C96802F00C020C2A00F00A81082A00F091
:108BE0000C816368B3F5803F00F03381B3F5A02FAB
:108BF00000F09B819C4D2A6822F480322A602A680A
:108C000022F480222A60002B40F02881FFF7BCFF6D
:108C1000064605E0FFF7B8FF801B642800F242819A
:108C20002B689F03F6D423689E0728D58E4A936845
:108C3000D26803F00C030C2B00F0EC80042B00F046
:108C4000EE80E368884D002B00F01D812B6843F413
:108C500080732B60FFF798FF064605E0FFF794FF4F
:108C6000801B022800F21E812B685805F6D56B6820
:108C7000226923F0FE4343EA02636B6023681A070C
:108C800019D56369784D002B00F09E80D5F894309B
:108C900043F00103C5F89430FFF776FF064605E080
:108CA000FFF772FF801B022800F2FC80D5F8943099
:108CB0009F07F5D52368590741D56B4B9A6DD200B4
:108CC00000F1F4809A6D42F080529A659B6D03F03A
:108CD00080530193019B0125644E3368DF0540F109
:108CE0001381A368012B00F0E380052B00F069815C
:108CF0005D4ED6F8902022F00102C6F89020D6F8FA
:108D0000902022F00402C6F89020002B40F0D7807B
:108D1000FFF73AFF41F28838074605E0FFF734FFD6
:108D2000C01B404500F2BE80D6F890309A07F5D4BB
:108D300025B14D4A936D23F08053936523689B06BC
:108D400018D5A369484D002B00F0CA80D5F898309B
:108D500043F00103C5F89830FFF716FF064605E01B
:108D6000FFF712FF801B022800F29C80D5F8983094
:108D70009F07F5D5E06918B33B4DAB6803F00C03D2
:108D80000C2B00F02C812B68022823F080732B60C1
:108D900000F0DA80EB6823F00303EB60EB6823F06C
:108DA000887323F48033EB60FFF7EEFE044604E0A3
:108DB000FFF7EAFE001B022874D82B689B01F7D44A
:108DC000002002B0BDE8F081D5F8943023F0010313
:108DD000C5F89430FFF7D8FE064604E0FFF7D4FE4E
:108DE000801B02285ED8D5F894309807F6D461E746
:108DF00001F0030103297FF4F4AE1B4A12689203C9
:108E00007FF512AF6268002A7FF40EAF012002B036
:108E1000BDE8F08102F00302022A7FF412AF124B88
:108E20001B685D0502D5E368002BEFD00E4A206970
:108E300053680F4923F0FE4343EA00635360086818
:108E4000FFF760FE0028E1D123681A077FF533AFF2
:108E500017E7054A136843F480331360FFF794FE65
:108E6000014E05460BE000BF0010024000700040BC
:108E700068070020FFF788FE401B642812D833687B
:108E80009B03F7D5CFE62B6823F480732B60FFF7A5
:108E90007BFE06462B685905D6D5FFF775FE801B6D
:108EA0000228F7D9032002B0BDE8F081002513E7BE
:108EB000654AD2F8903043F00103C2F89030FFF7D2
:108EC00063FE614F064641F2883804E0FFF75CFE1E
:108ED000801B4045E6D8D7F890309907F6D527E7AC
:108EE000D5F8983023F00103C5F89830FFF74CFE11
:108EF000064604E0FFF748FE801B0228D2D8D5F8CA
:108F000098309807F6D435E7336843F480733360BC
:108F1000FFF73AFE07463368D8053FF5E2AEFFF7A4
:108F200033FEC01B0228F6D9BCE703F18043A3F54A
:108F30003C331A6842F480221A601A6842F4803284
:108F40001A608BE701207047FFF71EFE064604E01B
:108F5000FFF71AFE801B0228A4D82B689901F7D4CA
:108F6000E9683A4B226A606A374E0B401343D4E9F2
:108F70000A1243EA012343EAC263D4E90C1201381E
:108F8000490843EA00130139520843EA4153013AC0
:108F900043EA4263EB602B6843F080732B60EB681D
:108FA00043F08073EB60FFF7EFFD044605E0FFF749
:108FB000EBFD001B02283FF675AF33689A01F6D52A
:108FC000FEE6214BD3F8902042F00402C3F8902033
:108FD000D3F8902042F00102C3F890206FE70128F7
:108FE0003FF4EFAEEB68226A03F0030191427FF495
:108FF0000DAF616A03F0F0020139B2EB011F7FF49B
:1090000005AFA16A03F4FE42B2EB012F7FF4FEAE7E
:10901000E16A03F07842B2EBC16F7FF4F7AE226BE6
:10902000520803F4C001013AB1EB425F7FF4EEAEA7
:10903000626B520803F0C063013AB3EB426F14BF96
:1090400001200020BDE600BF001002400C809F01FF
:10905000F0B587B00223029303250023CDE9033541
:109060000F4F04461646C0F30340FA6C01238340B9
:109070001343FB6400F59010A3B201930D46C4F3B3
:109080000753800201A9059300F0CCFAE30005D450
:10909000BA6822F0FE4216433543BD6007B0F0BD0A
:1090A00000100240184B9A6802F00C02042A27D0E4
:1090B0009A6802F00C02082A24D09A6802F00C0286
:1090C0000C2A01D000207047D968D86801F003014C
:1090D0000329C0F3031000F10102D8680CBF0B4B49
:1090E0000B4BB3FBF2F2084BDB68C3F34163C0F3F5
:1090F0000620013302FB00F05B00B0FBF3F0704789
:1091000003487047014870470010024000366E0166
:109110000024F400002800F0EE807F4A2DE9F84397
:10912000136803F00F038B420D4604460CD21368FC
:1091300023F00F030B431360136803F00F038B42FC
:1091400002D00120BDE8F8832368DF0763D5626899
:10915000032A00F09A80714B022A1B6800F091806C
:109160005B05EED5FFF79EFF6D4B984200F2C58080
:1091700062684FF00009694EB36823F003031A4395
:10918000B260FFF701FD41F28838074604E0FFF7BF
:10919000FBFCC01B404571D8B368626803F00C0348
:1091A000B3EB820FF3D123689F0736D4B9F1800F58
:1091B00003D1B36823F0F003B360574E336803F074
:1091C0000F03AB4246D823685A0706D55349E068D7
:1091D0008A6822F4E06202438A601B0707D54F4A7F
:1091E0002169936823F4605343EAC1039360FFF756
:1091F00059FF4A4A4B4C92684B49C2F3031203464B
:10920000A25C4A4802F01F02D3400B600068BDE830
:10921000F843FFF777BC9E07CFD5580704D53F49E1
:109220008A6842F4E0628A60190706D53B4A93686F
:1092300023F47C5343F4E0639360384AA168936855
:10924000354E23F0F0030B439360336803F00F03B4
:10925000AB42B8D9336823F00F032B433360FFF7D9
:1092600093FC41F288380746336803F00F03AB42A2
:10927000A9D0FFF789FCC01B4045F5D90320BDE804
:10928000F8839A033FF56EAF5BE7244908688001D5
:109290007FF557AFCE68C868C968214F06F003064E
:1092A000032EC0F303100CBF214E224E0130B6FB3B
:1092B000F0F01A4EC1F3062100FB01F1F068C0F393
:1092C000416001304000B1FBF0F1B94220D9B168F2
:1092D00011F0F00F05D013F002093FF44CAFA36872
:1092E000B3B90E498B6823F0F00343F080038B6021
:1092F0004FF080093FE701207047084A93684FF01C
:10930000800923F0F00343EA09039360626832E7BF
:109310004FF000092FE700BF00200240001002407C
:1093200000B4C404FCCE00086C07002068070020CD
:1093300000366E010024F400014B1868704700BF2E
:109340006C070020054B064A9B680649C3F30223BD
:109350000868D35C03F01F03D84070470010024038
:109360000CCF00086C070020054B064A9B68064995
:10937000C3F3C2230868D35C03F01F03D8407047CF
:10938000001002400CCF00086C0700202DE9F041CE
:109390000368044613F4002082B056D09F4B9A6DA8
:1093A000D50040F10C8100279D4D2B6843F480735C
:1093B0002B60FFF7E9FB064605E0FFF7E5FB831BA3
:1093C000022B00F207812B68D805F6D5934DD5F80E
:1093D000903013F4407327D0226C9A4225D0D5F8F0
:1093E0009010D5F8903043F48033C5F89030D5F81C
:1093F000903023F48033C5F8903021F44073C907CE
:10940000C5F8903040F10881FFF7BEFB41F2883883
:10941000064605E0FFF7B8FB801B404500F2DA8006
:10942000D5F890309B07F5D5236C7C49D1F8902076
:1094300022F440721343C1F89030002027B1774ADC
:10944000936D23F0805393652368DE0708D5734935
:109450006568D1F8882022F003022A43C1F88820E9
:109460009D0708D56D49A568D1F8882022F00C0227
:109470002A43C1F88820590708D56849E568D1F81A
:10948000882022F030022A43C1F888201A0708D524
:1094900062492569D1F8882022F0C0022A43C1F828
:1094A00088209F0608D55D496569D1F8882022F497
:1094B00040622A43C1F888205E0608D55749A5694D
:1094C000D1F8882022F440522A43C1F888201D0692
:1094D00008D55249E569D1F8882022F440422A4350
:1094E000C1F88820D90508D54C49256AD1F88820CB
:1094F00022F440322A43C1F888209A0508D547490A
:10950000656AD1F8882022F440222A43C1F88820D5
:109510005F050BD54149A56AD1F8882022F4401295
:109520002A43B5F5801FC1F8882055D01E050BD5FC
:109530003A49E56AD1F8882022F440022A43B5F579
:10954000800FC1F888204CD0DD040BD53349256B42
:10955000D1F8882022F040722A43B5F1807FC1F80B
:10956000882043D099040BD52C49656BD1F888200D
:1095700022F040622A43B5F1006FC1F888203AD04A
:109580005A040BD52549A56BD1F8882022F04062FA
:109590002A43B5F1006FC1F8882031D01B040BD5E8
:1095A0001E4AE16BD2F8883023F040530B43B1F1EF
:1095B000805FC2F8883028D002B0BDE8F0819A6D93
:1095C00042F080529A659B6D03F080530193019B9A
:1095D0000127E9E6032031E7CA6842F48012CA6035
:1095E000A4E7CA6842F48012CA60ADE7CA6842F4D0
:1095F0008012CA60B6E7CA6842F48012CA60BFE748
:10960000CA6842F48012CA60C8E7D36843F4803362
:10961000D36002B0BDE8F081134606E700100240B7
:10962000007000402DE9F04F0C6885B0002C00F070
:1096300083804FF0000CDFF8D8A163464FF0010B98
:1096400089460BFA03F515EA04086FD0D9F80470BF
:1096500007F00302511E012971D9032A40F0B0809E
:1096600002FA0CF2D143056829400A4317F4403F3F
:1096700002605BD0DAF8602042F00102CAF8602094
:10968000DAF8602002F001020392039A23F0030249
:1096900002F1804202F5803203F003059168AD00CB
:1096A0000F2606FA05FEB0F1904F21EA0E0119D0FF
:1096B000514EB04200F08F80504EB04200F08F808B
:1096C0004F4EB04200F081804E4EB04200F08D808F
:1096D0004D4EB0420CBF4FF0050E4FF0060E0EFA85
:1096E00005F529439160494A484992686FEA08059F
:1096F000FE0254BF2A4048EA02028A60CA68B902E0
:10970000424954BF2A4048EA0202CA6049683F4AB7
:10971000BE0354BF294048EA010151601268F903B1
:109720003A4954BF2A4048EA02020A60013334FA37
:1097300003F20CF1020C84D105B0BDE8F08F816812
:10974000D9F80C604FF0030E0EFA0CFE21EA0E0160
:1097500006FA0CF6314381606FEA0E01D0F804E09E
:109760002EEA050EC7F300159D4045EA0E0545603B
:10977000C56805EA010ED9F8085005FA0CF545EA66
:109780000E05022AC56002FA0CF27FF46CAFDD0808
:1097900000EB850501952E6AD9F81050009603F06C
:1097A000070E4FEA8E0E0F2605FA0EF506FA0EFE8C
:1097B000009E26EA0E0E019E45EA0E05356252E72E
:1097C000032101FA0CF1C943D2E74FF0030E0EFA60
:1097D00005F5294386E70BFA05F5294382E74FF0A3
:1097E000020E0EFA05F529437CE74FF0040E0EFA3F
:1097F00005F5294376E700BF00040048000800484B
:10980000000C00480010004800140048000401400B
:10981000001002400AB1816170478162704700BF49
:10982000002878D070B53D4B04689C425FD93C4A13
:109830003C4B3D492244A3FB023212099200022311
:10984000856880F82530C368C669C0E910120169CF
:109850002B430B4341690B4381690B4333435FFA4D
:1098600084FC304E2168ACF1080CA6FB0C6C066A37
:1098700021F4FF4121F0700133430B4323602B4E51
:10988000264B2B49CCF3041C9C4298BF31464FF029
:10989000010E284CC4640EFA0CF35418B5F5804F31
:1098A000036584644FEA92022AD04568ECB2013D18
:1098B000032D41F82240C6F8843027D81E4B1F499B
:1098C0002344013C9B0004F01F040EFA04F4002220
:1098D000C0E91531C4651A60194B5C64002301228C
:1098E000C36380F8243080F82520184670BD154ADF
:1098F0000C4B15492244A3FB0232120992009EE749
:109900000024446041F82240C6F884300023C0E9B6
:109910001533C365E2E70120704700BF070402402A
:10992000F8FBFDBFCDCCCCCC0004024000080240C7
:1099300020080240800802403F8200104009024097
:1099400000090240F8FFFDBF00000240F0B490F8AB
:109950002440012C51D0012480F8244090F8254067
:10996000012C05D0002380F82430F0BC0220704781
:10997000022480F825400024C4630468C66C25686E
:1099800025F001052560D0E91475776015B1D0E99F
:1099900016677760466C076C06F01F0C012606FA06
:1099A0000CF67E6063608368102B036B0BBFA260B4
:1099B000A160E160E260BBB1236843F00E03236065
:1099C000836C1A68D20303D51A6842F480721A6055
:1099D0001DB12B6843F480732B60236843F00103AF
:1099E00000202360F0BC7047236823F00403236049
:1099F000236843F00A032360E2E70220F0BC7047CB
:109A000090F82520022A034609D00422C2630121CE
:109A10000022012083F8251083F824207047026873
:109A2000596C30B4846C10681D6C20F00E0010600E
:109A3000206820F4807020601068DC6C20F0010049
:109A4000106001F01F0101228A40D3E914106A60FE
:109A5000616038B10268D3E9161422F480720260A2
:109A60004C6000200121002283F8251083F8242077
:109A700030BC704738B590F82530022B09D001234F
:109A800004210022C16380F8242080F82530184684
:109A900038BD0368846C1968426C056C21F00E01B6
:109AA0001960196821F0010119602368C16C23F461
:109AB0008073236002F01F0201239340D0E9144217
:109AC0006B604C6032B11368D0E9161423F48073D4
:109AD00013604C60836B0122002480F8252080F8FD
:109AE000244013B19847204638BD184638BD00BF02
:109AF00070B4436C066C056831682C6803F01F0372
:109B000004229A400A420ED014F0040F0BD02B68A6
:109B10009B0603D42B6823F004032B60036B726055
:109B2000CBB170BC184702229A400A4215D014F0FB
:109B3000020F12D02B68990606D42B6823F00A0373
:109B40002B60012380F82530C36A7260002180F801
:109B50002410002BE5D170BC704708229A400A42BD
:109B6000F9D02207F7D52A68416B22F00E022A604D
:109B7000012202FA03F300247360C26380F82440D8
:109B800080F825200029E6D070BC084710B43B4A75
:109B900070B9136803F4C063B3F5806FD2F88030F6
:109BA00023D023F480735DF8044BC2F880307047F3
:109BB000B0F5007F09D013685DF8044B23F4C0634F
:109BC00043F48063002013607047136803F4C0639C
:109BD000B3F5806FD2F880302FD043F4807300202B
:109BE0005DF8044BC2F88030704723F48073C2F8EC
:109BF00080301168224C234821F4C06141F4007187
:109C000011602368322101FB03F35169A0FB0303B8
:109C10009B0C480503F1010306D500E023B151690F
:109C2000490503F1FF33F9D4144B5B695C0554BF5C
:109C3000002003205DF8044B704743F48073C2F8A2
:109C4000803011680E4C0F4821F4C06141F400715E
:109C500011602368322101FB03F35169A0FB030368
:109C60009B0C480503F10103DED501E0002BDBD09E
:109C70005169490503F1FF33D6D5F7E7007000407D
:109C80006C07002083DE1B43024A936843F4804341
:109C900093607047007000400749CA6803024FF69E
:109CA000FF0003F4E0630240134343F0BF6343F457
:109CB0000033CB60704700BF00ED00E01C4BDB6859
:109CC000C3F3022300B5C3F1070EBEF1040F03F185
:109CD000040C28BF4FF0040EBCF1060F1BD9033B48
:109CE0004FF0FF3C0CFA03FC22EA0C024FF0FF3C61
:109CF0000CFA0EFC21EA0C019940002841EA02010D
:109D00000CDB00F16040090100F56140C9B280F848
:109D100000135DF804FB00221346E7E7054B00F053
:109D20000F0009010344C9B219765DF804FB00BFB6
:109D300000ED00E0FCEC00E0002808DB044A4109EB
:109D4000012300F01F0003FA00F042F821007047E1
:109D500000E100E00138B0F1807F10D210B44FF084
:109D6000E023084C58614FF0F00C84F823C0002227
:109D7000072110469A615DF8044B19617047012074
:109D8000704700BF00ED00E0B0B110B590F8213091
:109D9000044603F0FF0253B100200123606284F8FF
:109DA0002130C4E90100C4E90300606110BD80F8FE
:109DB0002020FDF707FCEFE70120704790F82120F5
:109DC000012A034605D0426A42F0020201205A628B
:109DD000704788690A6810B44C680243186842EA00
:109DE0000403D1E9044223431343D1E90221046867
:109DF0001343044A0B432240134303605DF8044BB2
:109E00000020704700F887FF88B110B50379044639
:109E100003F0FF023BB100230221012221712361E3
:109E20002271184610BD4271FDF7E4FBF3E70120F3
:109E3000704700BFF8B54379012B2ED004460226A7
:109E400022682671012060710D4605F01007116827
:109E500000FA07F30B431360FEF79CFE22686DB90E
:109E6000136803F03E03B34203D1536843F0010388
:109E700053600020012323716071F8BD1368BE4058
:109E800003F47813B342F4D1536843F002035360F0
:109E90000020012323716071EFE70220F8BD00BFAD
:109EA000026838B501F010011368012505FA01F1C7
:109EB000044623EA010128461160FEF76BFE257176
:109EC000002038BDF8B504464079069E01285ED0D2
:109ED0000D461146012262710222276822713DBBA4
:109EE000A0683A68DFF8D0C0C0F82CC0DFF8CCC05A
:109EF000C0F830C042F48052DFF8C4C0C0F834C0AB
:109F0000042E3A604CD0082E47D0002E42D02A466C
:109F10003E6846F400563E60FFF718FD00230646F3
:109F200063713EB3236943F0040323613046F8BDF7
:109F3000E0683A68DFF88CC0C0F82CC0DFF888C051
:109F4000C0F830C042F08052DFF880C0C0F834C0A2
:109F5000042E3A602DD0082E28D026B300223E6869
:109F600046F000563E60FFF7F1FC002306466371A1
:109F7000002ED7D1236801201A6805F0100500FAD9
:109F800005F515431D60FEF705FE3046F8BD0226B7
:109F90003046F8BD07F10802BAE707F11002B7E74B
:109FA00007F10C02B4E707F11402D8E707F11C022D
:109FB000D5E707F11802D2E731A0000841A0000858
:109FC00051A0000831A2000841A2000851A20008D7
:109FD00038B503680D4605F01002196804464FF4C1
:109FE0008050904021EA000119601968012000FAB0
:109FF00002F221EA02021A60FEF7CCFD5DB9A06808
:10A00000FFF7FEFC2268136823F40053136001235A
:10A010002371002038BDE068FFF7F2FC2268136866
:10A0200023F00053136001232371002038BD00BFCB
:10A0300010B5846A2046FAF79BF90123237110BDFD
:10A0400008B5806AFAF788F908BD00BF704700BFFD
:10A0500010B5846A236943F0040323612046FFF7A7
:10A06000F5FF0123237110BD2DE9F04143798F687D
:10A07000012B00F0C68001234371042F4FF002032F
:10A0800006460D461446037177D0036802F01004AB
:10A09000EA69012A08D1996B2A6A1F20A040A240D0
:10A0A00021EA00010A439A63A969D86B07220129B2
:10A0B00002FA04FC6A695ED0022916BFB2FA82F184
:10A0C0000121490911432A79012A4FF400724FF402
:10A0D000807802FA04F208FA04F842EA0C0220EA54
:10A0E00002026FEA080808EA02086A7947EA0107EB
:10A0F00008BF47F48077012A2A6808BF47F4007731
:10A10000022A28F4404873D048EA0208A74047EAE8
:10A110000807DF631A684FF48041A14022EA010278
:10A120001A60D5E90312186840F6FE75A54020EACA
:10A130000505920101FA04F02843C1F3830102F4FA
:10A14000706218600A4340F60F7101FA04F0C025EE
:10A150001968A24005FA04F421EA04041C60196E8F
:10A1600021EA000100240A4301211A6620463171C8
:10A170007471BDE8F0810021A4E7FEF705FD0746F4
:10A180002CB114E0FEF700FDC31B012B3CD8336853
:10A190005B6B1B04F6D40120FEF7FCFC33686A6A93
:10A1A0001A640EE0FEF7F0FCC31B012B2CD83368B9
:10A1B0005B6B002BF6DB0120FEF7ECFC33686A6A70
:10A1C0005A649A6CA96AAF6804F0100440F2FF3038
:10A1D000A040A14022EA00020A439A64DA6CE96ACC
:10A1E000FF20A040A14022EA00020A43DA644FE7C0
:10A1F000FFF7A2F80C4B98420ED9336848F4004898
:10A2000084E70220BDE8F0813369032243F00803AC
:10A21000336110463271ACE7044B984288BF48F472
:10A220008048336872E700BF0068890900B4C4043D
:10A2300010B5846A2046FAF7B1F80123237110BDE6
:10A2400008B5806AFAF79EF808BD00BF704700BFE6
:10A2500010B5846A236943F0040323612046FFF7A5
:10A26000F5FF0123237110BD2DE9F04782460E460C
:10A2700017464FF02008DAF800309D6915F0020506
:10A2800040F0C7809A6912F0100251D01022DA61B2
:10A29000B946741C9A6951D1900600F1B180002D25
:10A2A00040F0B1809C69A106FCD5C3F81C800D204C
:10A2B00007244FF0050C04220125996911F4807FD1
:10A2C00027D04FF480724E05DA6126D48D0579D4FB
:10A2D00060469A69940744BF00229A629A69D1073E
:10A2E00003D49A6942F001029A615A684B4C2240A9
:10A2F0005A60DAF84430002103432022CAF844307F
:10A300008AF840108AF8412001208AF84210BDE8FE
:10A31000F087480551D542F008004FF480628C0563
:10A32000DA61D6D540F002004FF40072DA61D0E76E
:10A33000092003244FF0010C1546BEE792065FD4B6
:10A34000002D60D1FEF720FCA0EB09008642DAF870
:10A35000003001D3002E9CD158689AF842209969A8
:10A360000C04D2B20FD541040DD4202A0BD05A6868
:10A3700042F480425A60FEF707FCDAF8003081466A
:10A3800001E0DAF800309C6914F0200481D1FEF776
:10A39000FBFBA0EB09001928F3D9DAF84420DAF81E
:10A3A00000308AF8404042F02002CAF844200125DB
:10A3B0008AF841808AF84240E5E7890504D542F0F1
:10A3C0000200B1E72046AFE735BB721C3FF455AF42
:10A3D000FEF7DAFBC01BB04202D8002E7FF44BAF71
:10A3E000DAF84430002243F020032021CAF8443038
:10A3F0008AF840208AF8411001208AF8422086E736
:10A40000002D3FF452AF0D2007244FF0050C04221D
:10A4100053E70020BDE8F08710465AE700E800FE49
:10A420002DE9F04782460E4617464FF02008DAF82D
:10A4300000309D6915F0200540F0C5809A6912F042
:10A44000100251D01022DA61B946741C9A6951D1B8
:10A45000900600F1AF80002D40F0AF809C69A1060E
:10A46000FCD5C3F81C800D2007244FF0050C0422F6
:10A470000125996911F4807F27D04FF480724E0531
:10A48000DA6126D48D0579D460469A69910744BF74
:10A4900000229A629A69D20703D49A6942F00102B3
:10A4A0009A615A684A4C22405A60DAF844300021D6
:10A4B00003432022CAF844308AF840108AF8412029
:10A4C0008AF842100120BDE8F087480551D542F0D6
:10A4D00008004FF480628C05DA61D6D540F00200A6
:10A4E0004FF40072DA61D0E7092003244FF0010C29
:10A4F0001546BEE792065DD4002D5ED1FEF744FB03
:10A50000A0EB09008642DAF8003001D3002E9CD17E
:10A5100058689AF8422099690C04D2B20FD54104C8
:10A520000DD4202A0BD05A6842F480425A60FEF7BC
:10A530002BFBDAF80030814601E0DAF800309C6944
:10A5400014F0200481D1FEF71FFBA0EB09001928AD
:10A55000F3D9DAF844308AF8404043F02003CAF8CF
:10A56000443001258AF84180DAF800308AF8424008
:10A57000E5E7880504D542F00200B1E72046AFE7E1
:10A5800025BBFEF701FBC01BB04202D8002E7FF4B2
:10A590004EAFDAF84430002243F020032021CAF8FD
:10A5A00044308AF840208AF841108AF8422001207D
:10A5B000BDE8F087002D3FF454AF0D2007244FF085
:10A5C000050C042255E70020BDE8F08710465CE743
:10A5D00000E800FE00284FD010B590F84130044646
:10A5E00003F0FF02002B42D02368242284F841208C
:10A5F0001968626821F0010122F0706219601A6125
:10A600009A68E16822F4004201299A60A2682AD07F
:10A6100042F4044202299A6004BF4FF400625A6077
:10A620005968226941F0007141F400415960616943
:10A63000D8680A43A16920F4004042EA0122E16996
:10A64000D860206ADA6001431960196841F001019D
:10A65000196000222023626484F84130226384F868
:10A660004220104610BD42F400429A60D8E780F8BC
:10A670004020FDF743F8B7E7012070472DE9F84F78
:10A680009A4690F84130BDF82CB0DDF83080202B90
:10A6900040F0A4800A9B0446002B00F09980BBF197
:10A6A000000F00F0958090F84030012B00F096806C
:10A6B000012380F840300F469146FEF765FA0646C2
:10A6C00005E0FEF761FA801B192800F28A802368F2
:10A6D0009D6915F40045F4D10A9A6262212284F83A
:10A6E0004120402284F842206564A4F82AB05A68C8
:10A6F000764965630A405FFA8AF142EA0142C7F38C
:10A7000009073A4342F0807242F400525A604146CF
:10A7100032462046FFF7A8FD002840F09680BAF1A7
:10A72000010F40F0868022685FFA89F39362B8F1E6
:10A73000FF3F65D193691D06FCD5638D9BB2FF2B4E
:10A740006BD8638D62489BB22385D9B253680340AE
:10A750003B4343EA014343F0007353605C4DDFF831
:10A7600078A14FF0FF0904E0638D9BB2002B00F04D
:10A770008D80324641462046FFF776FD002840F0A6
:10A780008380636A226813F8011B91626362638DA0
:10A79000013B9BB26385238D618D013B9BB289B2E6
:10A7A00023850029E0D0002BDED1B8F1FF3F51D145
:10A7B00093691906FCD5638D9BB2FF2B57D953685B
:10A7C000A4F828902B403B4343EA0A035360CBE7AD
:10A7D0004FF4007363640120BDE8F88F0220BDE8E8
:10A7E000F88F636C002243F020032021636484F817
:10A7F000402084F8411084F842200120BDE8F88F01
:10A800009369180699D4FEF7BFF9801B804552D38F
:10A81000B8F1000F4FD0226889E753682C490B40EC
:10A820003B4343F0FF7343F48033FF2121855360A2
:10A8300094E723684FEA19229A624146324620463D
:10A84000FFF712FD00283FF46EAF002384F840307C
:10A850000120C1E793691B06ADD4FEF795F9801B73
:10A860008045BED3B8F1000FBBD022689DE7638D51
:10A870009BB22385D9B253682B403B4343EA014343
:10A8800043F0007353606FE70120A5E7324641466D
:10A890002046FFF7C5FD0028F6D123680D4D202185
:10A8A000D9615A682A405A6084F8411084F84000FF
:10A8B00084F8420090E7636C20210B43002263641C
:10A8C00084F8411084F84220BFE700BF009800FCE4
:10A8D000009C00FC00E800FE0000FF012DE9F047AD
:10A8E000984690F84130BDF824A00A9D202B40F0F6
:10A8F000A680089B0446002B00F09B80BAF1000F55
:10A9000000F0978090F84030012B00F098800123F0
:10A9100080F840300F469146FEF736F9064604E0CF
:10A92000FEF732F9801B192874D82368986910F44F
:10A930000040F5D1089A6262222284F84120402228
:10A9400084F842206064A4F82AA05A6878496063B9
:10A950000A405FFA88F142EA0142C7F309073A4325
:10A9600042F400525A60294632462046FFF77CFCEA
:10A97000002840F0A980B8F1010F40F099802268CA
:10A980005FFA89F39362681C5CD193695906FCD520
:10A99000638D9BB2FF2B7FD8638D65489BB2238567
:10A9A000D9B2536803403B4343EA014343F0007389
:10A9B00043F410535360681CDFF87C81DFF87CA1FE
:10A9C0004FF0FF091CD193695907FCD5636A526A9D
:10A9D0001A70638D626A013B9BB263850132238DDD
:10A9E0006262628D013B9BB292B223850AB1002B59
:10A9F0003ED0638D9BB2002B79D0681C2268E2D0D8
:10AA000093695B07E2D4FEF7BFF8801B854201D350
:10AA1000002DF2D1636C002243F0200320216364F7
:10AA200084F8402084F8411084F842200120BDE8D9
:10AA3000F0874FF4007363640120BDE8F0870220C3
:10AA4000BDE8F08793695B06A2D4FEF79DF8801BF2
:10AA5000854260D3002D5ED0226894E793691B067F
:10AA60000CD4FEF791F8801B8542D3D3002DD1D0B2
:10AA7000681C2268F2D193691906FCD5638D9BB2DC
:10AA8000FF2B26D95368A4F8289003EA08033B4318
:10AA900043EA0A035360ACE7536825490B403B4344
:10AAA00043F0FF7343F49233FF212185536082E723
:10AAB00023684FEA19229A62294632462046FFF758
:10AAC000D3FB00283FF45BAF002384F84030012023
:10AAD000B3E7638D9BB22385D9B2536803EA0803B9
:10AAE0003B4343EA014343F00073536081E732463E
:10AAF00029462046FFF794FCB8B923680D4D202164
:10AB0000D9615A682A405A6084F8411084F840009C
:10AB100084F8420091E7636C20210B4300226364B8
:10AB200084F8411084F84220CEE7012085E700BF79
:10AB3000009800FC00E800FE009C00FC0000FF0103
:10AB40002DE9F04782B005460020019095F84100BC
:10AB500020284CD12C681E46A36913F4004346D12B
:10AB6000914695F84020012A41D00122C1F3090AFB
:10AB70004AF0007A85F84020242285F84120C1F36C
:10AB800009084AF4005A6B64EB68012B0CBF53466A
:10AB900048F420536360FDF7F7FF2C68A269A369AE
:10ABA00002F0200203F01003134307462BD1711C5F
:10ABB00021D04EB948E02C68A269A36902F02002B6
:10ABC00003F0100313431ED1FDF7DEFFC01BB0429C
:10ABD000F1D9202385F841306B6C002243F020032B
:10ABE00001206B6485F8402002B0BDE8F0870220A8
:10ABF00002B0BDE8F087A369A16903F0200301F06A
:10AC000010010B43F7D0A369DA0650D5721C10D19E
:10AC1000A3699B06FCD51023E3612023E361019B1C
:10AC20004B4514D0019B01330193019B4B45ABD3A2
:10AC3000CFE7A3699806EED4FDF7A6FFC01B8642B6
:10AC40001CD3DEB12C68E1E7FDF79EFFC1E7636826
:10AC500043F480436360711C05D1A3699A06FCD557
:10AC60002023E361DEE7A3699B06F9D4FDF78CFF9F
:10AC7000C01B864202D30EB12C68ECE76B6C00223D
:10AC800043F0200320216B6485F8402085F84110B3
:10AC9000012085F84220ABE7A36999060CD4FDF7A3
:10ACA00073FFC01B8642E9D3002EE7D02C68731CCB
:10ACB000F2D1A3699806FCD520220023E261184650
:10ACC00085F8412085F8403092E700BF90F8412098
:10ACD000202A23D15FFA82FC90F84020012A034603
:10ACE0001CD00268242000B583F84100106820F0D1
:10ACF00001001060106820F480501060106801435B
:10AD0000116011684FF0000E41F00101116083F8ED
:10AD100041C083F840E070465DF804FB02207047B4
:10AD200090F84120202A22D100B55FFA82FE90F8E7
:10AD30004020012A03461CD00268242083F84100E9
:10AD4000106820F001001060106820F4706040EA84
:10AD50000121116011684FF0000C41F001011160F8
:10AD600083F841E083F840C060465DF804FB0220B0
:10AD7000704702205DF804FB00287FD030B590F8C2
:10AD80003A30052B83B0044657D090F83A30022B66
:10AD900053D03B4B1A6E42F001021A661B6E03F051
:10ADA00001030193019B90F83A3003F0FF020BB9C5
:10ADB00080F839202046FCF7E7FCA3682168E06AA8
:10ADC00023F02002402A0A6822F0100242EA000220
:10ADD0000A6035D008682B4A656A02406068034300
:10ADE000E0680343206903432B43A56A207D2B437E
:10ADF000256B43EAC543656B012843EA05630CBF35
:10AE00004FF480700020134303430B608B69002BC9
:10AE100009DBD4E906308A690343206A22F03F0245
:10AE2000034313438B6194F83A3003F0FF0013BBE4
:10AE3000012384F83A3003B030BD012003B030BDA7
:10AE40000A681048656A1040626813432269134318
:10AE50002B43A56A227D2B43256B43EAC543656BD3
:10AE6000012A43EA05630CBF4FF4807200220343BA
:10AE700013430B60CAE7002003B030BD01207047C8
:10AE800000100240113E00E0034638B190F83A202D
:10AE9000052A03D090F83A20012A01D001207047FA
:10AEA00001680A684FF0040C42F001020A600020B9
:10AEB00083F83AC0704700BF034658B190F83A2073
:10AEC000052A07D090F83A20022A03D090F83A20B9
:10AED000042A01D00120704701680A684FF0010C74
:10AEE00022F001020A60002083F83AC0704700BFD8
:10AEF000002800F0818010B590F83D30044603F042
:10AF0000FF02002B6DD022683C49022384F83D30BB
:10AF10008A42136851D0B2F1804F21D0A1F594310B
:10AF20008A421DD001F580618A4219D001F596311F
:10AF30008A4242D001F540618A4257D001F58061D2
:10AF40008A4253D001F580618A424FD0A069E168FE
:10AF500023F08003034313606368D162936210E0BF
:10AF6000A168206923F070030B4323F44073A169A7
:10AF7000034323F08003E0680B4361681360D062F1
:10AF800091620123536184F8483084F83E3084F89C
:10AF90003F3084F8403084F8413084F8423084F8FF
:10AFA000433084F8443084F8453084F8463084F8DF
:10AFB000473084F83D30002010BDA068216923F09F
:10AFC0007003034323F440730B43A16923F0800310
:10AFD0000B431360E368D36263689362636913632E
:10AFE000CFE780F83C20FCF71FFC8CE72069A169C3
:10AFF00023F440730343E9E701207047002C01402C
:10B0000090F83D30012B1FD10368154A022193426D
:10B0100080F83D101AD0B3F1804F17D0A2F59432CA
:10B02000934213D002F5806293420FD002F596321C
:10B0300093420BD002F54062934207D01A6842F067
:10B04000010200201A607047012070479968054A84
:10B050000A40062A02D0B2F5803FEFD100207047A7
:10B06000002C0140070001000368196A41F2111227
:10B07000114208D1196A44F24442114203D11A68BC
:10B0800022F001021A60012380F83D300020704751
:10B0900090F83D30012B22D103681749022280F835
:10B0A0003D20DA688B4242F00102DA6019D0B3F138
:10B0B000804F16D0114A934213D002F5806293421A
:10B0C0000FD002F5963293420BD002F540629342C4
:10B0D00007D01A6842F0010200201A607047012070
:10B0E00070479968064A0A40062A02D0B2F5803FA6
:10B0F000EFD10020704700BF002C01400004004049
:10B100000700010090F83C30012B00F0898070B4FA
:10B110000223046880F83D30012280F83C20A568B5
:10B120005F4B2B40A3600B68702B00F0A88028D8E1
:10B13000502B78D03ED9602B1AD1CB684D68216A4C
:10B1400021F010012162A26922F4704242EA033226
:10B15000236AA26123F0A00343EA05132362A368D4
:10B1600023F4401323F0700343F067030022A3602D
:10B170000121002380F83D1080F83C3070BC10465F
:10B180007047B3F5005F69D038D946498B4206D085
:10B190002DD945498B4202D030318B42E8D1A1688C
:10B1A00021F4401121F070010B4343F0070300220A
:10B1B000A360DDE7402B26D14A68CE68216A256A64
:10B1C00025F001052562A36921F00A0123F0F003AF
:10B1D000114343EA0613A3612162A36823F44013D9
:10B1E00023F0700343F047030022A360C0E7B3F1EC
:10B1F000101FD4D010398B42D1D0B9E7B3F58052AB
:10B2000018BF0122B4E7B3D8202BC8D003D9302B04
:10B21000C5D00122ACE733F01002C0D00122A7E76D
:10B220000222104670474A68CE68216A256A25F0D6
:10B2300001052562A36921F00A0123F0F0031143FF
:10B2400043EA0613A3612162A36823F4401323F0A9
:10B25000700343F057030022A36089E7D1E901534B
:10B26000A268C9682B4322F47F4243EA01231343B7
:10B27000A360A36843F480430022A36078E7D1E988
:10B280000153A268C9682B4322F47F4243EA012399
:10B290001343A360A36843F077030022A36067E72A
:10B2A0008800CEFF3000100040001000704700BF43
:10B2B000704700BF704700BF704700BF03681A693E
:10B2C000910710B5044603D5DA68920700F18A8029
:10B2D0001A69520702D5DA68500770D41A69110743
:10B2E00002D5DA68120758D41A69D10602D5DA688D
:10B2F000D2063ED41A69D00703D5DA68D10700F127
:10B300008A801A69120603D5DA68100600F18B806C
:10B310001A69D10503D5DA68120600F18C801A6922
:10B32000500603D5DA68510600F18D801A6992063D
:10B3300003D5DA68900600F18E801A69D10203D530
:10B34000DA68D20200F18F801A69900203D5DA68B8
:10B35000910200F190801A69520203D5DA68500216
:10B3600000F191801A69110202D5DA6812024AD4FA
:10B3700010BD6FF01001082219612277DB6913F408
:10B38000407F204640F09080FFF790FF2046FFF777
:10B3900091FF002223682277ACE76FF008010422B6
:10B3A00019612277DB699B0720467AD1FFF77EFF80
:10B3B0002046FFF77FFF00222368227794E76FF093
:10B3C00004010222196122779B6913F4407F204611
:10B3D00064D1FFF76BFF2046FFF76CFF0022236864
:10B3E00022777BE76FF002010122196102779B69E6
:10B3F000990750D1FFF75AFF2046FFF75BFF002265
:10B400002368227764E76FF4000220461A61BDE8E2
:10B41000104000F0A3B86FF001021A612046F8F75F
:10B42000C7FF23686DE76FF080021A61204600F0C5
:10B430008BF823686CE76FF480721A61204600F085
:10B4400085F823686BE76FF040021A612046FFF72A
:10B4500033FF23686AE76FF020021A61204600F08C
:10B4600071F8236869E76FF480121A61204600F0D2
:10B470006FF8236868E76FF400121A61204600F045
:10B4800069F8236867E76FF480021A61204600F0CC
:10B4900063F8236866E7FFF70BFFB0E7FFF708FFE5
:10B4A0009CE7FFF705FF86E7FFF702FF71E700BFA4
:10B4B00090F83C30012B3ED070B402681F4D02233F
:10B4C00080F83D30AA425368946828D005F500659D
:10B4D000AA4224D00E6823F0007323F07003334394
:10B4E000B2F1804F53600CD0154B9A4209D003F54E
:10B4F00080639A4205D0AA4203D003F59C339A4256
:10B5000004D18B6824F080041C4394600023012242
:10B5100080F83D2080F83C3070BC184670474D687C
:10B5200023F470032B4323F000730D6823F07003A2
:10B530002B435360E5E70220704700BF002C014019
:10B5400000040040704700BF704700BF704700BF55
:10B55000704700BF704700BF704700BF704700BF13
:10B56000D0F88830202B5ED100295AD0002A58D03C
:10B5700090F88030012B56D030B403685D4C012523
:10B5800080F88050A3424FF00005C5660AD05C6881
:10B59000240207D553E8004F44F0806443E8004597
:10B5A000002DF7D1846881650025B4F5805FA0F88F
:10B5B0005C20A0F85E20056737D0002C7BD10169A4
:10B5C000002951D1FF21A0F8601000242221C0F8E9
:10B5D0008C40C0F8881003F1080151E8001F41F0C9
:10B5E000010103F1080545E80014002CF3D1416E78
:10B5F000B1F1005F3CD08268B2F5805F02691CD077
:10B600003D4C0467002180F88010E2B153E8002F20
:10B6100042F4907243E800210029F7D1002030BCA9
:10B620007047012070470220704701690029C9D185
:10B6300040F2FF11A0F86010C7E7002A41D12F495E
:10B64000016780F8802053E8002F42F0200243E891
:10B6500000210029E2D053E8002F42F0200243E805
:10B6600000210029EFD1D9E77F21A0F86010ACE7D5
:10B67000B0F868109142BED88268B2F5805F026966
:10B680002CD01F49016780F880403AB153E8002F61
:10B6900042F4807243E800210029F7D103F1080247
:10B6A00052E8002F42F0805203F1080040E80021E8
:10B6B0000029F3D1B2E7B4F1805F08D0A0F8605060
:10B6C00083E70D490167002280F880209EE7016929
:10B6D0000029C9D03F21A0F8601076E722B90949B6
:10B6E000016780F88020D9E7054A026780F880402A
:10B6F000CCE700BF0080004019BD0008D9BC00089D
:10B700005DBD000805BF0008F8B5D0F88460202EA4
:10B7100041D100293DD0002A3BD0044690F880005A
:10B72000012838D0A06FA4F8562000270125212336
:10B73000C4F88C702165A4F8542084F88050C4F8B3
:10B74000843090B1DFF864C0876313462268C0F884
:10B750002CC0DFF85CC0C0F830C0DFF858C0C0F8BB
:10B7600034C02832FEF7F2F8B8B92268402100232D
:10B77000116284F8803002F1080353E8003F43F07F
:10B78000800302F1080040E800310029F3D10020D5
:10B79000F8BD0120F8BD0220F8BD102384F88070A8
:10B7A000C4F88C302846C4F88460F8BDBDB70008E2
:10B7B00005B8000815B80008704700BF08B5036851
:10B7C000806A1B6813F0200317D10268A0F8563076
:10B7D00002F1080353E8003F23F0800302F1080060
:10B7E00040E800310029F3D152E8003F43F0400324
:10B7F00042E800310029F7D108BDFFF7DDFF08BDA1
:10B80000704700BF08B5806AFFF7FAFF08BD00BFA8
:10B81000704700BF806A0368D0F8841010B5D0F874
:10B8200088409A68120601D521290DD09A685206DF
:10B8300001D5222C23D0D0F88C3043F01003C0F86F
:10B840008C30FFF7E5FF10BD0022A0F8562053E82A
:10B85000002F22F0C00243E800210029F7D103F1B4
:10B86000080252E8002F22F4000203F1080C4CE811
:10B8700000210029F3D12022C0F88420D6E700223D
:10B88000A0F85E2053E8002F22F4907243E80021D4
:10B890000029F7D1134C03F1080252E8002F22408F
:10B8A00003F1080C4CE800210029F4D1C26E012AF2
:10B8B00006D000232022C0F888200367C366BAE7B9
:10B8C00053E8002F22F0100243E800210029F0D0B5
:10B8D00053E8002F22F0100243E800210029EFD1A5
:10B8E000E7E700BFFEFFFFEF08B5806A0023A0F87E
:10B8F0005E30A0F85630FFF78BFF08BD704700BFE1
:10B900000368DA6940F60F0C12EA0C0F70B51D6877
:10B910009968044600F0EA809A4E9B4805EA060CB6
:10B9200008405CEA000655D1E06E012822D0D00222
:10B9300002D54E0200F10381100606D501F4000184
:10B9400005F08000014340F0F280510634D56E06C8
:10B9500032D553E8002F22F0400243E800210029AD
:10B96000F7D120220023C4F8842063672046FFF724
:10B9700023FF70BDD606DAD5E806D8D510221A62A4
:10B980009A68520640F10681E06F01684A6892B2F7
:10B99000002AEED0B4F85C509542EAD9A4F85E20B3
:10B9A0000A68960640F12B81B4F85E10691A2046A9
:10B9B00089B2FFF7A3FF70BD100202D5690000F144
:10B9C000DB80D301D5D5002DD3DA2046BDE8704009
:10B9D00000F01EBED60709D5EE0507D501261E626A
:10B9E000D4F88C6046F00106C4F88C60960740F1EC
:10B9F0008F80CE070AD502261E62D4F88C6046F0EE
:10BA00000406C4F88C60560700F1888016070BD531
:10BA100005F02006304307D008201862D4F88C00C7
:10BA200040F00800C4F88C0010050AD56E0108D556
:10BA30004FF400601862D4F88C0040F02000C4F885
:10BA40008C00D4F88C00002893D090060BD505F01C
:10BA5000200501F0805155EA010204D0226F12B195
:10BA6000204690472368D4F88C509A6805F0280542
:10BA700002F04002154300F0F38053E8002F22F457
:10BA8000907243E800210029F7D1404803F10802F1
:10BA900052E8002F024003F1080545E80021002983
:10BAA000F4D1E26E012A52D000222021C4F888107D
:10BAB000E266996822674A065AD503F1080252E8FD
:10BAC000002F22F0400203F1080040E80021002985
:10BAD000F3D1E06F00284BD02D4B8363FDF7CAFFF5
:10BAE00000283FF446AFE06F836B0EE096067FF5CB
:10BAF0001BAF05F0200601F0805C56EA0C063FF40F
:10BB000013AF036F002B3FF434AFBDE8704018470C
:10BB100056077FF57BAFCE077FF578AF04261E6210
:10BB2000D4F88C6046F00206C4F88C606EE7636F50
:10BB3000002B3FF41EAF2046BDE8704018474FF47D
:10BB4000801220461A62BDE8704000F05FBD53E8E5
:10BB5000002F22F0100243E800210029A4D053E86E
:10BB6000002F22F0100243E800210029EFD19BE7CB
:10BB70002046FFF74DFE70BD2046BDE8704000F046
:10BB800049BD00BF2001000401000010FEFFFFEFCF
:10BB9000E9B80008B4F85E10B4F85E2092B289B239
:10BBA000002A3FF4E6AEB4F85C20511A89B20029AD
:10BBB0003FF4DFAE53E8002F22F4907243E80020F8
:10BBC0000028F7D1294D03F1080252E8002F2A403E
:10BBD00003F1080646E800200028F4D12022C4F82A
:10BBE00088202067E06653E8002F22F0100243E827
:10BBF00000200028F7D12046FFF780FE70BD53E8F3
:10BC0000002F22F4807243E800210029F7D103F1CC
:10BC1000080252E8002F22F0010203F1080545E86E
:10BC200000210029F3D103F1080252E8002F22F08D
:10BC3000400203F1080545E800210029F3D1202244
:10BC4000C4F88820E16653E8002F22F0100243E890
:10BC500000210029F7D1FDF7D3FEB4F85C50A3E62C
:10BC60002046FFF7D5FDC4F88C5070BDFEFFFFEFF6
:10BC700008B5036853E8002F22F4907243E80021CE
:10BC80000029F7D103F1080252E8002F22F0010247
:10BC900003F1080C4CE800210029F3D12022C0F860
:10BCA0008820C26E0167012A12D1C16653E8002FB5
:10BCB00022F0100243E800210029F7D1DA69B0F838
:10BCC0005C10D20644BF10221A62FFF717FE08BDAF
:10BCD000F8F77CFB08BD00BFD0F88820222A026854
:10BCE00004D0936943F0080393617047526AB0F837
:10BCF00060C0816D02EA0C0221F8022BB0F85E20D0
:10BD00008165013A92B2A0F85E20B0F85E309BB235
:10BD1000002BEAD1FFF7ACBFD0F88820222A0268B6
:10BD200004D0936943F0080393617047526AB0F8F6
:10BD300060C0816D02EA0C020A70B0F85E20816D6D
:10BD4000013A92B2A0F85E20B0F85E20013192B2C2
:10BD50008165002AE9D1FFF78BBF00BF2DE9F84FBD
:10BD600002680446D06917689668D4F888102229BA
:10BD700006D01346926942F008029A61BDE8F88F36
:10BD8000B4F86830002B00F0B58085067BD594F8B8
:10BD900060B0DFF86CA107F4807706F001064FF081
:10BDA00000084FF00409526AA36D0BEA02021A70F0
:10BDB000B4F85E102368A26D013989B2A4F85E1050
:10BDC000DD6901326807A2651AD0E90708D53FB1DD
:10BDD00001221A62D4F88C2042F00102C4F88C20AF
:10BDE000AA0715D54EB102221A62D4F88C20680732
:10BDF00042F00402C4F88C200ED4D4F88C30BBB9C5
:10BE0000B4F85E309BB2EBB1AB063CD52268CAE712
:10BE10006907F2D5002EF0D0C3F82090D4F88C300A
:10BE200043F00203C4F88C30D4F88C30002BE7D0F8
:10BE30002046FFF7EDFCC4F88C80B4F85E309BB26E
:10BE4000002BE1D1236853E8002F22F4807243E8ED
:10BE500000210029F7D103F1080252E8002F02EA7D
:10BE60000A0203F1080040E800210029F3D1202252
:10BE7000C4F88820E26E2167012A27D02046F8F70F
:10BE8000A5FAAB06C2D4B4F85E309BB2002B3FF4E7
:10BE900075AFB4F868209A427FF670AF236803F15B
:10BEA000080252E8002F22F0805203F1080040E817
:10BEB00000210029F3D1114A226753E8002F42F0F4
:10BEC000200243E800210029F7D157E7E16653E853
:10BED000002F22F0100243E800210029F7D1DA698F
:10BEE000B4F85C10D20644BF10221A622046FFF755
:10BEF00005FD89E7B4F85E3040E700BF19BD0008D2
:10BF0000FEFFFFEF2DE9F84F0368D9691E689D68B1
:10BF1000D0F88820222A05D09A6942F008029A6156
:10BF2000BDE8F88FB0F868208346002A00F0BB8097
:10BF30008C067ED5B0F860A0DFF8749106F48076A8
:10BF400005F0010500274FF004085A6ADBF8581085
:10BF50000AEA020221F8022BBBF85E20CBF8581047
:10BF6000013A92B2ABF85E20DC6960071AD0E107B3
:10BF700008D53EB101221A62DBF88C2042F00102A2
:10BF8000CBF88C20A20716D54DB102221A62DBF83D
:10BF90008C20600742F00402CBF88C200FD4DBF831
:10BFA0008C30C3B9BBF85E309BB2F3B1A30640D569
:10BFB000DBF80030C9E76107F1D5002DEFD0C3F8F9
:10BFC0002080DBF88C3043F00203CBF88C30DBF8B8
:10BFD0008C30002BE6D05846FFF71AFCCBF88C705B
:10BFE000BBF85E309BB2002BE0D1DBF8003053E8A9
:10BFF000002F22F4807243E800210029F7D103F1D9
:10C00000080252E8002F02EA090203F1080040E8A2
:10C0100000210029F3D12022CBF88820DBF86C2006
:10C02000CBF87010012A29D05846F8F7CFF9A306AB
:10C03000BED4BBF85E309BB2002B3FF471AFBBF8AF
:10C0400068209A427FF66CAFDBF8003003F10802FB
:10C0500052E8002F22F0805203F1080040E800214E
:10C060000029F3D1114ACBF8702053E8002F42F099
:10C07000200243E800210029F7D151E7CBF86C10EA
:10C0800053E8002F22F0100243E800210029F7D1E5
:10C09000DA69BBF85C10D20644BF10221A62584617
:10C0A000FFF72CFC82E7B0F85E3039E7D9BC000816
:10C0B000FEFFFFEF38B504460368826800696169D6
:10C0C0001D6802430A43E069A649024329400A4326
:10C0D0001A605A68E16822F440520A43A2495A6041
:10C0E0008B42A26999686BD0256A21F06E4121F4D8
:10C0F00030612A430A439A60DA6A616A22F00F02C9
:10C100000A43DA62994A934212D0994A934236D04E
:10C11000984A934200F0FA80974A934200F0A58033
:10C12000012000234FF00112C4E91C33A26638BD80
:10C13000924BD3F8883003F00303013B022B40F20B
:10C140008E80B0F5004F00F0FE80FDF70DF900285D
:10C1500000F0DA80616A6268894B33F81130B0FB15
:10C16000F3F04FF6EF7100EB5203B3FBF2F3A3F1E0
:10C1700010028A42D4D822680020D360D1E77F4BD6
:10C18000804AD3F8883003F00C03D35CB0F5004F3D
:10C190007DD0082BC4D801A252F823F0C7C20008F2
:10C1A0004BC1000843C3000821C1000889C2000830
:10C1B00021C1000821C1000821C1000833C30008C3
:10C1C00021F06E4121F430610A439A60DA6A616AB3
:10C1D0006A4822F00F020A43DA62D0F8883003F48A
:10C1E0004063B3F5006F00F0AA800BD8002B39D064
:10C1F000B3F5806F94D1FCF755FF002800F08480E0
:10C20000616A04E0B3F5406F8AD14FF400405C4BA3
:10C21000656833F81120B0FBF2F305EB4501994254
:10C220003FF67EAFB3EB053F3FF67AAF00231946EA
:10C23000F7F7F2FE0902030241EA106168081818D4
:10C240002A464FF0000341F10001F7F7E5FE4E4AA0
:10C25000A0F54071914203463FF662AF8BE74B4A2F
:10C26000D35C93E7FDF76EF8C7E7444BD3F888300B
:10C2700003F0C003802B6ED05ED80BB3402B7FF44D
:10C280004FAFB0F5004F21D0FCF70CFF5FE7082B54
:10C290003FF646AF01A252F823F000BF4DC300089D
:10C2A00047C3000853C3000821C10008CDC20008DD
:10C2B00021C1000821C1000821C10008D5C2000821
:10C2C000B0F5004F42D0FDF73DF840E7FCF7EAFE3D
:10C2D000D0B1616A62682A4B33F81110B0FBF1F0FB
:10C2E000530803EB40004FF6EF73B0FBF2F0A0F100
:10C2F00010029A423FF614AF20F00F0322689BB25F
:10C30000C0F342001843D06000200AE71B4BD3F86B
:10C31000883003F03003202B1DD004D8002BCFD061
:10C32000102BAED0FCE6302B7FF4FAAEB0F5004F08
:10C33000D0D04FF400400EE7C02BF7D0F0E6144801
:10C3400065E7134807E7FDF70FF8C1E7FCF7FAFFC9
:10C35000BEE70F48BEE7B0F5004F0D487FF4FBAED7
:10C36000B8E700BFF369FFCF00800040003801400C
:10C370000044004000480040004C004000100240D3
:10C38000D4CE0008C4CE0008FFFC0F00C0CE0008C9
:10C390000024F400836ADA0710B406D50168C46A81
:10C3A0004A6822F4003222434A609C0706D501689D
:10C3B000046B4A6822F4803222434A60590706D54A
:10C3C0000168446B4A6822F4802222434A601A07BB
:10C3D00006D50168846B4A6822F4004222434A6011
:10C3E000DC0606D50168C46B8A6822F480522243B9
:10C3F0008A60990606D50168046C8A6822F40052A6
:10C4000022438A605A0609D50168446C4A6822F4BE
:10C4100080122243B4F5801F4A600BD01B0606D55C
:10C420000268C16C536823F400230B4353605DF82A
:10C43000044B70474A68846C22F4C00222434A606D
:10C44000ECE700BF2DE9F843DDF8208004680746DB
:10C450000E4615469946B8F1FF3F0AD1E36936EA20
:10C4600003030CBF012300239D42F7D00020BDE849
:10C47000F883E36936EA03030CBF01230023AB42D0
:10C48000F4D1FCF781FBA0EB0900404533D8B8F1AB
:10C49000000F30D03C68236859072246DBD5E3699A
:10C4A0001B05D8D54FF40063236254E8003F23F402
:10C4B000D07344E8003139B152E8003F23F4D0731F
:10C4C00042E800310029F7D102F1080353E8003FA8
:10C4D00023F0010302F1080040E800310029F3D104
:10C4E0002023C7F8843087F88010C7F888300320ED
:10C4F000C7F88C30BBE73A6852E8003F23F4D073AA
:10C5000042E800310029F7D102F1080353E8003F67
:10C5100023F0010302F1080040E800310029F3D1C3
:10C520002023C7F8843087F88010C7F888300320AC
:10C530009DE700BF002866D070B5D0F8843082B087
:10C540000446002B4CD022682423C4F8843013689E
:10C5500023F0010320461360FFF7ACFD01283CD017
:10C56000A36A002B35D12368596821F490415960A2
:10C57000996821F02A0199601968002541F00101AC
:10C580001960C4F88C50FCF7FFFA23681A68120788
:10C5900006460ED41B685B0727D400232022C4F86C
:10C5A000842084F88030C4F888201846E36602B0FE
:10C5B00070BD6FF07E4300932A4603464FF400118E
:10C5C0002046FFF73FFFE0B923681B685B070CD4E8
:10C5D000E3E72046FFF7DEFEC5E7012002B070BDAD
:10C5E00080F88030FBF766F9ADE76FF07E4300938B
:10C5F000002233464FF480012046FFF723FF002836
:10C60000CBD00320D3E70120704700BF704700BFA5
:10C61000704700BF704700BF90F88030012B17D0E3
:10C620000268242310B4C0F8843011681468002311
:10C6300024F0010421F0005114604366116080F879
:10C6400080302022C0F884205DF8044B18467047E3
:10C650000220704790F88020012A37D003460268F4
:10C66000242030B5C3F884001468106820F001005D
:10C670001060906820F060400143586E916010B3E4
:10C6800091689068124DC1F3426C4FEA507E114997
:10C6900011F80E0011F80C1015F80EE015F80C50FA
:10C6A000C000C900B0FBFEF0B1FBF5F1A3F86810C3
:10C6B0000021A3F86A002025146083F88010084642
:10C6C000C3F8845030BD01210846EFE702207047CF
:10C6D000ECCE0008F4CE000890F88020012A37D074
:10C6E00003460268242030B5C3F88400146810683B
:10C6F00020F001001060906820F060600143586EE7
:10C70000916010B391689068124DC1F3426C4FEA8A
:10C71000507E114911F80E0011F80C1015F80EE0BA
:10C7200015F80C50C000C900B0FBFEF0B1FBF5F1EC
:10C73000A3F868100021A3F86A002025146083F88C
:10C7400080100846C3F8845030BD01210846EFE749
:10C7500002207047ECCE0008F4CE0008054BD3F859
:10C7600088204FF0006142F47002C3F8882099607D
:10C77000704700BF00ED00E0F8B51646DDE906722F
:10C78000B2FBF6F406FB14246CB943604B1E05465D
:10C790001A444180920021463846F3F743FE2E703A
:10C7A000AF602046F8BD6FF00100F8BD2DE9F04FF5
:10C7B00089B0B0F8029000920278846840680694CC
:10C7C00009F18046013E9A42049004EB8606204619
:10C7D0000292B3FBF2F4079400F29680A2F10208F1
:10C7E0004FEA5808134608F101084FEA820A013B54
:10C7F0004FEA480205924FEAC80701948346039323
:10C80000039A0B1D9E4218BF0B2A60D941EA06030A
:10C810005A075CD1A1F1080032460023F0E9024535
:10C8200001334345E2E80245F8D3029B059A93425F
:10C8300001D0CB59F35151445644B9F1000F54D0B3
:10C840000023DDF810E04A46DC461D465CF8044B48
:10C850005EF8040B013AC4FB0035F7D1DB0F43EA65
:10C860004503009A42F8043B019B0092013BD344EC
:10C870000193C5D1DDE9063202FB0A3AB9F101069E
:10C8800022D006990AF10402A9F10203914218BFCD
:10C890000B2B2CD941EA0A035B0728D1A9F103032A
:10C8A0005B080133AAF108000022F0E902450132D9
:10C8B0009A42E1E80245F8D3B6EB430F04D006995B
:10C8C0005AF8332041F8332009B0BDE8F08F029BBD
:10C8D000301F0A4652F8044B40F8044F013BF9D18F
:10C8E00051445644B9F1000FAAD14B46B9E7069B13
:10C8F000043B00E0043252F8041C43F8041F013EDC
:10C90000F8D109B0BDE8F08FDDF818A0B6E700BF98
:10C9100010B504460298218000F1FF3C8C44A260CF
:10C9200000214FEA8C021846F3F77CFD606010BDD1
:10C930002DE9F04F83B0D0F804B0078884680093E5
:10C94000002B5DD007F180400138800004380BEBEC
:10C95000000AD846CDF804B09946A34651F8040B16
:10C960004AF8040F00233846DE46C4461E465CF8EB
:10C97000045B5EF8044B0138C5FB0436F7D1DB0FCE
:10C9800043EA4603B9F1010942F8043B08F10408FF
:10C99000E4D1DDE9003B0BEB8306B7F1010C1ED0BF
:10C9A000331DBA1E9B4518BF0B2A1BD94BEA060242
:10C9B000520717D1FB1E5B080133A6F10800594648
:10C9C0000022F0E9024501329A42E1E80245F8D33B
:10C9D000BCEB430F03D056F833204BF8332003B0A1
:10C9E000BDE8F08FABF1040B00E0043353F8042CE6
:10C9F0004BF8042FBCF1010CF7D103B0BDE8F08F68
:10CA00005E46CAE700285ED0F0B590F8A93287B03C
:10CA1000044603F0FF02002B50D00323206884F863
:10CA2000A93200F073F865685DB300234FF0010E82
:10CA3000184603EB830104EBC10203F1010C82F8F9
:10CA40002830D3865FFA8CF3AB42C2E90E0082F83D
:10CA500029E082F82B001064EBD30022114602EB90
:10CA6000820304EBC303501C83F86821C2B2AA42BC
:10CA7000C3E95E1183F8691183F86B11C3F8801163
:10CA8000EDD32546EC4655F8107B0FCDACE80F00F2
:10CA90002B68CCF8003004F1040E9EE80E003846F6
:10CAA00000F03EF8E36901220026934284F82460F6
:10CAB00084F8A92209D0304607B0F0BD80F8A8223A
:10CAC000FAF762FFA9E701207047204600F004F85A
:10CAD000304607B0F0BD00BF0268002110B480F8F6
:10CAE000E012B2F8543001249BB22343C0F8E8426C
:10CAF000A2F85430B2F854305DF8044B9BB243F0C6
:10CB000002030846A2F85430704700BFB0F8401046
:10CB1000034644F27F020A400020A3F840207047F9
:10CB200084B0844601A880E80E0000200123ACF800
:10CB3000403004B0ACF84000ACF84400ACF8500011
:10CB4000704700BF0D4885460D480E490E4A002328
:10CB500002E0D458C4500433C4188C42F9D30B4AB1
:10CB60000B4C002301E013600432A242FBD3FFF719
:10CB7000F5FDF3F789FBF7F75BFDFEE7008000208A
:10CB8000000000207007002060CF00087007002020
:10CB90004C530020FEE70000F8B500BFF8BC08BC0D
:10CBA0009E467047F8B500BFF8BC08BC9E4670476B
:10CBB000FB21F93FFB2109407CD91240FB211940A0
:10CBC0007A6A1F407CD92240BBFD2540FB212940C9
:10CBD0003A462C407A6A2F405C4731407CD932403B
:10CBE0009C6B3440BBFD3540DB8F3740FB21394027
:10CBF0001BB43A403A463C405AD83D407A6A3F40DE
:10CC00004C7E40405C4741406C1042407CD94240E1
:10CC10008CA243409C6B4440AC344540BBFD454036
:10CC2000CBC64640DB8F4740EB584840FB2149408C
:10CC300083F9A200444E6E00FC291500D15727004D
:10CC4000DD34F50062DBC0003C9995004190430063
:10CC50006351FE00BBDEAB00B761C5003A6E240035
:10CC6000D24D42004906E00009EA2E001C92D10094
:10CC7000EB1DFE0029B11C00E83EA700F53582003F
:10CC800044BB2E009CE98400B4267000417E5F0006
:10CC9000D6913900538339009CF439008B5F8400AE
:10CCA00028F9BD00F81F3B00DEFF97000F98050034
:10CCB000112FEF000A5A8B006D1F6D00CF7E3600DA
:10CCC00009CB2700464FB7009E663F002DEA5F0064
:10CCD000BA277500E5EBC7003D7BF100F739070087
:10CCE00092528A00FB6BEA001FB15F00085D8D0065
:10CCF000300356007BFC4600F0AB6B0020BCCF003D
:10CD000036F49A00E3A91D005E619100081BE6005D
:10CD100085996500A0145F008D40680080D8FF00F1
:10CD200027734D0006063100CA561500C9A87300C6
:10CD30007BE260006B8CC00002000000030000007A
:10CD4000040000000600000000000040FB21F93F45
:10CD5000000000002D44743E000000809846F83C1E
:10CD60000000006051CC783B00000080831BF0394C
:10CD70000000004020257A38000000802282E3363F
:10CD8000000000001DF36935000000000000304382
:10CD900000000000000030C3252A6C640000000081
:10CDA000252A730025386C640000000025730000FC
:10CDB0001B5B25642C25647A000000002564202577
:10CDC0002D31327300000000545820534554204D3B
:10CDD000454D204E4F0000003E0000000C000000BA
:10CDE0001B5B2564620000001B5B3630302C357104
:10CDF000000000001B5B3132382C3132372C302CD4
:10CE0000302C302C302C3063000000001B5B3132A2
:10CE1000392C3132372C3132372C302C302C302C0D
:10CE2000306300001B5B3133302C3132372C313210
:10CE3000372C3132372C302C302C3063000000007E
:10CE40001B5B3133312C3132372C3132372C3132BC
:10CE5000372C3132372C302C306300001B5B3133E0
:10CE6000322C3132372C3132372C3132372C3132AF
:10CE7000372C3132372C3063000000001B5B31331C
:10CE8000332C3132372C3132372C3132372C31328E
:10CE9000372C3132372C3132376300001B5B25646D
:10CEA000730000001B5B3135302C313030710000D5
:10CEB0005054540053455400424C00002B000000D5
:10CEC00004020800001010100410101002101010BE
:10CED00008000000010002000400060008000A002B
:10CEE0000C00100020004000800000010804020433
:10CEF0000801010101010103070100000000000019
:10CF000000000000010203040607080900000000F9
:10CF100001020304232D302B20000000686C4C001C
:10CF20006566674546470000303132333435363761
:10CF30003839414243444546000000003031323325
:10CF40003435363738396162636465660000000045
:08CF5000F870FF7F01000000F2
:04CF58006902000862
:04CF5C004102000886
:10CF6000040000200000000000000000000000009D
:10CF700000000000000000000000000000000000B1
:10CF800000000000000000000000000000000000A1
:10CF90000000000000000000000000000000000091
:10CFA0000000000000000000000000000000000081
:10CFB0000000000000000000000000000000000071
:10CFC00000000000FF000000D03AFDFF000000005C
:10CFD00054183400000000002A04FFFE0000000086
:10CFE000A9A5D00400000008A9A5D00400000000F5
:10CFF0002A04FFFE00000000541834000000000066
:10D00000D03AFDFFD9D0EEFFA2D1EFFFBAB9F0FFC1
:10D01000C297F1FF5B7CF2FF037AF3FFF4A4F4FF05
:10D02000F512F6FF2EDBF7FFEE15FAFF75DCFCFFBD
:10D03000B1480000FE740400E37B0900C3770F00D1
:10D0400099821600AEB51E004929280067F4320007
:10D05000732C3F00FBE44C006E2F5C00DA1A6D006D
:10D06000ACB37F007B039400D310AA0006DFC1009D
:10D07000096EDB0052BAF600C0BC13018A6A3201A5
:10D0800038B55201A28A7401F7D49701D27ABC0153
:10D090004D5FE20128620902F15F310231325A022A
:10D0A000AEAF8302A2ACAD0208FBD702E66A020370
:10D0B0009ECA2C0348E756030C8D80037E87A90384
:10D0C00001A2D1032AA8F80320661E0400A9420485
:10D0D000413F650412F98504BAA8A404EC22C104F6
:10D0E000253FDB04F6D7F20451CB0705CEFA19052C
:10D0F000E64B29052CA8350576FD3E05033E450582
:10D100009B6048059B604805033E450576FD3E054E
:10D110002CA83505E64B2905CEFA190551CB070594
:10D12000F6D7F204253FDB04EC22C104BAA8A4041C
:10D1300012F98504413F650400A9420420661E04DB
:10D140002AA8F80301A2D1037E87A9030C8D8003CE
:10D1500048E756039ECA2C03E66A020308FBD7027F
:10D16000A2ACAD02AEAF830231325A02F15F31029E
:10D17000286209024D5FE201D27ABC01F7D497011F
:10D18000A28A740138B552018A6A3201C0BC130107
:10D1900052BAF600096EDB0006DFC100D310AA0008
:10D1A0007B039400ACB37F00DA1A6D006E2F5C0035
:10D1B000FBE44C00732C3F0067F43200492928003F
:10D1C000AEB51E0099821600C3770F00E37B0900FD
:10D1D000FE740400B148000075DCFCFFEE15FAFF98
:10D1E0002EDBF7FFF512F6FFF4A4F4FF037AF3FF4A
:10D1F0005B7CF2FFC297F1FFBAB9F0FFA2D1EFFF5B
:10D20000D9D0EEFF4681FEFFD01E05008FE20B0055
:10D21000A4A2120044231900D7101F00ACFD230064
:10D220003964270089AE2800D34227007F9422006A
:10D230004F381A00C0F90D0053EFFDFF408BEAFF95
:10D240000BA6D4FFC780BDFF62BDA6FF164C92FFA0
:10D25000014E82FF11EE78FF4E3278FFC5C881FF84
:10D26000DBD396FF9DBAB7FF9901E4FFD2301A00D5
:10D2700098CA57004A5699009880DA005C51160106
:10D280007375470137996801A9CE7401FFF86701EA
:10D290003B363F01F53EF90086B4960055561A001C
:10D2A0003C1889FFA115EAFE085F46FE52A2A8FDC0
:10D2B00057B01CFD3CE5AEFC047B6BFCE7CF5DFC8E
:10D2C00060AB8FFC708D08FDCD13CDFD987FDEFE29
:10D2D000F1643A00538BDA01FA02B5035E70BC05C3
:10D2E000918BE007FCCD0E0AF345330C1585390E02
:10D2F0007E9C0D10B9189D111AEFD712CE4EB113A6
:10D300007B4920147B492014CE4EB1131AEFD7125B
:10D31000B9189D117E9C0D101585390EF345330CFF
:10D32000FCCD0E0A918BE0075E70BC05FA02B503D6
:10D33000538BDA01F1643A00987FDEFECD13CDFD08
:10D34000708D08FD60AB8FFCE7CF5DFC047B6BFC50
:10D350003CE5AEFC57B01CFD52A2A8FD085F46FE9E
:10D36000A115EAFE3C1889FF55561A0086B49600AE
:10D37000F53EF9003B363F01FFF86701A9CE740185
:10D3800037996801737547015C5116019880DA007E
:10D390004A56990098CA5700D2301A009901E4FF02
:10D3A0009DBAB7FFDBD396FFC5C881FF4E3278FF29
:10D3B00011EE78FF014E82FF164C92FF62BDA6FF70
:10D3C000C780BDFF0BA6D4FF408BEAFF53EFFDFFE4
:10D3D000C0F90D004F381A007F942200D342270075
:10D3E00089AE280039642700ACFD2300D7101F0048
:10D3F00044231900A4A212008FE20B00D01E0500E6
:10D400004681FEFF0020204672657175656E637966
:10D41000000000000901000064000000E8030000B3
:10D42000F0B31A00010000000020487A000000005C
:10D43000881700202D4F0008355A000800202020B2
:10D44000566F6C756D65202000000000050200001D
:10D4500001000000000000002000000000000000AB
:10D46000007C000000000000EC3E0020E94F0008B6
:10D47000B159000800202020204761696E2020203B
:10D480000000000001020700010000000100000090
:10D49000060000000000000000780000000000000E
:10D4A000CC1C002021450008FD58000800204D6FCD
:10D4B00064756C6174696F6E0000000003020A00FD
:10D4C0000100000000000000060000000100000054
:10D4D0000000000000000000941B0020894F00089D
:10D4E0006D590008012046696C746572204346201E
:10D4F00000000000040100003200000032000000C3
:10D50000AC0D0000000000000020487A0000000080
:10D5100084170020D9580008FD58000801204669EA
:10D520006C74657220425720000000000402000065
:10D530003200000032000000C409000000000000BA
:10D540000020487A0000000080170020D958000809
:10D55000FD580008012046696C7465722051202036
:10D5600000000000020300000100000001000000B4
:10D57000200000000000000000205100000000001A
:10D580007C170020D9580008FD580008FF202020F3
:10D590005369676E616C2020000000040D040000D8
:10D5A0000000000000000000000000000053000028
:10D5B0000000000000000000D01C0020E94F00081F
:10D5C000B1590008FF2020205458207461622020A7
:10D5D000000000040305000000000000000000003F
:10D5E000000000000000000000000000000000003B
:10D5F000B0CE0008E94F000835590008FF20202070
:10D600005461627320202020000000040305040000
:10D61000000000000000000000000000000000000A
:10D620000000000000000000B4CE0008E94F000830
:10D6300035590008FF2020205461627320202020EB
:10D6400000000004020509000000000000000000C6
:10D6500000000000000000000000000000000000CA
:10D66000B8CE0008E94F000835590008FF202020F7
:10D6700054616273202020200000000401050C008A
:10D68000000000000000000000000000000000009A
:10D690000000000000000000BCCE0008E94F0008B8
:10D6A000355900080C000000444300004C53420070
:10D6B0005553420043574C0043575500414D00001D
:10D6C000464D000001000000100000000024F4009E
:040000050800CB45DF
:00000001FF
